:020000040000FA
:107800005469616E59696E673130300000000000C4
:1078100054593230302E303830303030625F747925
:10782000424154333247313339474B3634464200B4
:1078300043414E5F5354440000000000000000002C
:1078400043414E5F43485F300000000000000000ED
:1078500043414E5F3530304B6270730000000000D2
:107860009407000014070000DF070000000000007C
:020000040000FA
:10800000A02F0020E9800000F1800000F380000034
:108010000000000000000000000000000000000060
:10802000000000000000000000000000FB800000D5
:108030000000000000000000FF80000039CF0100B8
:10804000A1150100E51501001516010045160100F6
:1080500075160100A5160100D516010005170100CF
:10806000351701006517010099170100AD170100D0
:10807000BD170100F11701000118010011180100DE
:108080004518010089180100D118010019190100D3
:1080900061190100A9190100B9190100ED190100C8
:1080A000211A0100511A0100851A0100B91A0100B4
:1080B000C91A0100D91A01000D1B0100411B010062
:1080C000EF72E8FF03B40148019001BD897F0020F1
:1080D0000448854600F0C6F900480047E510020054
:1080E000C046C046A02F00201648804716480047CB
:1080F000FEE7FEE7FEE7FEE7FEE7FEE7FEE7FEE758
:10810000FEE7FEE7FEE7FEE7FEE7FEE7FEE7FEE747
:10811000FEE7FEE7FEE7FEE7FEE7FEE7FEE7FEE737
:10812000FEE7FEE7FEE7FEE7FEE7FEE7FEE7FEE727
:10813000FEE7FEE7FEE7FEE7FEE7FEE7FEE7FEE717
:10814000FEE700007DD50100D180000030B50B4670
:10815000014600202022012409E00D46D5409D4221
:1081600005D31D469540491B2546954040191546A7
:10817000521E002DF1DC30BD70B5002425460028CC
:1081800001DA01244042002901DA01254942FFF7C2
:10819000DDFFAC4200D04042002C00D0494270BD0F
:1081A000F0B51FB40646002082B005464024019178
:1081B00000901BE0019922460F46304600F000F97E
:1081C000049A059B801A994110D3104619462246FD
:1081D00000F0E6F8361A8F4101972246012000216F
:1081E000009F00F0DDF838184D4100902046641ED5
:1081F0000028DFDC019B00982946324607B0F0BD1D
:10820000F0B51FB486B0002000900190029006984F
:10821000069980B204900798090C020400141143D7
:1082200007900027089D099806913E463C4603901A
:108230000398A9B20204000C039004982D0C154376
:1082400048430021224600F0ABF8C71971411034B1
:108250000E46402CECDB3846029A00F0A1F8009A5A
:10826000019B8018009059410298019110300290B2
:108270004028CCDB00980BB0F0BD03460B439B07B6
:1082800003D009E008C9121F08C0042AFAD203E08B
:108290000B780370401C491C521EF9D27047D2B2B1
:1082A00001E00270401C491EFBD270470022F6E735
:1082B00010B513460A4604461946FFF7F0FF20465C
:1082C00010BD30B504460020034600E05B1C93421D
:1082D00003D2E05CCD5C401BF8D030BD0321001D13
:1082E000401E037812021A43491EF9D51046704702
:1082F000034603220870000A491C521EFAD518468C
:10830000704770B502464A40D50F40004A00ED075D
:1083100040085208002814D0002A12D0C40DD30DF2
:1083200041020120C0055202490A520AE41A091802
:1083300012187D34914201D3641C00E04900002CE6
:1083400001DA002070BD0023914201D3891A034352
:10835000400849000028F7D100290AD0914202D1F3
:108360000121C90705E0914201D2012101E001216B
:10837000C943E005C018401900F033F870BD10B5CE
:1083800000229623114600F034F810BD0122D207D6
:10839000002800DB101A002900DB511A88427047C0
:1083A00010B5202A04DB0146203A9140002010BD80
:1083B000914020239C1A0346E3401943904010BD8E
:1083C00010B5202A04DB0846203AD040002110BD19
:1083D0000B46D340D0402024A21A914008431946AE
:1083E00010BD002904DA401C490001D140084000BA
:1083F000704770B40024050C05D11024000402D18C
:10840000002921D01124050E01D100020834050FE6
:1084100001D10001241D850F01D18000A41C00287A
:1084200001DB4000641C002908D020252E1B0D46CE
:10843000F540A14000D001212943084301061B1B40
:10844000000ADB1D02D5002070BC7047DB05181840
:1084500080180029F8DA401C4900F5D170BC4008AA
:1084600040007047064C0125064E05E0E36807CC46
:108470002B430C3C98471034B442F7D3FFF72CFE43
:10848000EC2402001C25020070B58C180578401CF5
:108490006B075B0F01D10378401C2A1106D10278CB
:1084A000401C03E006780E70401C491C5B1EF9D18D
:1084B0002B0705D40023521E0DD40B70491CFAE77C
:1084C0000378401CCB1A921C03E01D780D70491CE8
:1084D0005B1C521EF9D5A142D8D3002070BD70B5E7
:1084E00007F01CFB0524204618F0A4FD00252846B3
:1084F00007F002FB204618F09DFD0126304607F0EC
:10850000CBFA204618F096FD284607F0C5FA20461B
:1085100018F090FD304607F0EFFA204618F08AFD7B
:1085200070BDB0B507F0FAFA0524204618F082FDB8
:108530000125284607F0E0FA204618F07BFD284682
:1085400007F0AAFA204618F075FD002007F0A4FAFB
:10855000204618F06FFDB0BDF0B581B007F0C2FA4B
:10856000052018F067FD08270026012007F094FA7F
:108570000524204618F05EFD204618F05BFD07F04C
:10858000A7FA0546204618F055FD002007F084FAAA
:10859000204618F04FFD76002E437F1E3806E4D1AA
:1085A000F0B201B0F0BD70B50446002007F074FAD7
:1085B00007F0B4FA052018F03DFD0826E0B2C00926
:1085C00007F09AFA0125284618F034FD284607F0EE
:1085D00063FA052018F02EFD002007F05DFA28460A
:1085E00018F028FD6400761E3006E7D1052018F04B
:1085F00021FD012070BDF0B583B0019314460E46F5
:108600000746012038430290032504E000F08EF86D
:108610006D1E280631D000F067F83846FFF7C3FF1B
:1086200000F0A6F80028F1D13046FFF7BCFF00F0BB
:108630009FF80028EAD100F057F80298FFF7B3FF3F
:1086400000F096F80028E1D1019802280BD3451ECE
:108650000026FFF781FF2070FFF741FF641C761CA6
:10866000F0B28542F5DCFFF777FF2070FFF759FF86
:1086700000F05CF8202003B0F0BD102003B0F0BD86
:10868000F0B583B01C46009201910290032504E0EE
:1086900000F04CF86D1E280623D000F025F8029853
:1086A000FFF781FF00F064F80028F1D10198FFF78F
:1086B0007AFF00F05DF80028EAD1002C0CD00026EB
:1086C000009F3878FFF76FFF00F052F80028DFD1E5
:1086D000761C7F1CA642F4D300F028F8082003B0D3
:1086E000F0BD102003B0F0BDB0B507F017FA0524B7
:1086F000204618F09FFC0125284607F0CDF92046BA
:1087000018F098FC284607F0F7F9204618F092FC7C
:108710000025284607F0F0F9204618F08BFC284683
:1087200007F0BAF9642018F085FCB0BDB0B507F0C9
:10873000F5F90524204618F07DFC0025284607F0B1
:10874000ABF9204618F076FC284607F0D5F920460C
:1087500018F070FC0125284607F09EF9204618F015
:1087600069FC284607F0C8F9642018F063FCB0BD26
:10877000B0B507F0B7F90524204618F05BFC0120DE
:1087800007F08AF9204618F055FC0B4D07F0A0F9C8
:10879000044607F07DF9002C02D06D1E2804F5D1A7
:1087A0000525284618F046FC002007F075F92846F4
:1087B00018F040FC2046B0BD33210000034801788A
:1087C0000B2901D8491C01707047C0468F2B00202F
:1087D00070B584B00025039502950195009507F0CA
:1087E00057F90F20C6430E4C1036F1B2A0206A464E
:1087F0001023FFF745FF204618F01CFC204618F018
:1088000019FC912EF0D3A020B0216A461023FFF767
:1088100037FF204618F00EFC0248058004B070BDFA
:10882000581B0000822B002070B5022902D2EB24D5
:10883000E0B270BD891EEB250022134605E0401C06
:108840005B1CDDB2A94225460EDB04786C40154660
:1088500004E034466E1C072D3546F0D26608E40766
:10886000F7D09A246640F4E7E0B270BDF0B58BB063
:108870000691044640780AA90870A27812021018DE
:10888000E27823791B029A1812041018020ECA709B
:10889000030C8B70050A4D70049001952818029303
:1088A000C018039280182178C94340186179A279D1
:1088B00012025118E279237A1B029A1812045218F4
:1088C0008018110A4018110C40180592110E40181A
:1088D000A17AE27A12025118227B0994637B1B026F
:1088E0009A18120452188018110A4018110C4018D6
:1088F00008900092100E079000263346304606E09E
:1089000039409940C9B208435B1C082B0ED001279F
:108910003A469A403446314602E0641C042CEFD0BB
:108920000AAD2D5D2A42F8D0491CF6E70899079A4E
:108930008918C9B2099CA27B914212D1617A8842FE
:108940000FD110212046FFF76FFF069A0399D170CF
:10895000029991700199517004991170059B009CC6
:1089600019E010212046FFF75FFFE17B88420BD121
:10897000069A049911700399D17002999170019926
:108980005170059B009C06E00023069AD3709370FB
:10899000537013701C4614721371210ED172210C86
:1089A0009172210A5172190ED171190C9171190A23
:1089B00051710BB0F0BDF0B58DB05522027000279B
:1089C00047720B784370CA79059202728A790492D1
:1089D000C2714A79039282710A7902924271CA7A0B
:1089E000089242738A7A019202734E7AC6720C7AA6
:1089F00084720CAA13704D782D02EB188D78C9780B
:108A0000090249190904CB18190E01711D0CC57012
:108A100009931B0A0B90837038460A91D170079511
:108A200095700693537031020919089A1202019B3E
:108A3000D21812045118089103990902029A891850
:108A4000059A1202049BD2181204511805913D4652
:108A50003A4605E02640AE4032436D1C082D0ED04C
:108A600001242146A9400346064602E05B1C042B74
:108A7000F0D00CAFFF5C3942F8D0761CF6E70B9BC8
:108A80005A72099806994018079940180A9940188F
:108A9000059A8018110A4018110C4018110E401840
:108AA000089A8018110A4018110C4018110E40182D
:108AB0005638987310211846FFF7B6FE0DB0F0BD7A
:108AC000F0B58FB00446FF20E070A07060700F20FA
:108AD000C04302900F302070704818F0ABFA704914
:108AE0000868632801D8642008606E4F0020388031
:108AF0006D4E0190308008E00B99814222D3388876
:108B00001030388080B2A1286DD206F0C1FF3978CC
:108B1000A02003AA1023FFF76EFD30802028EED19D
:108B200003AD0BA92846FFF7A1FEE97B8842E6D1F9
:108B300028785528E3D15D48017800290298DBD1D7
:108B40000846D9E73888A0284DD8C0B20021019145
:108B500005E006F09DFF3988C8B2A12943D2C1B211
:108B6000A02003AA1023FFF746FD3080398810317A
:108B70003980202837D103AD07A92846FFF776FEB4
:108B8000E97B8842E5D128785528E2D1474800782A
:108B90000028029900D1014607988842D9D240495D
:108BA0000A68962151430B9A824208D908189042CC
:108BB00019D30BA90E222046FFF75FFBC9E78918DE
:108BC000814210D307A90E222046FFF756FB0BA8BF
:108BD0000A99818107980B9008980C9009980D903C
:108BE00038880190B5E72078617809020818A178E3
:108BF000E2781202511809040818401C24D1002000
:108C000001903880A020B02103AA1023FFF7F3FCC5
:108C10003080202818D103AD0BA92846FFF726FE87
:108C2000E97B884210D1287855280DD11F4800785B
:108C3000002800D102900B980299884204D20BA917
:108C40000E222046FFF719FB2078617809020818E8
:108C5000A178E2781202511809040818401C0CD1BE
:108C60000020E072A07260722072E071A0716071E9
:108C70002071E070A07060702070019838802078BA
:108C8000617809020818A178E278120251180904E3
:108C900008180749086030880FB0F0BD7011010056
:108CA0007C2B0020822B0020782B00207B2B0020A7
:108CB000882B0020F0B581B00091064621480025A0
:108CC0000570002A2ED01446C036631B71190F2080
:108CD00008401022101A834200D303461A48027833
:108CE000102A01D0042A1AD1C809FE2707405F2F95
:108CF00013D80127B8436038C0B29E3282420CD3E9
:108D0000009A5219C9B2DFB23B46FFF774FC0F4913
:108D10000880ED19A542D8D304E0082000E0042023
:108D20000A490880094801880020042902D008293E
:108D300000D0012003490870411E8841400001B065
:108D4000F0BDC0468E2B00207A2B00208C2B0020FB
:108D50000A4A012313700A4A10700A4A11600A4A2B
:108D600000211160042801D105218901102801D1B9
:108D70001D208101054801807047C0467B2B0020E3
:108D80007A2B00207C2B0020882B0020802B0020B9
:108D9000F0B587B0994D00262E80994B1B688B4209
:108DA00024D1994C2188202925D102900092019646
:108DB000964C00272760964D964E2878062809D8AD
:108DC00006F066FE2068401C2060B042F5D38D4856
:108DD000042101802F70904C20880107029B31D024
:108DE000884820210180854D019E0BE00120400232
:108DF0008449088006E003A8FFF762FE20808148CE
:108E0000802101807F4800883F2807DD874988420C
:108E10000BDC402812D0802810D010E004280DD0A0
:108E200008280AD0202809D009E001214A029042EE
:108E300004D0C902884201D001E002262E80288891
:108E400007B0F0BDA128019E00D32780009A012A17
:108E50006A4D1ED1187B012856D1DF719F715F7159
:108E60001F711F73587B012804D1DF729F725F72DC
:108E70001F725F7303AF38461946FFF79CFDF87306
:108E80002088002846D01038C1B2A02003AA1023A1
:108E900044E0002AB6D1614801780029B2D00270BE
:108EA00018785978090208189978DA781202511856
:108EB000090408185A490978002901D00F21C9432B
:108EC000884233D2274603AC20461946FFF773FD8C
:108ED000E0733978A02010232246FFF7D1FB029AD5
:108EE0004849088008288DD138881030388010789B
:108EF0005178090208189178D278120251180904A1
:108F00000818484908607DE7597B012911D10128DB
:108F1000A3D0A7E7A02003AA10230146FFF7B0FBC8
:108F2000384908803D48009901706BE70120C00274
:108F30005EE73D480078012812D103AC204619466F
:108F4000FFF739FDE073A020B02110232246FFF780
:108F500097FB2C4908800828E4D133480770E1E7E3
:108F600018785978090208189978DA781202511895
:108F7000090408182B490968214A126851188842C7
:108F800003D2204840210180CCE7254909780029F7
:108F900001D00F21C94388422DD203AF384619466C
:108FA0001C46FFF708FDF8731B480178A02010232A
:108FB0003A46FFF765FB134908800828B2D11649E5
:108FC0000888103008802078617809020818A17894
:108FD000E278120251180904081812490860084979
:108FE0000A6815215143FFF7B1F800299AD10120F1
:108FF0000D49087096E70120C00291E7942B0020EC
:109000007C2B0020922B0020782B0020982B002016
:109010008F2B0020818D5B00822B0020842B002071
:109020007B2B0020882B0020902B0020FF010000CC
:10903000F0B585B00646434C0027278004921018EF
:10904000414A1288904241D201910397404F00203B
:10905000029038603F4C404D2078052809D806F032
:1090600017FD3868401C3860A842F5D33748042102
:109070000180029820703948018839480278102A06
:1090800001D0042A32D188190346C033049C651AE2
:109090000F2404401020001B854200DB0546DC093C
:1090A000603C01263002E7B27F09052F12D3B4439A
:1090B000E6B29E32B242234C039F0DD30198421870
:1090C000D9B2EBB23046FFF7DBFA05E01F482021AA
:1090D000018011E01B4C039F1C49088008280BD11C
:1090E000E8B21E4A11880818108005E001208002AD
:1090F00016490880134C039F144800881F2809DD77
:10910000202813D001210A0290420FD08902884200
:109110000CD00CE0042809D0082808D10F4800889A
:109120000499884201D3022700E001272780208884
:1091300002210143022902D1084900220A8005B018
:10914000F0BDC046942B0020802B0020922B0020E5
:10915000982B00208F2B0020818D5B009C2B002002
:109160007A2B0020F0B585B0044600200190042C35
:109170006FD20CF023FB002801D10CF09FFB0020E4
:10918000009000BF0098401C00900CF017FB03906B
:109190000398002803D0484900988842F2D30398E6
:1091A000002856D1042145480CF0EAFA44484549C4
:1091B00008802101444A515C4900404A505A4149C3
:1091C0000A880121090300F059F902900120049056
:1091D00020013D4940184078002801D100264BE08D
:1091E0002001394940184078012802D135480688C5
:1091F00042E0200134494018407802282AD1200159
:10920000401805792901304A515C49002B4A505ACF
:109210002C490A880121090300F030F9064628018B
:109220002A49431828012849401802892801401872
:109230000021C7683046B84706462801224BC018AF
:10924000C2882801C0188178304600F08BF80646A5
:1092500012E02DE020011C4940184078032804D07A
:10926000200140184078132804D1200116494018E5
:10927000868801E0002004900498002818D020017E
:109280001249431820011049401802892001401852
:109290003146C7680298B847019020010A4BC018B0
:1092A000C2882001C0188178019800F05BF8019015
:1092B000019805B0F0BD000050C300001C01002063
:1092C0008813000014010020881B0200C81B020044
:1092D000F8B507460C46154600200090002C00D13A
:1092E000F8BD01211C4801751C48007888431B49C2
:1092F00008700846807808210843184988700020C3
:10930000887108460078012108431449087008460E
:109310000772002617E011480078802108430F49A2
:10932000087000BF0E48007D0028FBD000200C49CB
:1093300008750A48C0892880AD1C0848C189009872
:1093400008180090761CA642E5D321460098FEF747
:10935000FDFE80B2C4E700004061004000500440C0
:109360004060004010B50346012908D1094CA41AF9
:109370009C4202D99C18A0B20BE0064809E00229E1
:1093800006D1934202DD9C1AA0B202E0002000E068
:10939000184610BDFFFF000010B504460121202033
:1093A00002F0EEF8002032490870012131480175C1
:1093B000002031490875152017F0BEFC2C48807834
:1093C000E17808432A498870084680782178084364
:1093D000274988702078802806D108460079E179ED
:1093E000490008432249087121488078E17A0843FE
:1093F0001F498870A078002803D1084600790871B9
:109400000FE0A078012806D11948007960210843AF
:109410001749087105E0164800798021084314496E
:1094200008711348807921790843114988710846E9
:109430008079617908430E498871207AC872607A10
:109440008872084600783821884309490870084620
:1094500000786178C900084305490870A07A08734C
:1094600008460078012108430149087010BD00003A
:10947000005004404061004040600040F8B50446A0
:109480000E461746002E01D100250FE0A64201DC52
:109490003D460BE00094009C204678430090314606
:1094A0000098FEF753FE0090009885B22846F8BD5C
:1094B0000146042904D28A00024BD218508800E0E9
:1094C00000207047142300200146042903D28A009B
:1094D000024B985C00E0002070470000142300203D
:1094E000FFB587B004460898844203DA0A9880687A
:1094F000002802D12448019042E00898001B82B263
:109500000292002625460A98806800212F463A4696
:109510003346049605910690FEF772FE05460E4608
:10952000002328463146029AFEF73AFE05460E46CB
:10953000304600210A4649405040014302D01248BB
:1095400001901DE003950A98C068039DA84202D3CC
:109550000020019014E00A98C1680398401A039013
:1095600009990398FEF7F2FD03900398000C00049C
:10957000002802D00448019002E0039880B20190D4
:1095800001980BB0F0BD0000FFFF000010B50848C7
:10959000007880218843064908700121054801753B
:1095A000002005490875152017F0C6FB10BD000006
:1095B000005004404061004040600040F8B505465E
:1095C0000E4614461F4621462846FEF7D5FD80B2BA
:1095D000F8BD0000FFB587B006460A98406800282D
:1095E00001D1029035E00A9801684068081803909C
:1095F00000253446002127460398069504910590DE
:1096000038462946049B059AFEF7FAFD04460D46A6
:109610000A98406802460023019020462946FEF73A
:10962000BFFD04460D46002320462946099AFEF751
:10963000B7FD04460D4628460749214000235940FE
:109640005840014303D00448C043029001E0A0B257
:10965000029002980BB0F0BD0000FFFF10B5FE486D
:1096600000688079030017F04DFB07059ED8F5F4DC
:10967000F3F2F100F84800684079030017F042FB6C
:109680000805138A2A8A468A638A13F08DFB002014
:10969000F1490968C873F04800684079401CEE49F8
:1096A000096848717DE0ED494969EB4A1268D27A50
:1096B000885C13F0F1FBE84800684079401CE649FB
:1096C00009684871E44800684079401CE24909682B
:1096D000487166E00AF0A2F9002810D113F0DCFB13
:1096E000DD4800684079401CDB4909684871DA4868
:1096F00000684079401CD8490968487105E013F0BA
:109700007DFB0020D449096848714AE00AF086F9D7
:10971000002811D1112013F0BFFBCF480068407919
:10972000401CCD4909684871CB4800684079401C0D
:10973000C9490968487105E013F060FB0020C6497B
:10974000096848712DE00AF069F900281BD1C24868
:109750000068C07A401CC0490968C872BE480068E9
:10976000C07ABE49097888420DDB0020BA490968F1
:10977000C872B94909684862B74800688079401CD6
:10978000B5490968887113F039FB0020B2490968AE
:10979000487106E013F032FB0020AF4909684871B8
:1097A00000BF00BF32E3AC480068407C002817D0FF
:1097B000AA48C068002803D0A848C1681920884773
:1097C0000020A54909684862A34800688079401CC8
:1097D000A1490968887100209F49096848711BE008
:1097E0009D480068406A282807D29B480068406A64
:1097F000401C9949096848620EE0002096490968B2
:109800004862954800688079401C934909688871CE
:109810000020914909684871F8E28F480068407952
:10982000030017F06FFA080518A42FA44CA480A415
:1098300013F0BAFA002088490968C873864800689E
:109840004079401C84490968487197E0D4E2C7E236
:1098500030E25DE194E0814949697F4A1268D27A39
:10986000885C13F019FB7C4800684079401C7A49F9
:1098700009684871784800684079401C7649096851
:1098800048717BE00AF0CAF8002811D1012013F0DA
:1098900003FB714800684079401C6F4909684871B2
:1098A0006D4800684079401C6B490968487105E0C3
:1098B00013F0A4FA00206849096848715EE00AF0D4
:1098C000ADF8002828D164490968C97A2422514397
:1098D000634A12688918604A1268D27B885C13F068
:1098E000DBFA5D480068C07B401C5B490968C873AF
:1098F00059480068C07B242814D357480068407931
:10990000401C554909684871534800684079401C1B
:1099100051490968487105E013F070FA00204E497A
:10992000096848712AE00AF079F8002818D14A48F5
:109930000068C07A401C48490968C87246480068F7
:10994000C07A4649097888420ADB00204249096802
:10995000C872414800688079401C3F490968887195
:1099600013F04CFA00203C490968487106E013F0F6
:1099700045FA002038490968487100BF00BF45E238
:10998000354800684079030017F0BCF90A0614B99D
:109990002BB948B978B995B913F006FA00202E49C9
:1099A0000968C8732C4800684079401C2A49096836
:1099B0004871ABE029494969274A1268D27A885C24
:1099C00013F06AFA244800684079401C224909686B
:1099D0004871214800684079401C1F490968487156
:1099E00094E00AF01BF8002811D14A2013F054FA31
:1099F000194800684079401C1749096848711648A1
:109A000000684079401C14490968487105E013F06A
:109A1000F5F9002010490968487177E009F0FEFF68
:109A2000002824D1FF2013F037FA0B480068C07BD0
:109A3000401C09490968C87307480068C07B24288E
:109A40001BD3054800684079401C034909684871E8
:109A500001480068407905E004080020602B0020E0
:109A600000080020401CEA490968487105E013F02D
:109A7000C5F90020E6490968487147E009F0CEFFC2
:109A8000002811D1FF2013F007FAE148006840795F
:109A9000401CDF4909684871DD4800684079401C76
:109AA000DB490968487105E013F0A8F90020D8499E
:109AB000096848712AE009F0B1FF002818D1D4489C
:109AC0000068C07A401CD2490968C872D048006852
:109AD000C07AD049097888420ADB0020CC4909685D
:109AE000C872CB4800688079401CC94909688871F0
:109AF00013F084F90020C6490968487106E013F0A4
:109B00007DF90020C2490968487100BF00BF7DE1AE
:109B1000BF4800684079030017F0F4F80C0715C33C
:109B20002CC349C366C382C39FC313F03DF9002011
:109B3000B7490968C873B64800684079401CB44901
:109B400009684871B4E0B3494969B14A1268D27AE8
:109B5000885C13F0A1F9AE4800684079401CAC491C
:109B600009684871AA4800684079401CA8490968FA
:109B700048719DE009F052FF002811D1772013F0C1
:109B80008BF9A34800684079401CA14909684871D5
:109B90009F4800684079401C9D490968487105E06C
:109BA00013F02CF900209A490968487180E009F007
:109BB00035FF002811D10C2013F06EF9944800688D
:109BC0004079401C92490968487191480068407981
:109BD000401C8F490968487105E013F00FF9002017
:109BE0008B490968487163E009F018FF002810D11B
:109BF00013F052F9864800684079401C844909688E
:109C00004871834800684079401C8149096848715F
:109C100005E013F0F3F800207D490968487147E03A
:109C200009F0FCFE002811D1132013F035F9784813
:109C300000684079401C764909684871744800689A
:109C40004079401C72490968487105E013F0D6F864
:109C500000206F49096848712AE009F0DFFE0028FA
:109C600018D16B480068C07A401C69490968C872FD
:109C700067480068C07A6749097888420ADB002093
:109C800063490968C872624800688079401C60496D
:109C90000968887113F0B2F800205D4909684871BD
:109CA00006E013F0ABF8002059490968487100BF7D
:109CB00000BFABE0564800684079030017F022F877
:109CC000080513872A874787638713F06DF80020FC
:109CD0004F490968C8734E4800684079401C4C4998
:109CE000096848717AE04B494969494A1268D27A51
:109CF000885C13F0D1F8464800684079401C44491C
:109D000009684871424800684079401C4049096828
:109D1000487163E009F082FE002811D1492013F058
:109D2000BBF83B4800684079401C394909684871D4
:109D3000374800684079401C35490968487105E09A
:109D400013F05CF8002032490968487146E009F0D8
:109D500065FE002810D113F09FF82D480068407967
:109D6000401C2B4909684871294800684079401C0B
:109D700027490968487105E013F040F8002024499C
:109D8000096848712AE009F049FE002818D12048E6
:109D90000068C07A401C1E490968C8721C480068E7
:109DA000C07A1C49097888420ADB002018490968F2
:109DB000C872174800688079401C15490968887185
:109DC00013F01CF8002012490968487106E013F0EE
:109DD00015F800200E490968487100BF00BF15E062
:109DE00000200B49096888710949096848710620F3
:109DF00007490968C87009E013F000F80020044919
:109E00000968487102490968887100BF00BF10BD28
:109E100004080020602B002010B56A4800684079D3
:109E2000030016F06FFF090610C627C644C6608EF1
:109E3000C60012F0B9FF634800684079401C6149D0
:109E400009684871BCE0604949695E4A1268D27A83
:109E5000885C13F021F85B4800684079401C594940
:109E600009684871574800684079401C554909689D
:109E70004871A5E009F0D2FD002811D17F2013F030
:109E80000BF8504800684079401C4E4909684871F9
:109E90004C4800684079401C4A490968487105E00F
:109EA00012F0ACFF002047490968487188E009F0CA
:109EB000B5FD002810D112F0EFFF4248006840794C
:109EC000401C4049096848713E4800684079401C80
:109ED0003C490968487105E012F090FF00203949BB
:109EE000096848716CE009F099FD002822D13548D5
:109EF0000068C07A401C33490968C872314800685C
:109F0000C07A3149097888420FDB00202D49096861
:109F1000C8722C4800684079401C2A490968487179
:109F2000002028490968486208E00020254909689E
:109F3000487103E0002023490968487112F05EFF70
:109F40003EE020480068407C002816D01E48C068CB
:109F5000002803D01C48C1681920884700201949EF
:109F60000968486217490968487116490968887183
:109F7000052014490968C8701AE012480068406A50
:109F8000282807D20F480068406A401C0D4909681C
:109F900048620DE000200B490968486209490968D8
:109FA0004871084909688871052006490968C87020
:109FB00006E012F023FF002002490968487100BF43
:109FC00000BF10BD04080020602B002010B5002445
:109FD000F7480068807A01287ED1F5480068C0798A
:109FE00000287AD0F24800688079002804D001283F
:109FF00074D0022873D191E1ED480068007B2428D9
:10A000006ED2EB480068C07901287AD1002475E04F
:10A01000E7480068C07A24214843E64909684018A7
:10A02000E3490968097B415CE1480068C07A242261
:10A030005043E14A12688018DD4A1268127B805C46
:10A04000814229D0DA480068C07A24214843DA499D
:10A0500009684018D6490968097B415CD448006802
:10A06000C07A24225043D34A12688018D04A12681A
:10A07000127B8154CE480068407B242805D3CC480D
:10A080000068007BCA4909684873C9480068007BBA
:10A09000C7490968887308E0C5480068407B2428E0
:10A0A00003D20120C24909688871C1480068007B59
:10A0B000401CBF4909680873BD480068007B24281C
:10A0C00008D3BB480068407B242803D20120B8494C
:10A0D00009688871B64805E0D3E1CDE169E0BAE1ED
:10A0E00038E00EE00068007B242804D2B048006805
:10A0F0008079012800D103E0601CC4B2242C87D3EE
:10A1000056E0002413E0AA480068C07A242148439E
:10A11000A94909684018015DA5480068C07A242251
:10A120005043A44A126880180155601CC4B2242C04
:10A13000E9D300209E490968487323209C49096897
:10A14000887301209A490968887124209849096810
:10A1500008732DE000209649096808739448006848
:10A16000C07A401C92490968C87291480068C07A58
:10A1700092490978884217DB8D480068007C0128E5
:10A1800004D102208A490968887106E000208849C4
:10A190000968887186490968C8710020844909687E
:10A1A000C8728349096808740020814909684871A8
:10A1B00061E17F4800684079030016F0A3FD0805BF
:10A1C00013A62AA651A68EA601207949096808740B
:10A1D00012F0EAFD764800684079401C744909682D
:10A1E000487199E075494969714A1268D27A885C68
:10A1F00012F052FE6E4800684079401C6C490968B4
:10A2000048716B4800684079401C69490968487189
:10A2100082E009F003FC00281BD165490968497BED
:10A22000491CC8B212F038FE61480068407B6049A2
:10A230000968C8735E4800684079401C5C49096839
:10A2400048715B4800684079401C59490968487169
:10A2500005E012F0D3FD00205549096848715BE024
:10A2600009F0DCFB00282BD151490968C97A242266
:10A270005143504A126889184D4A1268D27B885C53
:10A2800012F00AFE4A480068C07B401C4849096831
:10A29000C87347480068C07B45490968897B884284
:10A2A0001ADD434800684079401C414909684871FB
:10A2B0003F4800684079401C3D49096848710BE0FF
:10A2C00012F09CFD3A480068407B39490968C87320
:10A2D00000203749096848711EE009F09FFB0028FB
:10A2E0000CD1334909688871242031490968C87341
:10A2F0002F49096848732E490968887312F07EFD5A
:10A3000000202B490968487106E012F077FD002013
:10A3100027490968487100BF00BFACE024480068C5
:10A320004079030016F0EEFC08050F8E268E4C8E49
:10A33000688E12F039FD1E4800684079401C1C49A7
:10A340000968487185E01D494969194A1268D27A3D
:10A35000885C12F0A1FD164800684079401C144941
:10A3600009684871124800684079401C1049096822
:10A3700048716EE009F052FB002811D1492012F01B
:10A380008BFD0B4800684079401C094909684871F9
:10A39000074800684079401C05490968487105E094
:10A3A00012F02CFD002002490968487151E00000BC
:10A3B0000408002000080020FC070020602B00207B
:10A3C00009F02CFB002810D112F066FD9C480068B3
:10A3D0004079401C9A490968487199480068407959
:10A3E000401C97490968487105E012F007FD0020FC
:10A3F0009349096848712CE009F010FB00281AD134
:10A400008F480068C07A401C8D490968C8728C4822
:10A410000068C07A8B49097888420CDB00208849A3
:10A420000968C87286490968887185490968487150
:10A4300083490968C87112F0E1FC0020804909686D
:10A44000487106E012F0DAFC00207D490968487185
:10A4500000BF00BF0FE012F0D1FC0020784909686E
:10A4600048717749096888717549096808737449A2
:10A470000968C87200BFE2E000207149096888726B
:10A48000DDE06F480068807A0228F4D16C480068EB
:10A49000007A002879D06A4800684079030016F0F5
:10A4A00031FC0B0711BB25BB41545EBB7590BB0053
:10A4B00012F07AFC624800684079401C60490968E3
:10A4C0004871B7E05F494969087812F0E5FC5C48DB
:10A4D00000684079401C5A4909684871584800682A
:10A4E0004079401C564909684871A3E009F096FA82
:10A4F000002810D112F0D0FC514800684079401C6F
:10A500004F49096848714E4800684079401C4C49E1
:10A510000968487105E012F071FC0020484909689B
:10A52000487187E009F07AFA002807D144480068AA
:10A530004079401C42490968487103E000204049C5
:10A540000968487112F05AFC74E012F02DFC3C4886
:10A5500000684079401C3A49096848716AE0394905
:10A5600049690978491CC8B212F096FC3448006861
:10A570004079401C32490968487131480068407987
:10A58000401C2F490968487154E054E009F046FA2C
:10A5900000280FD112F0DAFB2949096888700120E0
:10A5A00012F04EFC264800684079401C2449096896
:10A5B000487105E012F022FC002021490968487129
:10A5C00038E01F480068807811280CD100201C4911
:10A5D00009680872AA201A49096888700020184979
:10A5E0000968487011E0164800684078401C14491A
:10A5F00009684870124800684078032805D309F0BC
:10A60000B1FA00200E490968487012F0F7FB0020EB
:10A610000B49096848710DE012F0F0FB0020084971
:10A6200009684871064909684870AA200449096800
:10A63000887000BF03E0002001490968887210BDDE
:10A6400004080020602B002010B502469000074B44
:10A65000C018405C002802D00320C04310BD012078
:10A660009300024C1B1958540020F7E7DC26002009
:10A6700070B5002508E06D1C1848854202D20BF029
:10A6800049F901E0002503E00BF098F80028F2D129
:10A6900000BF002406E01248015D00200BF09CF88A
:10A6A000601CC4B2042CF6D3002408E00020A100F2
:10A6B0000C4A5054A10089184880601CC4B2042C74
:10A6C000F4D30120084908700020487005208870E4
:10A6D0000020C87005480649088070BD50C30000BE
:10A6E000841B02001423002018010020881300009E
:10A6F00014010020F8B58D480078030016F002FB25
:10A70000060405163D5EFDFC0EE10BF0D7F80020B7
:10A710008649C870487008468078002802D1032016
:10A72000087002E0022081490870FDE07F488078CF
:10A73000002804D07D488078401E7C4988700BF04A
:10A740003DF800280BD10BF0B9F800207749C8700C
:10A750000846807800280FD1032008700CE0734869
:10A76000C078401C7149C8700846C078052803D3DA
:10A77000052008700BF0CEF8D6E00BF01FF800288B
:10A780000ED104216A480AF0FBFF00206749C87017
:10A7900048706848684908800420644908700CE0E3
:10A7A0006248C078401C6149C8700846C0780528D6
:10A7B00003D3052008700BF0ADF8B5E05B4949788C
:10A7C00009015E4A515C4900594A505A5A490A885F
:10A7D00001210903FEF752FE0090012553484078FD
:10A7E0000001564940184078002801D100243CE07F
:10A7F0004E4840780001514940184078012802D164
:10A800004D48048831E04948407800014B494018E0
:10A810004078022812D1454949780901474A8918E8
:10A820000879FEF745FE0446404949780901434A44
:10A8300089180879FEF748FE054616E03B4840783F
:10A8400000013E4940184078032806D03748407838
:10A85000000140184078132806D1344840780001A0
:10A8600036494018848800E00025002D2FD02F485D
:10A8700040780001324943182C48407800012F49A4
:10A880004018028929484078000140182146C768CD
:10A890000098B8470646254840780001274BC01865
:10A8A000C288224840780001C01881783046FEF7FF
:10A8B00059FD06461D4840788000224940184680D0
:10A8C00001201A49497889001E4A50540AE00020A4
:10A8D0001649497889001B4A8918488013494978E4
:10A8E0008900505411484078401C1049487008466F
:10A8F0004078042809D301E013E007E00AF0DEFF06
:10A9000000200A494870032008700DE00AF056FF45
:10A91000002803D101200549087001E00AF0FAFF80
:10A9200002E0FFF7A5FE00BF00BFF8BD1801002040
:10A930001C0100208813000014010020881B020065
:10A94000C81B02001423002010B50AF001FF0024E8
:10A9500005E00020A100074A5054601CC4B2042C3A
:10A96000F7D3002004490870052088700348044983
:10A97000088010BD14230020180100208813000057
:10A980001401002010B50346002000F0D7F8002085
:10A9900000F03AF9002000F0AFF8002000F012F9C2
:10A9A000002000F087F8002000F0EAF800BF012046
:10A9B00000F0A2F8012000F005F9002421E00020B9
:10A9C00000F09AF8002000F0FDF8802018400028E0
:10A9D00006D0012000F0B2F8012000F015F905E0E2
:10A9E000002000F0ABF8002000F00EF900BF0120BD
:10A9F00000F082F8012000F0E5F85806030E601C14
:10AA0000C4B2082CDBDB012000F054F8012000F078
:10AA1000B7F810BD30B503460C46012000F08EF8A3
:10AA2000012000F0F1F8002000F066F8002000F0AE
:10AA3000C9F8002000F03EF8002000F0A1F800BFA7
:10AA4000012000F059F8012000F0BCF8002528E0B2
:10AA5000002000F051F8002000F0B4F880201840E9
:10AA6000002803D0012000F069F802E0002000F087
:10AA700065F880202040002803D0012000F0C4F8B1
:10AA800002E0002000F0C0F800BF012000F034F820
:10AA9000012000F097F85806030E6006040E681CAB
:10AAA000C5B2082DD4DB012000F004F8012000F02D
:10AAB00067F830BD00B5014600290CD00C4800787D
:10AAC000082290430A4A107008200A4A1070052094
:10AAD00009F060FF0BE00648007808229043044A22
:10AAE00010700820034A1074052009F053FF00BDC0
:10AAF000200304408000044000B5014600290CD02A
:10AB00000C480078102290430A4A107010200A4A1C
:10AB10001070052009F03EFF0BE006480078102277
:10AB20009043044A10701020034A1074052009F065
:10AB300031FF00BD200304408000044000B5014601
:10AB400000290CD00C480078042290430A4A107067
:10AB500004200A4A1070052009F01CFF0BE006488B
:10AB6000007804229043044A10700420034A1074B1
:10AB7000052009F00FFF00BD2003044080000440C1
:10AB800000B5014600290CD00C48C0790222904340
:10AB90000A4AD07102200A4AD071052009F0FAFE53
:10ABA0000BE00648C07902229043044AD07102208B
:10ABB000034AD075052009F0EDFE00BD20030440D6
:10ABC0008000044000B5014600290CD00C48C07933
:10ABD000400840000A4AD07101200A4AD07105207D
:10ABE00009F0D8FE0BE00648C07940084000044A4E
:10ABF000D0710120034AD075052009F0CBFE00BDBD
:10AC0000200304408000044000B5014600290CD018
:10AC10000C48C079042290430A4AD07104200A4AA1
:10AC2000D071052009F0B6FE0BE00648C079042279
:10AC30009043044AD0710420034AD075052009F0DE
:10AC4000A9FE00BD200304408000044010B532215D
:10AC5000464805F063FEF920FFF794FE3221444890
:10AC600005F05CFE8820FFF78DFE9020FFF78AFE3E
:10AC70009820FFF787FE08210846FFF7CBFEE82063
:10AC8000FFF780FE12210846FFF7C4FEA020FFF761
:10AC900079FE70210846FFF7BDFEA820FFF772FE7F
:10ACA00070210846FFF7B6FEB020FFF76BFE70215B
:10ACB0000846FFF7AFFEB820FFF764FE0021084604
:10ACC000FFF7A8FEC020FFF75DFE00210846FFF752
:10ACD000A1FEC820FFF756FE00210846FFF79AFEA6
:10ACE000D020FFF74FFE2F210846FFF793FED82014
:10ACF000FFF748FE2F210846FFF78CFEE020FFF704
:10AD000041FE2F210846FFF785FE4020FFF73AFE5F
:10AD100000210846FFF77EFE0A20FFF733FE0024DD
:10AD200005E000210846FFF775FE601CC4B25A2CEE
:10AD3000F7DB00240AE000200E4908550E490855AB
:10AD40000E4908550E490855601CC4B25A2CF2DB56
:10AD50008120FFF717FE00200A4908600A490870A1
:10AD60008870C8700871487010BD0000C0D4010020
:10AD7000204E00007C200020D62000203021002022
:10AD80008A210020EC000020E400002000B5802093
:10AD9000FFF7F8FD00BD00000B48007800280CD13B
:10ADA0000A480068582805D808480068801C0749E8
:10ADB000086002E00020054908600120024908708F
:10ADC0000020487070470000E4000020EC000020E4
:10ADD00000B54E480078002879D04C4880780300B0
:10ADE00015F090FF060450576067768B474800794E
:10ADF0004749085C45490979464A515C884216D161
:10AE0000424800794449085C40490979434A515C09
:10AE100088420CD13D48007941490968884222D3D3
:10AE20003A4801793E480068801C81421BD8374867
:10AE300000793749085C35490979364A5054334816
:10AE400000793549085C31490979344A50542F4812
:10AE5000C078002803D004202C49887011E001201C
:10AE60002A4988700DE000202849C87008460079FA
:10AE7000401C0871084600795A2802DB002008713E
:10AE8000087041E04020FFF77DFD02201F498870D7
:10AE90003AE01E4A11791079FFF7BCFD03201B49E7
:10AEA000887031E00A20FFF76DFD04201749887093
:10AEB0002AE0164A1279194B995C144A1279154BFB
:10AEC000985CFFF7A7FD0520104988701CE01CE086
:10AED0000E480079401C0D490871084600795A282F
:10AEE00004DB002008710870C87002E001200749E7
:10AEF000C87000200549887006E0002003490870EA
:10AF00008870C870087100BF00BF00BDE400002059
:10AF10007C200020D6200020302100208A21002023
:10AF2000EC00002010B501F069FE01281ED101F0EF
:10AF300053FE1149884212D3072009F0A1FB0028D3
:10AF400006D04B22D2000021012014F095F812E027
:10AF50007D22D2000021012014F08EF80BE07D222A
:10AF6000D2000021012014F087F804E000221146ED
:10AF7000012014F081F810BDD60B00000020034919
:10AF8000087248708870486070470000280A0020E6
:10AF900058221152704710B504460121022000F0DA
:10AFA000EFFA0021022000F0EBFA10BD014600206C
:10AFB0005322525C10231A40002A08D05322525CBC
:10AFC0000C231A409210032A18D1032016E05422B1
:10AFD000525A0123DB031A40002A0ED05322525C3E
:10AFE0000C231A409210032A05D05322525C920778
:10AFF000920F032A01D1022000E00120704702468F
:10B00000002058239B5A0B40002B01D0012000E068
:10B010000020704710B5002A0AD056231B5A0C0294
:10B0200023435624235256231B5A8B43235209E0B1
:10B0300056231B5A0C02A3435624235256231B5A51
:10B040000B43235210BD0000F8B504460D460127FE
:10B0500000263448844203D10121022000F090FAF6
:10B060002878401EA0702088FF21013108432080ED
:10B070002088400840002080A878401EC1B25A2095
:10B08000015568790007000CE97909020843A9799C
:10B0900008435C210853288981B240200153A868E5
:10B0A000C000C10C42200153A88981B24420015341
:10B0B000E868C000C10C46200153288A81B24820AC
:10B0C00001532869C000C10C4A200153A88A81B2EB
:10B0D0004C2001536869C000C10C4E200153502020
:10B0E000005B297909020843502108535020005B76
:10B0F000297988435021085300E0761C5020005BDA
:10B100004007400F2979884202D007488642F4D18F
:10B110005020005B4007400F2979884200D000276B
:10B120003846F8BD00540440FFFF000030B5034628
:10B1300000201C898C4209DD082A05D218244C43C2
:10B140001D682C19A05C02E0002000E0002030BD4A
:10B1500010B5024613898B4205DD18234B43146852
:10B16000E318987C00E0002010BD00000146144A5E
:10B17000C889C007C00F00280AD00120C88100E09C
:10B18000521EC889C007C00F002801D0002AF7D17D
:10B19000C889C007C00F00280FD10220C881042031
:10B1A000C881487A400840004872487A382398435A
:10B1B000487200204872012070470020FCE7000020
:10B1C000FFFF00000246507A012318435072507A64
:10B1D0000B78DB0018435072087A012808D1888860
:10B1E00050814868000C0123DB031843908108E07C
:10B1F000087A002805D1508148688000204B18400B
:10B200009081487A012804D1507A40231843507223
:10B2100006E0487A002803D1507A402398435072C0
:10B22000087D002804D0507A80231843507203E030
:10B23000507A8023984350720878002811D1C87A38
:10B240001072087B1070487B5070887B9070CB7BAD
:10B25000D370087C10714B7C5371887C9071CB7CCF
:10B26000D371887A002803D00120C002D08101E088
:10B270000820D081FF200130D081012070470000DC
:10B28000FC1F0000002904D0427A80231A43427236
:10B2900003E0427A80239A434272704730B50246F7
:10B2A00000200F4B5024A45A0D022C435025AC52C1
:10B2B0005024A45A8C43AC5200E05B1E5024A45A84
:10B2C0006407640F8C4201D0002BF6D15024A45A9D
:10B2D0006407640F002C01D0002000E0012030BD85
:10B2E000FFFF0000827A80231A40802A00D08172FA
:10B2F00070470000F0B587B006460C4600270020D6
:10B3000006906020875BF807C00F002802D001215B
:10B310006020815355E0FF20000238400005000FF7
:10B3200006902B48864204D1069800012949451809
:10B3300006E02948864203D10698000127494518AE
:10B340000420E881A8890121C9030840002809D008
:10B35000012069460872A889C004C00869890843A9
:10B36000019007E0002069460872A8891C4908403E
:10B3700080100190287A6946C872002003E02A5C98
:10B3800003A90A54401C6946C97A8142F7DCA088A7
:10B39000172801DB0020A080618818225143224633
:10B3A0000832881818226946FCF767FF6188481C34
:10B3B0001721FCF7E1FE6180A088401CA08060207E
:10B3C000875B022038400028A5D007B0F0BD000000
:10B3D0000054044000550440005804400059044003
:10B3E000FC1F000005480078002803DD0020034909
:10B3F000087002E0002002490880704783000020A6
:10B400008000002000200149087070478200002061
:10B4100010B5A0210C48FCF749FF0B480B494860C8
:10B420000B480860052008810A48C860002008749D
:10B43000084B05220649054800F0A4FE55210348A3
:10B4400000F00AF810BD00004C0900209008002010
:10B450001817020075B70000027C80231A40802A6A
:10B4600000D001747047000010B502461D4BD08912
:10B47000C007C00F00280AD00120D08100E05B1E69
:10B48000D089C007C00F002801D0002BF7D1D08988
:10B49000C007C00F002801D0002010BD507A012441
:10B4A00020435072507A3824A0435072C87A1072E8
:10B4B000487A00280FD1087B1070487B5070887B39
:10B4C0009070CC7BD470087C10714C7C5471887C5B
:10B4D0009071CC7CD471FF200130D0814000D081AC
:10B4E000107ADAE7FFFF0000FFB581B004460D4691
:10B4F0000020012C03D140262E43304306E0002CCF
:10B5000000D103E0022C01D1C0263043012A06D12C
:10B51000049E760010273E430643F0B206E0002A60
:10B5200000D103E0022A01D130263043134E30709F
:10B5300076788027BE43114F7E70012C08D1FF2101
:10B5400000BF0E4EB3781E460E4033468B42F8D1F4
:10B550000A4E76784027BE43084F7E70012A0BD1F1
:10B560000026009603E000BF009E761C0096FF2791
:10B570006937009EBE42F6D905B0F0BD0004024016
:10B58000002905D0054A12780243044B1A7004E0E2
:10B59000024A12788243014B1A707047200402401D
:10B5A000002905D0054A927E0243044B9A7604E0B6
:10B5B000024A927E8243014B9A767047000802400D
:10B5C00070B5034614460020002B01D1C0B202E042
:10B5D00005468035E8B2012902D1051DE8B206E032
:10B5E000022903D105460835E8B200E0C0B2012CBB
:10B5F00002D1851CE8B200E0C0B2084DA870AD7859
:10B6000001263543054EB570002201E000BF521CF3
:10B610007D252D01AA42F9D970BD0000000C024021
:10B6200070B500242448007920210840002801D06A
:10B63000224D3FE000F046F8054621480078802181
:10B640000840002836D01E4880780840002801D0E5
:10B650001A4D02E000F036F80546194880780007D8
:10B66000840F022C01DBAD0804E0012C01D16D0830
:10B6700000E000BF124880788007C00F002801D08A
:10B680002D0101E00C2045430D4800784007840F50
:10B69000002C02D1601CC4B207E0032C03D1601C53
:10B6A0004006040E01E06006040E21462846FCF721
:10B6B0004DFD0546284670BD0004024000127A0088
:10B6C000000C024000B5C0229178F82211401C4ABB
:10B6D00012781143EA2923D00ADC0A46E03A130023
:10B6E00015F010FB0A181C20242A2A2A2A161A2AC6
:10B6F000ED291FD004DCEB2916D0EC291CD117E072
:10B70000F02903D0F82917D10E4817E00E4815E0AC
:10B710000E4813E00E4811E00E480FE00E480DE011
:10B720000E480BE00E4809E00E4807E00E4805E021
:10B730000E4803E00E4801E00D4800BF00BF00BD09
:10B74000201C02400090D003006CDC020048E8019D
:10B7500000366E010024F400001BB70000127A00CE
:10B76000808D5B0000093D00C0C62D0080841E0056
:10B7700040420F0070B586B00446002500262068C0
:10B780000190A1796846C17261794172002101720C
:10B79000017000BF05E020460830415D03A8415517
:10B7A0006D1C6846C07AA842F5D80B22D2010199D7
:10B7B000881A914237D007DC2C48081A1FD0232161
:10B7C0000901401A48D113E0FF386F38002802D031
:10B7D000012841D105E069462548FFF745FE0646A8
:10B7E0003BE0694622484030FFF73EFE064634E023
:10B7F00069461F485030FFF737FE06462DE0694680
:10B800001B482030FFF730FE06461A4800880728FC
:10B8100005DA18480088401C1649088002E000201C
:10B820001449088019E005F0EBFC002813D01248F9
:10B8300001780078401C104A1070022906DC694625
:10B840000B486030FFF710FE064604E000200A496E
:10B8500008700A49087000E000BF00BF002E02D146
:10B86000012006B070BD0020FBE7000020020000B0
:10B8700080550440800000207C000020080100204A
:10B8800010B5A8210A48FCF711FD094809490860CC
:10B89000094848600720088100208872072206496D
:10B8A000044800F0BFFA00210248FFF71BFD10BD5D
:10B8B000A408002084080020A41702000C4A127873
:10B8C00012060B4B5B781B041A43094B9B781B0237
:10B8D0001A43074BDB781A43104642084240D20015
:10B8E00083085A401146034A5140034A1160704789
:10B8F00047070020010200004C070020F8B504466D
:10B900000F46A07A4006400E002874D10025ACE016
:10B910001820684321680818407C01283CD1012187
:10B920001820684322681018017400260CE01820C3
:10B930006843216808180830815D18206843226830
:10B9400010188155701CC6B2082EF0D300211820A3
:10B950006843226810180174182068432268101880
:10B960004174182068432268101841611820684308
:10B970002268101881742C20684361680818406A96
:10B98000002809D018236B432268D0182C236B435E
:10B990006268D218516A88471820684321680818DD
:10B9A0004069FF21C94388425DD818206843216857
:10B9B00008184069C11918206843226810184161AD
:10B9C000182068432168081841692C206843626880
:10B9D00010188069814246D31820684321680818EE
:10B9E000807C55283FD055211820684322681018C4
:10B9F0008174002624E03CE0182068432168081880
:10BA0000805D2C216943626851181031895D0840BE
:10BA10001821694322685118885518206843216805
:10BA20000818805D2C216943626851180831895DCE
:10BA3000084318216943226851188855701CC6B202
:10BA4000082ED9D32C20684361680818806A002822
:10BA500009D018236B432268D0182C236B436268EB
:10BA6000D218916A8847681C85B22089A84200DDF7
:10BA70004EE7F8BD0120014908707047940000208E
:10BA800010B50446002015F019FB022859D10120F9
:10BA900038490880FFF7A6FC00203749087037486E
:10BAA0000078002802D1012034490870334800781A
:10BAB000012826D131484078401C30494870214641
:10BAC0005A20FCF743FB2D494978884250D8002082
:10BAD0002A49487008468078401C8870084680785B
:10BAE0000A2803D30020887002200870FFF77AFC30
:10BAF00000202149087000F07FF8002015F00EFBAF
:10BB000036E01E480078022832D11C484078401C9C
:10BB10001A49487021467D20C000FCF717FB1749E1
:10BB20004978884224D8002014494870FFF75AFC0D
:10BB300000201149087000F05FF8002015F0EEFABF
:10BB400016E00E48C078401C0C49C8700846C07802
:10BB5000042804DB0020C87008704870887005480D
:10BB60000088012804D100200249088000F05AF81A
:10BB700010BD00007E0000207C0000207800002026
:10BB800000B587B0002010490870FFF72BFC00219A
:10BB900068460171042141710C48029041100391E3
:10BBA0000B49049105910B480690FFF769FE01A827
:10BBB00015F0F4FA00F09CFB00F034F80021064880
:10BBC00009F0A6FF07B000BD7C000020FFFF1F00AA
:10BBD000FFFFFF1FF15C01000205000030B50346C6
:10BBE00000201C898C4204D94D015C686419626094
:10BBF00000E0022030BD000010B5002400BF09E0C5
:10BC00001C20604305494018214682680448FFF71C
:10BC1000E5FF641C052CF3D310BD000018170200CB
:10BC20009008002010B508207A49C87200200873D7
:10BC30000021784841738173C17301744174817428
:10BC4000C174002073490875FF200230486000204D
:10BC500008720120087000204872012088726E4826
:10BC6000FFF784FA6B496C48FFF7ACFA01216A4888
:10BC7000FFF708FB69486749486000200872012007
:10BC80000870002048720120887263481030FFF766
:10BC90006DFA604960481030FFF794FA01215E4860
:10BCA0001030FFF7EFFA5D48401E5A494860002007
:10BCB00008720120087000204872012088725648DE
:10BCC0005030FFF753FA534953485030FFF77AFA90
:10BCD000012151485030FFF7D5FA5048C1384D493D
:10BCE000486000200872012008700020487201207E
:10BCF000887249484030FFF739FA46494648403093
:10BD0000FFF760FA012144484030FFF7BBFAFF20FB
:10BD1000123040494860002008720120087000205D
:10BD20004872012088723C486030FFF71FFA394999
:10BD300039486030FFF746FA012137486030FFF795
:10BD4000A1FAFF2021303349486000200872012009
:10BD5000087000204872012088722F48A030FFF739
:10BD600005FA2C492C48A030FFF72CFA01212A486B
:10BD7000A030FFF787FA29488F382649486000200D
:10BD80000872012008700020487201208872224841
:10BD9000E030FFF7EBF91F491F48E030FFF712FAD8
:10BDA00001211D48E030FFF76DFA1D481949486030
:10BDB000002008720120087000204872012088725B
:10BDC00015482030FFF7D2F9124913482030FFF709
:10BDD000F9F9012110482030FFF754FA1048CB3010
:10BDE0000C49486000200872012008700020487249
:10BDF0000120887208483030FFF7B8F90549064835
:10BE00003030FFF7DFF9012103483030FFF73AFA0D
:10BE100010BD00009C2600201055044002040000C4
:10BE200014070000F0B50B4614464360048100215E
:10BE300036E0002216E02C254D4346687519AD5CAE
:10BE400018274F430668F619B5542C254D4346680C
:10BE50007519AD5C18274F430668F6190836B554B6
:10BE6000551CEAB2082AE6D3002518274F43066876
:10BE7000F619357418274F430668F6197574182794
:10BE80004F430668F619B57418274F430668F6192C
:10BE9000F57418274F430668F61975614D1CA9B251
:10BEA00005898D42C5DC00258572F0BD70B504465C
:10BEB000606800F02DFE0546E27A23460C332946E1
:10BEC000094800F0EDFD09496068884204D007493F
:10BED000CB396068884206D1E17AA28890B22246C6
:10BEE0000C3203F04FF970BD84080020DF0700001A
:10BEF000F8B505460026002704F04CFF07462C46FF
:10BF0000002C25D000BF03E00020A055701CC6B255
:10BF1000082EF9D3207808218843F900082211401F
:10BF200008432070E079E02188430A4909884901E3
:10BF3000E02211400843E071E07940094001012FFF
:10BF400001D1082100E00021C906C90E0843E071B3
:10BF5000F8BD000080000020FEB506460025002741
:10BF60000020029005F010F8019005F015F90090FE
:10BF70003446002C64D033480078012858D100BFE3
:10BF800003E000206055681CC5B2082DF9D304F009
:10BF9000E7FF00280DD005F027F9022809D1062176
:10BFA0002948FFF7D5F8552803D004F0D3FF00281F
:10BFB00003D10020207060700FE0019892307D2145
:10BFC000C900884203D80198923087B201E07D27EA
:10BFD000FF003804000E2070677005F0C9F80028D3
:10BFE0000DD005F007F9022809D106211648FFF700
:10BFF000AFF8552803D005F0B5F8002803D100208C
:10C00000A070E0701CE0009892307D21C900884249
:10C0100004D80098923080B2029002E07D20C000E7
:10C02000029002980004000EA0700298E07007E0F1
:10C03000002503E000206055681CC5B2082DF9D327
:10C04000FEBD00008200002084080020F8B50546EF
:10C05000002605F0D5F807462C46002C20D000BF5E
:10C0600003E00020A055701CC6B2082EF9D3012FA2
:10C070000AD131202070012060705920A070082062
:10C08000E070002020710BE0022F09D131202070D8
:10C09000012060705920A0700820E07001202071FC
:10C0A000F8BD0000FEB50646002500200290019074
:10C0B00001F08EFD074604F09DFE0A210090FCF77A
:10C0C0005BF880B2029004F075FF01903446002CBA
:10C0D00023D012480078012817D100BF03E00020C8
:10C0E0006055681CC5B2082DF9D33802000E607186
:10C0F0003804000EA071E7710198FF2802DDFF20CF
:10C10000A0700AE00198A07007E0002503E000207D
:10C110006055681CC5B2082DF9D3FEBD8200002011
:10C12000FEB50646002400200190002704F054FCD0
:10C1300064210090FCF720F880B20190002001F00B
:10C1400069FD87B23546002D18D00D4800780128CA
:10C150000CD100BF03E000202855601CC4B2082C9D
:10C16000F9D33804000EA870EF7007E0002403E054
:10C1700000202855601CC4B2082CF9D3FEBD000075
:10C1800082000020FFB581B004460F46002500263E
:10C19000002000902760039820810498E060002030
:10C1A000207400BF9DE01C206843216808586A0184
:10C1B000616888501C2068432168081880686A01FB
:10C1C0006168891848601C20684321680818406825
:10C1D0006A016168891888601C2068432168081812
:10C1E000C0686A0161688918C8601C2068432168BA
:10C1F0000818007C6A016168891808741C2068436B
:10C2000021680818407C6A016168891848741C20FC
:10C21000684321680818807C6A01616889188883EE
:10C220001C20684321680818C07C6A01616889186D
:10C23000887400206A0161688918C8741C206843EA
:10C24000216808184068002813D01C206843216822
:10C250000818C07C002805D1401E6A016168891851
:10C26000C8831AE00020C0436A0161688918C88346
:10C2700013E01C20684321680818C07C002805D002
:10C2800000206A0161688918C88306E000206A01FD
:10C2900061688918C88301200090002607E000210A
:10C2A0006A016068801814308155701CC6B269013B
:10C2B00060684018808BB042F1DC1C206843216824
:10C2C0000818406900280AD06B016268D21810462D
:10C2D00014301C236B432268D21851698847681CAC
:10C2E000C5B22089A84200DD5DE7009805B0F0BD29
:10C2F00000B58DB068480890002108A80171684613
:10C30000017708A84171002064498872082108A8B3
:10C31000C171002004E000220AA90A54411CC8B2DD
:10C3200008A9C9798142F6DC5D48FEF71FFF07A91D
:10C330005B48FEF747FF5848401C0890002108A8BA
:10C3400001716846017708A841710020534988723D
:10C35000082108A8C171002004E000220AA90A549B
:10C36000411CC8B208A9C9798142F6DC4C4840306A
:10C37000FEF7FCFE07A94A484030FEF723FF4520A0
:10C3800000010890002108A801716846017708A8FB
:10C390004171002041498872082108A8C17100201C
:10C3A00004E000220AA90A54411CC8B208A9C979AC
:10C3B0008142F6DC3A485030FEF7D8FE07A93848EB
:10C3C0005030FEF7FFFE112040010890002108A820
:10C3D00001716846017708A8417100202F498872D1
:10C3E000082108A8C171002004E000220AA90A540B
:10C3F000411CC8B208A9C9798142F6DC284820301E
:10C40000FEF7B4FE07A926482030FEF7DBFE0B201E
:10C41000C0010890002108A801716846017708A8AA
:10C42000417100201D498872082108A8C1710020AF
:10C4300004E000220AA90A54411CC8B208A9C9791B
:10C440008142F6DC16486030FEF790FE07A91448DA
:10C450006030FEF7B7FE1048A63002900021684613
:10C4600001730171417381730821C173002004E0DD
:10C47000002204A90A54411CC8B26946C97B814202
:10C48000F6DC07481030FEF771FE01A904481030B1
:10C49000FEF798FE0DB000BDEE0600009C260020C1
:10C4A00080550440F0B585B004460F4600250026AF
:10C4B000207C4006400E55287ED100BF76E1690100
:10C4C00060684018807C002877D169016068401856
:10C4D00040686A01616889188968884209D26901DF
:10C4E000606840184068C0196A016168891848602E
:10C4F0005AE1690160684018C068AF49884208D8AD
:10C50000690160684018C068401C6A016168891848
:10C51000C860690160684018C07C002821D10026ED
:10C5200007E000216A016068801814308155701C92
:10C53000C6B2690160684018808BB042F1DC1C20F3
:10C54000684321680818406900280AD06B016268B6
:10C55000D218104614301C236B432268D21851693C
:10C560008847690160684058009069016068401818
:10C57000017C6846017100214171690160684018C1
:10C58000017F68468171690160684018417C684696
:10C59000C171002608E06901606840181430815DAF
:10C5A00002A88155701CC6B2690160684018808B72
:10C5B000B042F0DCE06801E0FCE01DE0002806D0BD
:10C5C0006846E16888476A0161688918C87469012A
:10C5D00060684018C07C002804D16A01616889182D
:10C5E0004860E1E06901606840184068C01B6A016A
:10C5F000616889184860D7E0690160684018806800
:10C600000028EED0690160684018C08B0028E8D08F
:10C61000690160684018C08B6A0161688918C9683F
:10C62000884207D1690160684018C08B6249C943DC
:10C6300088427DD169016068401840686A0161687C
:10C6400089188968884209D2690160684018406881
:10C65000C0196A01616889184860A5E000206A0174
:10C66000616889184860690160684018C06852496B
:10C67000884208D8690160684018C068401C6A0197
:10C6800061688918C860002607E000216A016068B7
:10C69000801814308155701CC6B26901606840185A
:10C6A000808BB042F1DC1C20684321680818406987
:10C6B00000280AD06B016268D218104614301C237F
:10C6C0006B432268D21851698847690160684058F5
:10C6D0000090690160684018017C68460171002182
:10C6E0004171690160684018017F68468171690184
:10C6F00060684018417C6846C171002608E0690105
:10C70000606840181430815D02A88155701CC6B263
:10C71000690160684018808BB042F0DCE068002856
:10C7200008D06846E16888476A016168891800E0B6
:10C7300015E0C874690160684018C07C002804D105
:10C740006A016168891848602EE0690160684018D4
:10C750004068C01B6A0161688918486024E01C2099
:10C76000684321680818406800280FD00020C043A3
:10C770006A0161688918C8831C2068432168081809
:10C7800040686A0161688918886008E000206A01D1
:10C7900061688918C8836A01616889188860002007
:10C7A0006A0161688918C860681CC5B22089A842FE
:10C7B00000DD84E605B0F0BD0000FFFF7CB500BFE2
:10C7C00019212B480078FBF7C1FC04462948604337
:10C7D000294A8118002201200DF032FA20460A224F
:10C7E000504364300119002201200FF09BFA012010
:10C7F0000A2262431219D1B20A226243121900902E
:10C80000D0B201231A4609F0CFFCFF2207210020F5
:10C8100006F09CFF0120009001900B20604302462F
:10C820000B2060430146002301200EF097FF6F208C
:10C830006043014601200FF01BFD10486043024693
:10C84000032101200BF076FF002505E00121284699
:10C850000BF0AAFE681CC5B20F2DF7DB21460B2298
:10C8600051436431C8B20FF067FF0FF055FF7CBD34
:10C870006F000020672B0000A0860100FCB10100C2
:10C8800000200549087005490870054908700549E8
:10C890000870054908707047700000207100002082
:10C8A0006F0000206E0000206D000020F0B589B000
:10C8B00000BF00BF00BF00BF00BF00BF00BF00BF80
:10C8C00000BF00BF00F088F91E2822D3614800781D
:10C8D0003C2805DA5F480078401C5E49087002E099
:10C8E0003C205C4908705B4800781D2805DC5A48EC
:10C8F0000078401C584908700BE057480078002821
:10C9000002D15549087004E053480078401E52494E
:10C910000870032150480078FBF72EFC4F4948432C
:10C92000039005214C480078FBF710FC0890032188
:10C9300049480078FBF720FC0B214843643087B25C
:10C94000454909788A0088180621FBF715FCFF2164
:10C95000F531484386B203213F480078FBF70CFCD1
:10C960000B214843643085B203213B480078FBF734
:10C9700003FC3B4948433B49401804900321364897
:10C980000078FBF7F9FB0B214843C0B20690032166
:10C9900031480078FBF7F0FB0B214843C0B205900B
:10C9A00003212D480078FBF7E7FB6F21484380B255
:10C9B000079003210120039A0BF0BCFE0120089987
:10C9C0000BF082FC01233A461846089909F0C6FE8E
:10C9D000FF21F5313046FBF7CFFBC0B20146029094
:10C9E00001200AF09DFB0022294601200FF09AF950
:10C9F0000022012004990DF023F9012007990FF07E
:10CA000037FC01200346024600900599069809F07C
:10CA1000CBFBFF220721002006F098FE03210E48E1
:10CA20000078FBF7A9FB0B21484384B2012000905A
:10CA300000232246214601900EF090FEFF220321A2
:10CA4000002006F083FEFF220421002006F07EFE77
:10CA500009B0F0BD7100002070000020FCB10100A1
:10CA6000672B0000A0860100002000BF06E0002127
:10CA7000044A1154044A1154411CC8B25A28F6DB26
:10CA8000704700007C200020302100200348007AFD
:10CA9000002801D10149487070470000280A002091
:10CAA000FFB581B004460F463D462089A8422DDDE2
:10CAB0001820684321680818007C002826D1002629
:10CAC00009E00498815D1820684322681018083036
:10CAD0008155701CC6B2082EF3D30121182068437B
:10CAE0002268101841742C20684361680818006A95
:10CAF00000280BD018236B432268D2181046083048
:10CB00002C236B436268D218116A884705B0F0BDC8
:10CB100001460720124BCA1A994211D008DCCA1FDD
:10CB2000FA3A002A14D0102A0CD01F2A14D10DE092
:10CB3000322A0FD0C02A07D0C12A0DD100200DE023
:10CB400001200BE0022009E0032007E0042005E0BB
:10CB5000052003E0062001E0072000BF00BF70476A
:10CB60004103000010B504467D21C9006143084619
:10CB7000322103F0D3FE10BDFF200B4908700020C6
:10CB8000C0430A4908800A490880FF200949087003
:10CB900009490870094908700020094908600949D5
:10CBA00008600949086070475400002056000020C2
:10CBB000580000205A0000205B0000205C0000208C
:10CBC000480000204C000020500000200148006870
:10CBD000704700004C0000200148006870470000CA
:10CBE00048000020014800887047000056000020DF
:10CBF00001480078704700005B0000200148007881
:10CC0000704700005400002010B510F025FD0128E9
:10CC10002CD100F063F8012000F066F803F0E2FE8A
:10CC2000044600F043F804F0C3F8044600F04AF864
:10CC300004F008FB012805D100F03EF8012000F0C7
:10CC400047F805E0002000F037F8002000F040F839
:10CC500000201349086013480068134988421ED217
:10CC600010480068801C0F49086018E000200D493A
:10CC700008600B4800680C49884204D208480068E4
:10CC8000801C07490860002000F028F8012000F00F
:10CC90002BF8002000F00AF8002000F013F810BD77
:10CCA0004C00002048000020FFFFFF7F0149088062
:10CCB00070470000560000200149087070470000CE
:10CCC0005B000020014908807047000058000020E8
:10CCD00001490870704700005C000020014908709D
:10CCE00070470000540000200149087070470000A0
:10CCF0005A0000200021014A117170470060004075
:10CD0000002201494A757047006000400022014935
:10CD10004A767047006000400021014A1172704756
:10CD2000006000400021014A11737047006000401C
:10CD30000021014A11747047006000400021014A3F
:10CD400011757047006000400021014A117670475C
:10CD500000600040002201494A73704700600040B3
:10CD6000002201494A7470470060004010B51C4C15
:10CD70001C49206888421ED106221B49201DFBF752
:10CD8000A0FA002817D11222184920460A30FBF7D2
:10CD900098FA00280FD10622154920461C30FBF7CF
:10CDA00090FA002807D10622124920462230FBF7CC
:10CDB00088FA00280DD000F051FF0A480E4908609B
:10CDC000074814F0B4FA0C4A2C21054814F0DAFA9A
:10CDD00004E02C2221460848FBF74FFA10BD000062
:10CDE000000850007AA7A55A5D07002063070020BD
:10CDF0005707002051070020AC2A002000200849D6
:10CE00000870084908700120074908700020074988
:10CE100008700748074908600020074908707047F4
:10CE20003F0700203E070020410700204607002062
:10CE300025060000780700205007002070B5044642
:10CE400000BF9120604305460A212846FBF77EF982
:10CE50000546284670BD000070B5A8B00546002400
:10CE60000026A0216846FBF721FA00F067FD1E4965
:10CE70000A6814216943505000211B48026814209D
:10CE8000684310184160184802681420684310185D
:10CE9000816015484068002824D000BF17E0600674
:10CEA000060E282E00D316E00F48016814206043B8
:10CEB0000858B1006A4650500B480168142060437E
:10CEC00008184168701C80001150601CC4B20648EC
:10CED000007AA042E3DC00BF620003486946436871
:10CEE0000220984728B070BD282B002030B5A9B08B
:10CEF00000240025A02101A8FBF7D8F900BF25E0F8
:10CF00006006050E00F01AFD1F490A6814216143EE
:10CF1000505000211C4802681420604310184160E2
:10CF2000194802681420604310188160282D0BD224
:10CF300015480168142060430858A90001AA505000
:10CF40000021681C80001150601CC4B20E48007A99
:10CF5000A042D5DC0C484068002813D00A48007A6B
:10CF60004000282806D30848282201A94368022047
:10CF7000984707E00448007A4200034801A9436843
:10CF80000220984729B030BD282B0020FFB585B07E
:10CF900005460E461F460020049003900024029090
:10CFA00001900097681C80004149085A0490002DA8
:10CFB00005D0681E800040184088039003E0A80058
:10CFC0003B49085A039003990E98884205D3049967
:10CFD0000E98884201D80E9C08E0012E01D1049CD5
:10CFE00004E0002E01D1039C00E00E9C3148006853
:10CFF000052805D22F480068401C2E49086053E0E0
:10D0000000202C49086005210798FBF79FF8029043
:10D010000298002844D028480068A04215D226482B
:10D020000068201A019002990198FBF78FF801908F
:10D0300021480168019808181F49086008460068DF
:10D04000A04217D90846046014E01B480068001B82
:10D05000019002990198FBF779F801901648016850
:10D060000198081A1449086008460068A04201D2D5
:10D0700008460460104800680090002E14D10E4845
:10D0800000686330B84201D300970DE064210A487C
:10D0900000686330FBF75AF864214843009003E0CE
:10D0A0000548046000680090009809B0F0BD0000D9
:10D0B000F61A0200D8000020E000002008B5FFF7B3
:10D0C0009DFD01287ED1FFF787FD8949884216D250
:10D0D0000F2088498871C87108468078002801D1DE
:10D0E0000520487083488078052802D100208149B6
:10D0F000487000207F4948728872087047E0FA2023
:10D100007C498871C8717C49088803F093FD7A488E
:10D110008078002815D17749087008468079C87052
:10D120000846C0794871002088704870887272483B
:10D1300000886421484371490860FA206D490871EC
:10D1400025E001206B4908700846807A022805D145
:10D15000012088720020C870487118E06548807A04
:10D16000002814D1022063498872084640788870EC
:10D1700008468079C8700846C07948715E480088C2
:10D18000642148435D490860FA205A490871FFF755
:10D1900023FD5749884277D35648807855494978C6
:10D1A000884229DD54480088642148435149009051
:10D1B000C979504B5B79CA1A4E4988784F490B6838
:10D1C000002100E086E0FFF7E1FE4C490860002006
:10D1D0004849C870087108464079401C48710846A3
:10D1E0004079C979884255DB002042494871084698
:10D1F0008078401E88704DE03E4880783D494978EF
:10D20000884227DA3C480088642148433949009025
:10D210008979384BDB78CA1A3649887837490B68E0
:10D220000121FFF7B3FE35490860002031494871FC
:10D2300008710846C078401CC8700846C0788979D3
:10D24000884227DB00202B49C87008468078401CA4
:10D2500088701FE0002027494871C870FA200871C3
:10D260002548008864214843224900900979FA231F
:10D270005A1A2049887821490B680221FFF786FE57
:10D280001E49086006E0FFE71B4800886421484308
:10D290001A49086018488078002803D101201549F0
:10D2A000487223E003F004F8732803DB02201149DD
:10D2B00048721BE002F0FCFF702803DC00200D49DF
:10D2C000487213E00B48407A01280FD10020094929
:10D2D00048720BE000200749087008468079C87042
:10D2E0000846C079487100204872887208BD000065
:10D2F000D60B000070200020D4000020DC000020AD
:10D300000020044988704870C8704871487288725B
:10D3100070470000702000200020064908808870B7
:10D32000054988704870FA20C8704871002048721A
:10D3300088727047D400002070200020F8B50024C7
:10D3400000250026002703F07DFB044603F08CFB3C
:10D350000546FFF753FC01282ED105211A48FDF799
:10D36000F7FE552804D1002018498870088027E06E
:10D37000012D04D1002015498870088020E001208B
:10D38000124988701248844202DB201A84B200E0FD
:10D3900000240A212046FAF7EFFE052901DB601D73
:10D3A00084B20C48844200DD04460A212046FAF784
:10D3B000E3FE0649088003E00020044988700880E5
:10D3C000FFF77CFEF8BD000084080020D400002098
:10D3D000AA0A0000C60700001CB5002000900190BA
:10D3E00000F0ACFA0B49086000200B49096808609E
:10D3F0000A48006800280CD00749096808680A2113
:10D40000FAF7A4FE0090012269460520034B1B6831
:10D4100098471CBD140800200808002010080020B0
:10D4200000200849488008490880084908800849C0
:10D4300008700849887208490880488001200871EE
:10D44000704700002C0000201C0000201E0000205F
:10D45000200000206808002024000020F8B503F018
:10D46000D3FA074603F0E2FA0090FFF7C7FB012862
:10D4700060D10521C548FDF76BFE552802D0009804
:10D48000012807D10020C2490870C2490880C2495A
:10D49000887256E0BE480078002810D10120BC49AF
:10D4A00008703D462846E917890F091889030D0CB5
:10D4B000BA48854200DD0546B648058041E0B648D9
:10D4C000807A4000B4490F520846867A0EE0700018
:10D4D000B1490D5A701E4000085A7100AE4A5052B0
:10D4E000701E400011460D52701EC6B2002E08DD9F
:10D4F0007000A949095A701E4000A74A105A81427B
:10D50000E5DBA548807A401CA34988720846807AEA
:10D51000052816DB002088720846C5882846E917CA
:10D52000890F09188D109D48854200DD05469948F0
:10D53000058006E0002096490870964908809649C3
:10D5400088729448058896480088A84257DA94481B
:10D550000088281A84B292480079012827D190487F
:10D560004088A0420BDA8E4840880A308C494880B7
:10D5700008464088A04204DD0846448001E088480F
:10D5800044808748448803212046FAF7F5FD84B299
:10D59000192C00DA19248248008800198049088073
:10D5A00008460088A84201DD08460580CDE07C4899
:10D5B0004088142805DD7A48408814387849488026
:10D5C00002E00020764948807548448803212046BF
:10D5D000FAF7D2FD84B2192C03DA012070490871E0
:10D5E000B3E06F480088A04205DD6D480088001B4D
:10D5F0006B490880A9E0002069490880A5E06848D7
:10D600000088A84259DD66480088401B84B26448FF
:10D610000079012827D162484088142805DD604838
:10D62000408814385E49488002E000205C49488008
:10D630005B48448803212046FAF79EFD84B2192CEA
:10D6400003DA0220564908717FE055480088001926
:10D6500053490880084600885049884275DD0846CD
:10D660004F49088071E04E484088A0420BDA4C4890
:10D6700040880A304A49488008464088A04204DD74
:10D680000846448001E046484480454844880321D8
:10D690002046FAF771FD84B2192C00DA19244048AB
:10D6A00000882919884202DA3D4805804DE03C484F
:10D6B0000088001B3A49088047E039484488032124
:10D6C0002046FAF759FD84B2192C3EDD34484088D3
:10D6D000142805DD3248408814383149488002E07A
:10D6E00000202F4948802E48448803212046FAF71D
:10D6F00043FD84B22A480079012813D1192C03DA9A
:10D7000002202749087120E0254800880019244993
:10D710000880084600882149884216DD08462049CD
:10D72000088012E0192C03DA01201D4908710CE071
:10D730001B480088A04205DD19480088001B1849D5
:10D74000088002E00020164908801648008850280A
:10D7500004DC134800881349088016E0104800884C
:10D7600010490988884204DD0D4800880D49088069
:10D770000BE00B4800880B490988081A84B2502C2A
:10D7800003DB0748008807490880F8BD84080020AB
:10D79000200000201C00002068080020E02E00006F
:10D7A000240000201E00002010B5044664204443DD
:10D7B000A1212046FAF7CAFC0446204610BD00000D
:10D7C00010B501200F49087000200F490968086052
:10D7D0000D49096848600C490968886000F07EF9C5
:10D7E000FFF7FAFDFFF782FB08480068002807D022
:10D7F00001220548016808310020044B1B68984746
:10D8000010BD0000E1070020DC070020D807002041
:10D8100010B5184800681849884229D1174800688F
:10D82000002804D01548006880471549087015483D
:10D830000068002804D01348006880471249087027
:10D8400012480068002804D010480068804710493A
:10D85000088010480068002805D00E4800688047FE
:10D860000D49088002E00D480B49088000F078F867
:10D8700010BD0000EC07002078563412C8070020C5
:10D88000E0070020CC070020E2070020D00700209E
:10D89000E4070020D4070020E6070020102700003E
:10D8A00010B50023174C2360174C2370174C2370BE
:10D8B000174C2370174C2380174C2380174C237070
:10D8C000174C13682360174C53682360164C9368F9
:10D8D0002360164CD3682360154C1369236000281D
:10D8E0000CD0144B1860134C0B682468A360002301
:10D8F000104C246823600F4C246863600E4B014C6D
:10D90000236010BDEC070020E8070020E00700209E
:10D91000E2070020E4070020E6070020E1070020DE
:10D92000C8070020CC070020D0070020D407002023
:10D93000D8070020DC07002078563412054800681C
:10D940000549884203D10548006880687047002077
:10D95000C043FBE7EC07002078563412DC070020B8
:10D9600070B50024002500263048007801285CD1DD
:10D970002F480078002858D12E480078012854D12B
:10D980002D4805882D490988694308462C49FAF72E
:10D99000DDFB85B2E1200001854207D819216943EA
:10D9A00008460921FAF7D2FB044600E0244C25483A
:10D9B0000068006800192349096808602148006868
:10D9C0000068204909684968884207D31D480068F3
:10D9D00000681C4909684968461A0AE01948006845
:10D9E00040680021C943081A1649096809684018A7
:10D9F000461C1548864218D3344601462046FAF79D
:10DA0000A5FB04460F48006841680F4860430818AA
:10DA10000C490968486001200C49087009480068F1
:10DA20008068001907490968886070BDE007002018
:10DA3000E1070020E2070020E4070020E6070020BD
:10DA400010270000DC070020A0860100E807002066
:10DA500000220C4B1A600C4B0A681A600B4B4A6888
:10DA60001A600B4B8A681A600A4BCA681A600A4B24
:10DA70000A691A60002801D0084A1060084A014B60
:10DA80001A607047EC070020C8070020CC07002070
:10DA9000D0070020D4070020D8070020DC07002092
:10DAA0007856341210B50A48006800280ED009488C
:10DAB000007801280AD10020064908700122064892
:10DAC000016808310020024B1B68984710BD000018
:10DAD000D8070020E8070020DC0700201CB5002044
:10DAE000009001900024FFF729FF04460E480068CB
:10DAF000046000200C49096848600B490968886087
:10DB00000A48006800280DD00748006800680090A7
:10DB10000548006840680190022269460120034BD5
:10DB20001B6898471CBD0000F0070020F407002088
:10DB3000F8B505460C4616460027002D17D00E48AE
:10DB40000560FFF7FBFE07462068B84203D90A4884
:10DB50000068076003E00849206809680860064912
:10DB60006068096848600449A0680968C86003489B
:10DB7000066000F005F8F8BDF0070020F40700206B
:10DB800070B500240025FFF7D9FE04460F48006851
:10DB90000068A04200D903E00C4800680068251A1C
:10DBA0000A480068406840190849096888600748C1
:10DBB0000068806805490968C968884205D9034832
:10DBC0000068C06801490968886070BDF0070020DE
:10DBD0000148006880687047F0070020002801D0E5
:10DBE000024A1060024A116070470000F0070020EE
:10DBF000F40700200549002005E00A1D135C044AD3
:10DC00001354421CD0B22028F7DB704700065000A6
:10DC1000DC2A0020014610480268142048431018EE
:10DC200082680D480368142048431818C06882426F
:10DC30000BD909480268142048431018C2680648E6
:10DC400003681420484318188260034802681420AF
:10DC50004843101880687047282B002010B5002119
:10DC60000022002005E01B4B1C5C1B4B1C54431C7A
:10DC7000D8B20628F7DB1221002006E0174B1C5C07
:10DC8000154B9B1D1C54431CD8B28842F6DB002068
:10DC900006E0134B1C5C104B18331C54431CD8B2C9
:10DCA0000628F6DB002006E00E4B1C5C0A4B1E33F8
:10DCB0001C54431CD8B20628F6DB0422002005E0E1
:10DCC0000024054B24331C54431CD8B29042F7DB8C
:10DCD00010BD00005D070020B02A0020630700206F
:10DCE000570700205107002038B504460020009057
:10DCF000009401226946FF202130FBF799F938BDD5
:10DD000008B50020009002226946FF204130FAF752
:10DD1000D1FF684600780F49C8716846407808729C
:10DD20000846C0790C4948730A48007A8873094844
:10DD3000407AC8730748807A08740020087307493E
:10DD400008600749086007490860074908600749F3
:10DD5000087008BD30220020EC090020840000205B
:10DD6000880000208C0000209000002094000020FB
:10DD700008B50020009002226946FF204130FAF7E2
:10DD800099FF684600781249C87168464078087261
:10DD900000201049086048600872487288720C4878
:10DDA000C07948730A48007A88730948407AC87372
:10DDB0000748807A087400200873074908600749FB
:10DDC000086007490860074908600749087008BDEE
:10DDD00030220020EC090020840000208800002070
:10DDE0008C000020900000209400002038B5002412
:10DDF0000025002000900121F948FDF7A9F95528D8
:10DE00000AD002F075FEF749487302F085FEF54925
:10DE100088730120087308E0F348C079F14948731A
:10DE2000F148007A8873002008730621EC48FDF75A
:10DE30008FF9552830D002F0A3FE002808D002F058
:10DE40009FFE401C002803D00120E649087502E02F
:10DE50000020E449087502F075FE002808D002F0A1
:10DE600071FE401C002803D00120DE49C87402E086
:10DE70000020DC49C87402F083FE002808D002F0BC
:10DE80007FFE401C002803D00120D649087507E01A
:10DE90000020D449087503E00020D249C8740875F1
:10DEA000D048407B00282BD1D0490860D04800687A
:10DEB000D049884208D8CE480068401CCC49086048
:10DEC0000020C84948736CE0C748C079022812D0C6
:10DED000C548C07903280ED00121C148FDF738F9A3
:10DEE000552803D00320BF4948735AE0BE48C07983
:10DEF000BC49487355E0BC48C079BA49487350E002
:10DF0000B848407B01282CD10020B9490860B748A7
:10DF10000068B849884208D8B4480068401CB34932
:10DF200008600120AF4948733BE0AF48C079022840
:10DF300012D0AD48C07903280ED00121A848FDF7C2
:10DF400007F9552803D00320A649487329E0A648BD
:10DF5000C079A449487324E0A348C079A149487313
:10DF60001FE0A048407B022805D10020A04908609E
:10DF70009E49086015E09B48407B032808D100209B
:10DF80009B4908609949086003209649487308E056
:10DF9000002097490860954908609348C0799149E5
:10DFA00048739048807B00282BD1934908609348A0
:10DFB00000689049884208D890480068401C8F4902
:10DFC00008600020874988736CE08748007A02283F
:10DFD00012D08548007A03280ED001218048FDF731
:10DFE000B7F8552803D003207E4988735AE07E484D
:10DFF000007A7C49887355E07B48007A79498873B8
:10E0000050E07848807B01282CD100207B490860B3
:10E01000794800687749884208D877480068401CEA
:10E020007549086001206F4988733BE06E48007AAB
:10E03000022812D06C48007A03280ED001216848CB
:10E04000FDF786F8552803D003206649887329E038
:10E050006548007A6349887324E06348007A61491F
:10E0600088731FE05F48807B022805D10020634948
:10E0700008606149086015E05A48807B032808D190
:10E0800000205E4908605C49086003205549887398
:10E0900008E0002059490860574908605248C07993
:10E0A000504988734F48407B4F49C979884205D110
:10E0B0004C48807B4C49097A884251D04948407B82
:10E0C0004949C979884202D001204649C873454868
:10E0D000807B4549097A884202D001204149087471
:10E0E0004048407B022803D03E48407B032817D19C
:10E0F0003C48407B3C49C979884211D03948407B33
:10E100003949C8710846C179684601703648017AB4
:10E110006846417002226946FF204130FAF788FFC5
:10E120003048807B022803D02E48807B032817D1FB
:10E130002C48807B2C49097A884211D02948807B61
:10E14000294908720846C179684601702648017A53
:10E150006846417002226946FF204130FAF768FFA5
:10E1600002F0D0FC044602F0E3FC054601211C4805
:10E17000FCF7EEFF552807D100201A4908724872B3
:10E18000086048608872B9E0FF2C01D0FF2D77D17C
:10E19000FF2C3FD1FF2D3DD00020124908720120F5
:10E1A0004872174808601748684348604868662105
:10E1B000F9F7CCFF0B49486008464068124988428D
:10E1C00002D908460749486002F0D8FF112803DB4E
:10E1D00002F0D4FF192819DD0120024988728DE070
:10E1E00084080020EC090020302200208800002054
:10E1F0008400002070170000900000208C00002098
:10E20000DE030000BE0A0000AC26000000205D49CD
:10E21000887273E0FF2C29D0FF2D27D101205949A6
:10E2200008720020487258484860584860430860A7
:10E2300008686621F9F78AFF5249086008460068B5
:10E240005349884202D908464E49086002F08EFEC2
:10E25000112803DB02F08AFE172803DD012049495B
:10E2600088724BE000204749887247E0484845499A
:10E270000860486000208872087248723EE0FFE73C
:10E2800001204049087248724048604308600868AD
:10E290006621F9F75BFF3B490860084600683C4986
:10E2A000884202D9084637490860384868433549EA
:10E2B000486048686621F9F749FF324948600846D6
:10E2C00040683349884202D908462E49486002F026
:10E2D0004DFE11280BDB02F049FE172807DC02F087
:10E2E0004DFF112803DB02F049FF192803DD01204F
:10E2F0002449887202E00020224988722148407B2C
:10E30000002802D11F49C87315E01E48407B012830
:10E3100002D11C49C8730EE01A48407B022802D182
:10E320001849C87307E01748407B032803D11549F3
:10E33000C873174808601348807B002802D1114930
:10E34000087415E00F48807B012802D10D4908743C
:10E350000EE00C48807B022802D10A49087407E0CD
:10E360000848807B032803D10649087408484860A0
:10E370000448406807490860024800680649086088
:10E3800038BD0000EC090020DE030000BE0A0000DA
:10E39000AC260000980000209C000020FFB583B050
:10E3A00006460D46174600240020029000BF1420A8
:10E3B000784380190190002E57D00198002854D03E
:10E3C0002B4806602A49069848600846077200BF35
:10E3D00045E0FFF7B3FA02902001295802988142E4
:10E3E00004D820012858401C002806D12049029852
:10E3F0000A6814216143505006E0200129581C4846
:10E400000268142060431150200140194068401CEC
:10E41000002807D100211648026814206043101814
:10E42000416008E020014019416811480268142049
:10E430006043101841602001401981680C4802684F
:10E44000142060431018C16020014019017B084866
:10E4500002681420604310180161601CC4B20448B3
:10E46000007AA042B5DC00F005F807B0F0BD00006E
:10E47000282B002070B5002400250026FFF75EFA47
:10E48000054600BF4EE02A48016814206043085842
:10E49000A84239D8264801681420604308582E1A2B
:10E4A00023480168142060430818406881192048F7
:10E4B000026814206043101881601D480168142010
:10E4C0006043081881681A480268142060431018D5
:10E4D000C068814224D91648016814206043081896
:10E4E0000069002803D02046FEF7B6FC18E010486B
:10E4F0000168142060430818C1680D4802681420A0
:10E500006043101881600BE00948016814206043E3
:10E510000818406806490A68142161435118886048
:10E52000601CC4B20248007AA042ACDC70BD00009E
:10E53000282B002010B500BF14244C4323180028BA
:10E5400005D0002B03D0024C20606260217210BD08
:10E55000282B0020F8B506460F4614460025002E4D
:10E5600004D0012E10D0022E52D12FE02A48FAF703
:10E57000A7FA2A4908802848F9F7B0FE64210090DC
:10E58000F9F7E4FD386044E00025A004020C3946A8
:10E590002020FAF78FFB2149088011E0A004020C2B
:10E5A00039462020FAF786FB1C490880681C85B292
:10E5B00008460088022800D106E0032D00DB03E0B6
:10E5C000164800880228E9D100BF22E00025A004F7
:10E5D000020C39466020FAF76DFB1049088011E003
:10E5E000A004020C39466020FAF764FB0B4908804E
:10E5F000681C85B208460088022800D106E0032D79
:10E6000000DB03E0054800880228E9D100BF00E0F4
:10E6100000BF00BF0020F8BD22220020F80000202B
:10E62000F8B507460E4614460025002F04D0012FEA
:10E630001AD0022F5CD139E03068002802D1FAF7F5
:10E64000C7F810E064223168514308462A49F9F7B7
:10E650004FFE002029490880012264212648FAF74C
:10E6600097FB2649088044E00025A004020C3146AF
:10E670002020FAF7DDFC2249088011E0A004020CFA
:10E6800031462020FAF7D4FC1D490880681CC5B229
:10E6900008460088022800D106E0032D00DBF8BD03
:10E6A000174800880228E9D100BF22E00025A00415
:10E6B000020C31466020FAF7BBFC1249088011E0D9
:10E6C000A004020C31466020FAF7B2FC0D49088024
:10E6D000681CC5B208460088022800D106E0032D58
:10E6E00000DBDCE7074800880228E9D100BF00E032
:10E6F00000BF00BF00BFD2E714220020F0000020BE
:10E70000F2000020F400002000B5B5B0502121A88F
:10E71000F9F7CCFD14211CA8F9F7C8FD00201B90C7
:10E72000142116A8F9F7C2FD00201390149015903B
:10E730001290402102A8F9F7B9FD0020019042494A
:10E740000860012221A9FFF705FF2198401C00283D
:10E7500001D11B9001E021981B903C4816903C4849
:10E7600017903C481890002019903B481A9016AA20
:10E770001BA93A48FFF794F8022222A90120FFF7CB
:10E78000E9FE2298401C002801D1139001E0229854
:10E7900013902298401C002801D1149001E0229887
:10E7A00014902F48159013A92E481A9AFFF7C0F914
:10E7B000022224A91046FFF7CDFE2498401C002811
:10E7C00001D1029001E0249802902598401C002875
:10E7D00001D1039001E02598039023480490012182
:10E7E00068460175012202A920481A9BFFF7D6FD51
:10E7F00001221CA9FF202130FAF75CFA18A8007C3E
:10E80000FF2808D101201A4988710122891DFF20A3
:10E810002130FAF70DFC02221CA9FF204130FAF743
:10E8200049FA18A8007CFF2809D100216846017127
:10E830004171022201A9FF204130FAF7F9FB0D488E
:10E840000149086035B000BDFC000020FDCB000090
:10E85000F1CB0000E5CB000021E60000E421002020
:10E8600076841E00F02100200F27000000220020E7
:10E8700030220020A33AA55A00B585B0142168467D
:10E88000F9F714FD00200F4908600F4800900F4869
:10E8900001900F480290002003900E4804906946B2
:10E8A0000D48FFF7D5F80D480499FFF797F90121B6
:10E8B0000B48049AFFF73EFE0A480249086005B07B
:10E8C00000BD0000FC000020FDCB0000F1CB0000EB
:10E8D000E5CB000021E60000E4210020F02100202B
:10E8E00000220020A33AA55A00200C4908800C49B8
:10E8F00008800C49088001200B49087000200B4952
:10E9000008730B49088048800120087100200749DE
:10E9100048800880074908607047000034000020E4
:10E92000360000203C0000203E000020740800203B
:10E930004000002038000020F8B502F09FF806469D
:10E9400002F0A6F80746FEF759F9012865D105211E
:10E95000AB48FCF7FDFB552807D10020A9490870FA
:10E96000A9490880A94988805FE0012F07D10020CC
:10E97000A4490870A4490880A449888055E0A148AA
:10E980000078002808D101209E49087035460A20E9
:10E9900068439D49088048E09C48007B41009B48B3
:10E9A000801D4652801F047B11E061009748801D46
:10E9B000455A601E41009548801D415A62008152AF
:10E9C000601E41009148801D4552601EC4B2002C5B
:10E9D0000ADD61008D48801D415A601E42008B484F
:10E9E000801D805A8142E0DB8848007B401C8749BB
:10E9F00008730846007B032807DB002008730846DD
:10EA000005890A206843804908807F4800887F493B
:10EA1000888001207B49087007E000207949087050
:10EA2000794908807949087388807748008878494F
:10EA3000086074480078002815D0084600686C21EA
:10EA4000484373490860642171480068F9F77EFB08
:10EA50006F490860084600686E49884206D9084632
:10EA60006B49086002E00020694908606848006856
:10EA700069490988884203D2654800680F2804D292
:10EA800063480088644908800AE063480088604958
:10EA90000968401A0F2803D35D4800885E49088042
:10EAA0005A480088401C59490880084600880A28AE
:10EAB0002CDB002008805948008857490988884283
:10EAC00003DA01205649087108E054480088524989
:10EAD0000988884202DD02205149087150480079B6
:10EAE000012840D14C4800884C49098888420DDBF8
:10EAF0004948018849480088FF309130814206DD4D
:10EB000046480088FF3073304449088077E0424827
:10EB10000188424800889630814205DD3F480088E0
:10EB200078303E4908806AE03B4801883B480088CD
:10EB30003230814205DD394800881E30374908806F
:10EB40005DE035480188354800880A30814205DD9E
:10EB5000324800880A303149088050E02E48008849
:10EB60002E4908804BE02E480079022847D12A48D8
:10EB700000882A490988884239DA27480088FF3006
:10EB8000913026490988884206DA24480088FF38EF
:10EB90007338224908802AE01F48008896301F49B0
:10EBA0000988884205DA1D48008878381B490880A2
:10EBB0001DE019480088323018490988884205DA72
:10EBC000164800881E381549088010E01248008851
:10EBD0000A3012490988884205DA104800880A3844
:10EBE0000E49088003E00C4800880C4908800B4857
:10EBF00000880849884202DB084608490880F8BDB9
:10EC0000840800203E00002034000020740800200A
:10EC100038000020C60700003C000020360000201D
:10EC20004000002000200849088008490880084961
:10EC3000088048800120087100200649488008802B
:10EC40000549086070470000360000203C000020A5
:10EC500040000020740800203800002000200349F4
:10EC6000087003490870034988777047A0000020A6
:10EC7000A1000020040A002070B500250024FDF743
:10EC8000BDFF01284FD103212A48FCF761FA55281E
:10EC900007D100202849087028490870284988773A
:10ECA00046E026480078002807D101F087FF224976
:10ECB00008700120214908703AE001201F490870BE
:10ECC00001F07CFF1E49897F1D4A50541046847F05
:10ECD00008E01B48055D601E1949085C0855601E68
:10ECE0000D54C4B2002C06DD1548015D601E144AA7
:10ECF000105C8142EDDB1248807F401C1049887710
:10ED00000846807F1E2813DB00208877897B0C4A09
:10ED1000D27B89180A4A127C88180321F9F72CFA49
:10ED20000549087004E00020034908700349087091
:10ED300070BD000084080020A0000020A100002079
:10ED4000040A0020F0B5A9B004460E4600250027AD
:10ED500000202890A0216846F9F7A8FAFEF7EEFDFA
:10ED600026490A6814216143505024480168142040
:10ED700060430818C068B0420CD2204801681420D3
:10ED800060430818C1681D480268142060431018C9
:10ED9000416005E019480168142060430818466086
:10EDA00016484068002826D0002517E06806070EA0
:10EDB000282F00D316E01148016814206843085832
:10EDC000B9006A4650500D4801681420684308187D
:10EDD0004168781C80001150681CC5B20748007A51
:10EDE000A842E3DC00BF6A00044869464368022089
:10EDF000984701202890289829B0F0BD282B0020A2
:10EE000010B500F0F9FD00F0D7F810F095FE00F015
:10EE10000DFB00F001F810BD70B541480078912855
:10EE200000D070BD00F0BEF8012876D13D480088C2
:10EE30003D49088008468078F021884320303A49CF
:10EE4000887008468078000900013549097A090769
:10EE5000090F0843344988703148807A401E304990
:10EE6000887208460089401C088108460089C988C4
:10EE7000884216DA08202C49887200240EE02848BF
:10EE800041882848001D415C2748C01C0155244882
:10EE90004088401C22494880601CC4B2072CEEDB2D
:10EEA0002DE01F4800891E49C98888421CD11C4892
:10EEB00000791B498978401AC5B2681C1A498872C2
:10EEC00000240EE0164841881648001D415C164893
:10EED000C01C015512484088401C11494880601CE4
:10EEE000C4B2AC42EEDB0AE000F012FD00200C4997
:10EEF00008700C490888092100F0B8F991E7012051
:10EF000000F0C8FC084A917A1088921C00F070F951
:10EF100005490888002100F0C1F800BF81E7000022
:10EF200060280020FC2700208C2700201B49097E38
:10EF3000002932D01949897E0C225143174A515A6F
:10EF4000174A118000200CE01449897E0C2251439D
:10EF5000124A8918891C0A5C1149891C0A54411CEF
:10EF6000C8B20828F0DB0D49897E0C2251430B4AB8
:10EF70008918897A0A4A91720121D1720749097E5A
:10EF8000491E064A11761146897E491C9176114622
:10EF9000897E022901DB00219176704758270020E5
:10EFA000802700200349487B012802D10021014A23
:10EFB000517370477028002010B53348406800280E
:10EFC00061D13148007B030011F09CFE0759051206
:10EFD000212E3D4A59002D480078002807D00020F6
:10EFE0002A4908702A490888012100F03FF947E0C2
:10EFF00026480078002809D00020244908702549B7
:10F000004A8808880123091D00F040F938E01F48AC
:10F010000078002807D000201C4908701C49088887
:10F02000022100F023F92BE018480078002809D0CD
:10F0300000201649087017494A8808880923091DC5
:10F0400000F024F91CE011480078002807D00020C7
:10F050000E4908700E490888092100F007F90FE0F1
:10F060000A480078002809D000200849087009499A
:10F070004A8808880323091D00F008F900E000BF52
:10F0800000BF00F045FC10BD702800206028002063
:10F09000FC270020982700207047000070B5044628
:10F0A0000D4634480088A04263D1002D61D132481A
:10F0B000007822284ED004DC20283DD0212856D1CB
:10F0C00041E0902802D0912851D115E02A48C0880B
:10F0D00001280AD100202849087000F019FC2749AE
:10F0E0000888002100F0C2F805E0032000F0D2FB00
:10F0F000A020214908703BE01F4800891E49C988AB
:10F1000088420AD100201C49087000F001FC1B490C
:10F110000888002100F0AAF80DE01748807A00283E
:10F1200006D000F0F5FB1449087B00F095FB02E0E7
:10F13000032000F0AFFB1BE0062000F0ABFB11202A
:10F140000D49087014E0062000F0A4FB11200A49C4
:10F1500008700DE000200849087000F0D9FB08494C
:10F160004A8808880923091D00F090F800E000BFD4
:10F1700000BF70BD7427002060280020FC270020FD
:10F180009827002070B50346184C247E022C00DB23
:10F1900070BD164C647E0C256C43144D2B5300201F
:10F1A0000AE0155C114C647E0C2674430F4EA419C2
:10F1B000A41C2554441CE0B28842F2D30B4C647E5C
:10F1C0000C267443094EA419A1723446247E641C93
:10F1D00035462C762C46647E641C6C762C46647E08
:10F1E000022C01DB00246C7600BFD1E758270020F9
:10F1F000F0B587B007460D4616461A48078000242A
:10F2000006E031781748801C0155761C601CC4B29A
:10F21000AC42F6DB2C4605E0AA211248801C0155C1
:10F22000601CC4B2082CF7DB0E480088029008214D
:10F230006846C1730021417301730171002406E027
:10F240000848801C015D04A80155601CC4B2082C4C
:10F25000F6DB01A90448FCF707F90120014988728F
:10F2600007B0F0BD742700209055044070B50446E7
:10F270000D462946204610F081FB70BD70B504464E
:10F280000D462946204610F087FB70BDF8B50446B0
:10F290000D4616461F463B4632462946204610F08C
:10F2A0007CFBF8BDF8B507460E4615465C4800786D
:10F2B000002804D009213846FFF7D8FFF8BD002DFB
:10F2C00001D0602D04DD09213846FFF7CFFFF5E7B7
:10F2D000544807804580002406E031785148001DDD
:10F2E0000155761C601CC4B2AC42F6DB00204C49D0
:10F2F000487008468580FF2088727F200873084682
:10F30000808808282EDA0120C88008468088488036
:10F3100001200881434800884349088008468078D6
:10F32000F021884340498870084680780009000130
:10F330003B4909790907090F08433B498870384858
:10F340000079401C8872002407E03648001D015DEA
:10F350003548C01C0155601CC4B231488088A042A9
:10F36000F3DC4AE00721681CF8F706FF002907D004
:10F37000072128460830F8F7FFFE2949C88005E034
:10F380000721681CF8F7F8FE2549C88006202449A3
:10F3900048800120088123480088234908800846C6
:10F3A0008078F021884310301F49887008468078A3
:10F3B000000900011A4989880905090F08431A49FB
:10F3C000887008464088FF210902884314498988CB
:10F3D0000902FF2212021140084313494880082005
:10F3E0008872002407E00F48001D015D0E48001DD3
:10F3F0000155601CC4B2062CF5DB012000F04AFA6E
:10F40000094A917A1088921CFFF7F2FE9020044975
:10F410000870054908880021FFF740FE00BF4DE74E
:10F4200060280020FC2700208C27002010B5FFF763
:10F430007DFD1448C07A002822D012488078000947
:10F44000002806D0012807D002280AD0032810D1AE
:10F450000CE000F0A7F90FE000F09EF800F066FA6B
:10F460000AE000F011F800F061FA05E000F000F9A0
:10F4700002E0FFF711FE00BF00BF00200149C87283
:10F4800010BD00008027002010B53F4800781128EB
:10F4900000D010BD3D4800883D49884200D0F8E7C3
:10F4A0003A4880780007000F3749097A0907090FA1
:10F4B00088420CD000203449087000F029FA354900
:10F4C0004A8808880423091DFFF7E0FEE1E72E487B
:10F4D0000089401C2C4908810846807A401E8872A9
:10F4E00008460089C98888421BDA2848807A08289B
:10F4F00000D0CEE700240EE02448C01C015D224865
:10F5000042882448001D81541F484088401C1E49E1
:10F510004880601CC4B2072CEEDB062000F0BAF96C
:10F5200030E01948808818494988401A1749897A73
:10F53000884203DA1548807A082800D0A9E7002419
:10F540000EE01248C01C015D0F4842881148001DA2
:10F550008154601CC4B20C484088401C0A49488051
:10F5600009484088084989888842EADB0020064922
:10F57000087000F0CDF907494A8808880023091D62
:10F58000FFF784FE00BF84E760280020802700206A
:10F59000140700009827002070B5314800788021BA
:10F5A0000840802800D170BD2E4800882E4988422E
:10F5B00000D0F8E72B48807A082800D0F3E72948E4
:10F5C000807805072D0F2D0226484088000A054344
:10F5D000082D00DAE7E7002021494870062048801E
:10F5E0000846858001200881082088720020C872A2
:10F5F0008988481C0721F8F7BFFD002909D0184960
:10F600008988084608300721F8F7B6FD1449C880F4
:10F6100007E013498988481C0721F8F7ADFD104918
:10F62000C880104800881149088008464580002499
:10F6300007E00C48001D015D0C48001D0155601CD1
:10F64000C4B2062CF5DB042000F024F91020044994
:10F650000870064A51881088FFF710FE00BFA2E725
:10F660006028002080270020140700009827002031
:10F6700010B548480078A02808D04648007891285E
:10F6800004D044480078A12800D010BD424800882A
:10F69000424988420AD0424908880921FFF7E6FD1D
:10F6A00000F036F900203B490870EEE73A48807ACE
:10F6B00008280AD03A4908880921FFF7D7FD00F049
:10F6C00027F9002033490870DFE7334880780007C6
:10F6D000000F002804D001282DD002284BD136E09D
:10F6E0002C484078002800D050E02B48C0780028F3
:10F6F00003D101202749487003E02748C0782549F5
:10F7000088722448007891280BD02348007900287B
:10F7100003D101201F49087303E01F4800791D49E8
:10F72000087391201B49087000F0F2F81949087B12
:10F7300000F092F82AE017484078002800D025E031
:10F74000A12014490870032000F0A4F81EE011481D
:10F750004078002800D019E00E480078A02809D190
:10F760000F4908880821FFF781FD00F0D1F800203B
:10F77000084908700AE00A4908880521FFF776FD64
:10F7800000F0C6F800200349087000BF00BF00BFAA
:10F790007BE700006028002080270020140700007D
:10F7A000FC27002010B528480078802108408028D8
:10F7B00000D110BD24480078002805D023480088D7
:10F7C0002349884200D0F4E72048807A1F4989788D
:10F7D0000907090F884203DD1C48807A082800D0F9
:10F7E000E7E71A4880780007000F002805D017487F
:10F7F00080780007000F072800DDDAE7134800884B
:10F8000014490880114880780007000F48800024C0
:10F8100007E00E48C01C015D0E48001D0155601C2C
:10F82000C4B20C484088A042F3DC002006490870AE
:10F8300000F06EF807494A8808880023091DFFF781
:10F8400025FD00BFB5E700006028002080270020CC
:10F8500014070000982700207F2805DC7D21C900BF
:10F8600041430A4A91600DE0F12808DBF92806DCE3
:10F870000107090F64225143044A916002E00449E0
:10F88000024A91600221014A51737047702800209A
:10F8900018F0010000B5030011F034FA0729050B38
:10F8A00011171D2329000121144A117314495160B5
:10F8B00022E00221114A1173114951601CE0032119
:10F8C0000E4A11730F49516016E004210B4A11735F
:10F8D0000D49516010E00521084A11730021516063
:10F8E0000AE00621054A11730849516004E000212D
:10F8F000024A1173516000BF00BF00BD7028002094
:10F90000A8610000F824010028230000F04902004B
:10F9100000200149087370477028002002490988B7
:10F920000918014A118070477028002010B52E4830
:10F930000078102818D12D48408860280ADD2C480E
:10F94000807800090001801C2949887022202649FE
:10F95000087025E026488078000900012449887055
:10F960002020214908701BE01F480078112816D17B
:10F970001D48807A002800D010BD1B484078002820
:10F9800000D0F9E7082018498872194880780009E2
:10F9900000011749887020201349087000E0EBE748
:10F9A00014481349088008468078F0218843303095
:10F9B0000F4988700846C0780020C8700846007952
:10F9C00014200871032088720220FFF763FF084AA1
:10F9D000917A1088921CFFF70BFC054908880021DA
:10F9E000FFF75CFB00BFC7E76028002098270020D6
:10F9F0008C27002094070000244A118852888A42EC
:10FA000042D0224A52888A4204DA204A52888A1A0C
:10FA100090B207E01D4A52880023DB439A1A521C19
:10FA2000521890B2194A5180127B002A10D0174AFE
:10FA30005268002A0CD0154A5268824205D9134AEE
:10FA40005268121A114B5A6002E000220F4B5A60A2
:10FA50000E4A527B022A17D10C4A9268002A0CD017
:10FA60000A4A9268824205D9084A9268121A074BDC
:10FA70009A6002E00022054B9A60044A9268002ACC
:10FA800002D10122014B5A737047000070280020F8
:10FA900010B506F011F910BD002806D00649897985
:10FAA00001221143044A917105E00349897949080B
:10FAB0004900014A9171704700030440034880796E
:10FAC000400840000149887170470000200304404D
:10FAD00010B50224024805F0FFFF0446204610BD81
:10FAE000010600000348807902210843014988711A
:10FAF0007047000020030440002806D00649897999
:10FB000002221143044A917105E0034989790222D6
:10FB10009143014A91717047000304400348807982
:10FB20000221884301498871704700002003044086
:10FB300000B548220249034804F075FE00BD0000EC
:10FB4000501F0020441F002070B516480088401C3C
:10FB50001449088001F03CF8044613488079A0421B
:10FB600004D011498C71084604F00AFE0E4804F0D6
:10FB700051FEA04202DD0C4804F002FE002C0FD022
:10FB800001F048F905462946074804F060FE012CBB
:10FB900006DD01F086F905462946034804F057FEC4
:10FBA00070BD0000D0000020441F00202E480078C7
:10FBB000401C2D4908702D480078401C2B490870C6
:10FBC0002B480078401C2A4908702A480068401CCD
:10FBD0002849086008460068FF219131884202D90F
:10FBE00000202449086020480078C82802D9002055
:10FBF0001D4908701D480078842802D900201B493F
:10FC000008701B480078502802D900201849087055
:10FC1000194818490968405C184908701848124981
:10FC20000978405C17490870174810490978405C0A
:10FC30001649087016480E490978405C1549087045
:10FC4000154809490978405C144908701448064968
:10FC50000978405C13490870134803490978405CEF
:10FC600012490870704700008707002088070020AD
:10FC7000890700208C070020231F02008007002036
:10FC8000B3200200810700207B21020082070020B0
:10FC9000C722020084070020FF2102008307002002
:10FCA0001723020085070020DF23020086070020BB
:10FCB00010B58200054BD218525C012A04D10022F3
:10FCC0008300024C1B195A5410BD0000DC26002092
:10FCD00010B50446204600F055FA204600F002F820
:10FCE00010BD000010B50446B348007800287DD14F
:10FCF000B2480088B249884278DAB24800780028D1
:10FD00004FD0B1480078002803D0AC480088AF49F4
:10FD10000880AF480078002818D1A8480188AB486F
:10FD200000880A30814206D30120A9490870A348FF
:10FD30000088A6490880A1480088A449098888420B
:10FD40001CDA9E480088A149088017E09F48018876
:10FD50009A4800880A30814206D300209C490870E6
:10FD600096480088994908809448008897490988EE
:10FD7000884203DD914800889449088094480078BF
:10FD8000002858D193480078042803D08E48007882
:10FD9000002807D089480088822803DA05208D4989
:10FDA0000870A3E08B480078032803D086480078C9
:10FDB000002809D081480088FF211931884203DAE0
:10FDC00004208449087091E082480078022803D01A
:10FDD0007D48007800280AD078480088FF21AF319C
:10FDE000884204DA03207B4908707FE0E2E079482A
:10FDF0000078012803D074480078002809D06F48A3
:10FE00000088AF218900884203DA02207149087016
:10FE10006CE070480078002803D06B480078002818
:10FE200064D066480088E121890088425EDA0120BA
:10FE3000684908705AE066480078012856D165483C
:10FE40000078012803D060480078002809D05B487A
:10FE50000088E1218900884203DB00205D490870A9
:10FE600044E05C480078022803D057480078002816
:10FE700009D052480088AF218900884203DB012065
:10FE80005449087032E053480078032803D04E48A4
:10FE90000078002809D049480088FF21AF31884206
:10FEA00003DB02204B49087020E04A480078042810
:10FEB00003D045480078002809D040480088FF2139
:10FEC0001931884203DB0320424908700EE04148A3
:10FED0000078052803D03C480078002806D0374831
:10FEE0000088822802DB04203A490870FCF774FE7F
:10FEF0003349463988425DD337480068001936498E
:10FF0000086031480078002808D000202E49087089
:10FF1000314908602F4800783049087000F062FDD0
:10FF200000281FD12C4800682D49884239D3002071
:10FF3000294908602948007826490978884205DA65
:10FF400026480078401C254908702AE0234800789C
:10FF500020490978884224DD20480078401E1F4946
:10FF600008701EE01C4800681E49884219D3002012
:10FF7000194908601948007816490978884205DA55
:10FF800016480078401C154908700AE013480078AC
:10FF900010490978884204DD10480078401E0F4956
:10FFA00008700E4800780B490978884202D1002079
:10FFB0000949086010BD00000B000020020000206D
:10FFC0001C0C00001200002008000020040000208B
:10FFD0000A00002006000020180000200700002072
:10FFE000C05D0000407E050000200B4908700B49F1
:10FFF000087001200A4908700A49087000200A495F
:020000040001F9
:1000000008700A4908700A4908800A4908800A49A4
:1000100008800A4908707047060000200700002089
:1000200008000020090000200A0000200B0000202A
:100030000C0000200E000020100000201200002004
:1000400000200B4908700B49087001200A4908700C
:100050000A49087000200A4908700A4908700A49CC
:1000600008800A4908800A4908800A4908707047D0
:1000700006000020070000200800002009000020E2
:100080000A0000200B0000200C0000200E000020C1
:100090001000002012000020F8B5064600270024BA
:1000A00000250020009031480078002809D0032066
:1000B000F9F70AFA002804D00320F9F7F9F92C49D6
:1000C00008802C4800880A284AD300202949088043
:1000D00029480078282829D20320F9F7E9F90746AA
:1000E000002407E060002549085AB84200DD05E019
:1000F000601CC4B2204800788442F3DB00BF1E4875
:10010000057808E0681E40001C49085A69001B4A2F
:100110005052681EC5B2A542F4DC600017490F5268
:1001200015480078401C1449087019E00020009020
:100130000F2407E060001149095A00980818009040
:10014000601CC4B2192CF5D30A210098F7F7FEFF02
:1001500007490880002008490870012008490870F4
:1001600004480088801903490880F8BD0900002070
:1001700002000020160000200000002018080020C7
:1001800012000020394909881E2928DA0021384A3E
:100190001180384A118038490988384A914207DC71
:1001A00037490978002914D033490988914210DC75
:1001B0000121344A11700021334A1170334A117001
:1001C0002F4A11700121324A11700021314A1170F9
:1001D0004BE0294909880918274A118045E023493D
:1001E0000988264A643291422ADB0021224A118082
:1001F000204A11801E490988204A914207DC204983
:100200000978002916D01A490988914212DC022186
:100210001C4A117000211C4A117005211B4A1170E3
:100220000021174A11700121194A11700021194A41
:1002300011701AE00E49098809180D4A118014E05E
:1002400000210D4A11800A4A11800A4909880B4A87
:10025000914205DD00210B4A1170094A117004E03A
:10026000044909880918034A1180704702000020D8
:10027000100000200C0000200E000020B80B000031
:10028000090000200B0000200600002007000020CD
:10029000080000200A000020014800787047000094
:1002A000702000200148407A704700007020002034
:1002B00010B5642102480068F7F748FF80B210BD0E
:1002C000DC0000200148807870470000702000208A
:1002D000F8B50023002500950024002200BF94E01B
:1002E00001259D40ACB20D8825400095009DA5429A
:1002F0006FD11A468D79012D0DD1464D0326360258
:10030000AD192D5C012696403543424E03273F022E
:10031000F61935540CE03F4D03263602AD192D5C1D
:1003200001269640B5433B4E03273F02F61935544C
:10033000CD78002D4ED1374D60352D5CCE78002E16
:1003400001D1012600E000269640B543314E6036CB
:1003500035548D78002D2ED12E4D19267601AD19EC
:100360002D5C8E78002E01D1012600E000269640FB
:10037000B543284E19277F01F61935540D79002D04
:100380000ED1244D50352D5C0E79002E01D1012661
:1003900000E000269640B5431E4E5036355423E00B
:1003A0001C4D50352D5C0E7996403543EEB2194DFB
:1003B00050352E5418E0174D19267601AD192D5CD5
:1003C0008E7896403543134E19277F01F619355420
:1003D0000AE018E00F4D60352D5CCE78964035432D
:1003E000EEB20C4D60352E544D79012D0AD1094DD8
:1003F00030352D5C012696403543EEB2054D303543
:100400002E5400E000BF5D1CABB2082B00DA67E79A
:10041000F8BD000000000440FFB5074615461E4623
:1004200000243846019900F01FF8002802D001206E
:1004300004B0F0BD00240CE00A2060430949085CC8
:10044000B04204D12946204600F05EF807E0601C67
:1004500084B20A2060430349085C0028ECD100BF45
:100460000020E5E7DC0100200246002A03D14029F4
:1004700001DD01207047032A03D1022901DD01209B
:10048000F8E7042A03D1202901DD0120F2E7052A3B
:1004900003D1202901DD0120ECE70C2A03D110292A
:1004A00001DD0120E6E70D2A05D1012903DD402900
:1004B00001DA0120DEE70E2A03D1202901D1012033
:1004C000D8E70020D6E7000010B5064A03231B0238
:1004D000D218125C8A43034B032424021B191A54BA
:1004E00010BD00000000044010B5064A03231B02A3
:1004F000D218125C0A43034B032424021B191A541A
:1005000010BD00000000044070B502460020B1E0BC
:100510000A2353435A4C1B195B1C440004191B1932
:100520009B788B427DD10A235343554C1B195B1C8E
:10053000440004191B195B78082B33D10A23534359
:100540004F4C1B195B1C440004191B574D4C4E4D5E
:100550006419E35C012423430A245443484D64197D
:10056000641C450045196457464D474EAD192B553F
:100570000A235343424C1B195B1C440004191B57AC
:10058000404C35466419E35C022423430A24544357
:100590003B4D6419641C450045196457394DAD192C
:1005A0002B5564E00A235343354C1B195B1C440054
:1005B00004191B195B78092B34D10A235343304C9F
:1005C0001B195B1C440004191B572E4C2E4D64193B
:1005D000E35C402423430A245443294D6419641CDA
:1005E000450045196457274D274EAD192B550A2351
:1005F0005343234C1B195B1C440004191B57214C0B
:1006000035466419E35C8024A3430A2454431C4DFB
:100610006419641C4500451964571A4DAD192B55D2
:1006200025E025E00A235343154C1B195B1C4400AD
:1006300004191B57134C144D6419E35C0A245443EA
:100640000F4D6419641C450045196419657801242F
:10065000AC402343DCB20A235343094D5B195B1CB6
:10066000450045195B57074D074EAD19EC5404E0A2
:10067000431CD8B2032800DA4AE700BF70BD00006F
:10068000DC0100200000044075080000F8B50024DB
:10069000FCF7B4FA012861D100F064FB0446FF22A4
:1006A0000721002003F052F8012C21D100F040FC7A
:1006B00000280ED000F068FB054600F059FB064606
:1006C00001200346024629460090304605F06CFDA5
:1006D00050E000F059FB054600F04AFB06460120B9
:1006E0000023024629460090304605F05DFD41E0BA
:1006F000022C21D100F01CFC00280ED000F044FB9D
:10070000054600F035FB0646012003460246294611
:100710000090304605F048FD2CE000F035FB054622
:1007200000F026FB0646002001231A4629460090C9
:10073000304605F039FD1DE000F0FAFB054600F0FB
:1007400023FB064600F014FB0746012003462A4619
:1007500031460090384605F027FD0BE000200346A7
:1007600002460146009005F01FFD002207211046B9
:1007700002F0ECFFF8BD0000FEB50024FCF73EFAE5
:1007800001287DD15B480078012815D1FCF716F8C7
:1007900000BF0EE0182C0AD0152C08D00D2C06D066
:1007A0001A2C04D0FF222146002002F0CFFF601C4B
:1007B000C4B2242CEEDB9CE0FCF70EFA4E498842D2
:1007C0007ED34E480078032805DA4C480078401C58
:1007D0004A49087011E000204849087000F0CEFA3C
:1007E000064600F0E5FA07460A21F7F7AFFC054692
:1007F0003246294601200BF095FA00F007FD064627
:1008000000F090FC0A210290F7F7A0FC054600F0EA
:10081000B5FA07463246294609F012FAFFF736FFC5
:1008200000F08AFA05462946012007F04DFD00F048
:10083000B9FA0646FF21F531F7F79EFCC5B2294605
:10084000012006F06DFCFFF727FD0546FFF730FDA0
:100850000646FFF737FD07462B463246394601204C
:1008600005F07CFF00F0C4F80546294601200BF096
:10087000FFFC00F07DFC054600F072FB064600E040
:100880002AE000F07BFC074600F070FB00233A46AC
:10089000014600960195029001200AF05FFFFF22B9
:1008A0000321002002F052FFFF220421002002F069
:1008B0004DFF00F02BFC054600F022FC064600E050
:1008C00007E000F029FC07462A46314607F032FFD0
:1008D0000FE0FBF7EBFF0CE0FCF7C6F8002406E0A6
:1008E00000222146104602F031FF601CC4B2242CC5
:1008F000F6DBFEBD11010020D60B000072000020C7
:100900000149086070470000B407002002480068F1
:10091000401C014908607047B0070020F3B581B062
:10092000064600200E49086000F01EF8044600F05C
:100930001BF805462F1B3046029903F0ABFF0090D1
:100940000AE000F011F805462F1B06480068002851
:1009500002D004480068804700988742F1D3FEBD6A
:10096000B0070020B407002001480068704700006D
:10097000B00700200B490978012901D101200FE0BF
:1009800008490978022901D1022009E005490978BE
:10099000032901D1042003E00121024A1170012042
:1009A000704700004107002010B5094B1B8899B221
:1009B0000A12C8B2D3433133064C2370C3432333E6
:1009C000637013465633A37003467133E37010BD52
:1009D0007807002047070020014800887047000082
:1009E0001C000020014800887047000034000020EF
:1009F0000148007870470000A000002001480078FE
:100A000070470000A100002010B500220521064813
:100A1000FAF78CFB0402012205210348FAF786FB52
:100A2000201880B210BD00008408002010B50622F6
:100A300005210348FAF77AFBC006C00F10BD00007D
:100A40008408002010B5042205210648FAF76EFB41
:100A50000402052211460348FAF768FB201880B209
:100A600010BD00008408002010B5062205210248B0
:100A7000FAF75CFBC01110BD8408002010B50222FB
:100A800005210248FAF752FB10BD0000840800203F
:100A900010B5062205210348FAF748FB8006C00F6F
:100AA00010BD00008408002010B504220221034874
:100AB000FAF73CFBC007C00F10BD000084080020FF
:100AC00010B5052202210348FAF730FBC007C00F1A
:100AD00010BD00008408002010B500220421034846
:100AE000FAF724FB4006400F10BD000084080020E8
:100AF00010B5042201210248FAF718FB801110BD3D
:100B00008408002010B5002201210248FAF70EFBEC
:100B100010BD00008408002010B505220121034803
:100B2000FAF704FB8007800F10BD00008408002046
:100B300010B5012211460248FAF7F8FA10BD00007C
:100B40008408002010B5002206210C48FAF7EEFABE
:100B50000402012206210948FAF7E8FA20180402E3
:100B6000022206210548FAF7E1FA201804020322BE
:100B700006210248FAF7DAFA201810BD840800208E
:100B800010B5042206210C48FAF7D0FA0402052217
:100B900006210948FAF7CAFA20180402062211466B
:100BA0000548FAF7C3FA2018040207220621024872
:100BB000FAF7BCFA201810BD8408002010B50222F4
:100BC00003210248FAF7B2FA10BD000084080020A1
:100BD00010B5032200210248FAF7A8FA10BD000060
:100BE0008408002010B5002211460248FAF79EFA48
:100BF00010BD00008408002010B504220021024826
:100C0000FAF794FA10BD00008408002010B5012204
:100C100000210248FAF78AFA10BD0000840800207B
:100C200010B5052200210248FAF780FA10BD000035
:100C3000840800200146322915DA3E4880780128D0
:100C400003DD01203B4A507070E03A48807800286C
:100C500005DD2F296ADC0020364A507066E000204E
:100C6000344A507062E03E2917DA322915DB3148E8
:100C70008078022803DD02202E4A507056E02D486D
:100C80008078012805DD3B2950DC0120294A50707D
:100C90004CE00120274A507048E0502917DA3E29DD
:100CA00015DB24488078032803DD0320214A507097
:100CB0003CE020488078022805DD4D2936DC022002
:100CC0001C4A507032E002201A4A50702EE062290D
:100CD00017DA502915DB17488078042803DD042033
:100CE000144A507022E013488078032805DD5F29FC
:100CF0001CDC03200F4A507018E003200D4A50708E
:100D000014E073290FDA62290DDB0A488078042881
:100D100005DD70290ADC0420064A507006E0042034
:100D2000044A507002E00520024A507001484078A1
:100D300070470000702000200148007870470000D4
:100D40000700002000B50249024803F023FD00BD62
:100D5000D0000020441F00200148007870470000A8
:100D600005010020014800787047000004010020C0
:100D7000014800787047000009010020014800790F
:100D80007047000030220020014840787047000082
:100D900009010020014880797047000030220020BE
:100DA0000020704701480088704700001E000020A6
:100DB00010B50024FFF7E2FF00280AD10A48008896
:100DC0000A49884202DB0846074908800648048829
:100DD00008E005480088FCF7E7FC84B20448844238
:100DE00000DB0446204610BD36000020C607000088
:100DF000CE040000002005490988054A914202DB23
:100E00001146024A118001490888704736000020C7
:100E1000C6070000F8B50027002500260024FFF7CC
:100E2000E1FE0546FFF7F2FE0646F02028400011DD
:100E30000A2805DBF02028400011C01C044303E011
:100E4000F02028400011044324022807000F0A283C
:100E500004DB2807000FC01C044302E02807000F32
:100E600004432402F020304000110A2805DBF02062
:100E700030400011C01C044303E0F020304000115A
:100E8000044324023007000F0A2804DB3007000F58
:100E9000C01C044302E03007000F044327463846D5
:100EA000F8BDF8B50027002500260024FFF7A4FEB2
:100EB0000546FFF7B5FE0646F020284000110A2837
:100EC00005DBF02028400011C01C044303E0F020A3
:100ED00028400011044324022807000F0A2804DBDD
:100EE0002807000FC01C044302E02807000F04433A
:100EF0002402F020304000110A2805DBF0203040A9
:100F00000011C01C044303E0F020304000110443F2
:100F100024023007000F0A2804DB3007000FC01C32
:100F2000044302E03007000F044327463846F8BD6B
:100F300001480078704700008107002001480078D0
:100F400070470000830700200148C07B7047000005
:100F5000EC0900200148C07C70470000EC0900202B
:100F60000148007A70470000EC09002010B5002409
:100F70006421044800683230F7F7E8F884B220466C
:100F800010BD00009800002070B5002407480068DC
:100F9000FBF754FF05466421F7F7D8F884B20448FC
:100FA000844200DD0446204670BD00009C00002005
:100FB000DE03000010B5002400F014F8012800D171
:100FC0000CE000F00FF8022802D1FF24373405E0CE
:100FD0000A2103480088F7F7CFF884B2204610BDF5
:100FE0000200002001480078704700000B0000203C
:100FF000002005490968002903D0034909680868E9
:1010000000E00248704700009401002030750000A5
:1010100010B50024044804F05FFD002801D001242D
:1010200000E00024204610BD0407000010B5002495
:10103000044804F051FD002801D0012400E0002400
:10104000204610BD0507000010B50024044804F038
:1010500043FD002801D0012400E00024204610BDFB
:101060000707000010B50024062004F035FD002815
:1010700001D0012400E00024204610BD10B500245A
:10108000052004F029FD002801D0012400E00024FF
:10109000204610BD10B50024044804F01DFD0028B2
:1010A00001D0012400E00024204610BD0607000006
:1010B00010B50024044804F00FFD002801D00124DD
:1010C00000E00024204610BD0305000010B50024F8
:1010D000044804F001FD002801D0012400E00024B0
:1010E000204610BD040500000148807A70470000CA
:1010F000EC0900200148006870470000FC00002057
:101100000148807870470000280A002001484068A4
:1011100070470000280A002001484078704700000E
:10112000280A002070B50024FFF728FE002803D10C
:10113000FCF74EFD04460DE0FFF720FE012806D126
:10114000FCF746FD0546FCF72FFB044602E0FCF7E2
:101150003FFD0446204670BD0148007C70470000FA
:10116000EC0900200148007D70470000EC090020D8
:101170000148407A70470000EC09002010B50024B7
:101180006421044800683230F6F7E0FFC4B220461C
:1011900010BD00009800002070B5002407480068CA
:1011A000FBF74CFE05466421F6F7D0FF84B20448F5
:1011B000844200DD0446204670BD000098000020F7
:1011C000DE03000070B50BF05BFB0546002D01D17E
:1011D000012400E00024204670BD00000148007B8F
:1011E00070470000EC0900200148407B7047000078
:1011F000EC0900200148807B70470000EC090020CA
:1012000001480078704700000801002070B50024F4
:10121000FFF7B4FD002803D1FCF7FCFC04460FE007
:10122000FFF7ACFD012807D10020FCF7F3FC0546D1
:10123000FCF7BAFA044603E00020FCF7EBFC044696
:10124000204670BD01480078704700003E00002035
:1012500070B505460024032D00D170BD002D01D0CE
:10126000012D1BD181210320800204F0E5FB8021A8
:10127000134804F0E1FB32211248FFF74FFB002432
:1012800009E0A200104BD2189178A200985A04F0FD
:10129000D3FB601CC4B23B2CF3DB0FE0022D0DD15D
:1012A000002409E0A200094BD2189178A200985AB4
:1012B00004F0C2FB601CC4B23B2CF3DB00BFCCE7E4
:1012C00002060000A0860100401502002C16020054
:1012D000F8B5002100240023002200BF0AE0012508
:1012E0008D40ABB205881D402C469C4200D10A4679
:1012F0004D1CA9B21029F2DB0588FF2D1FDC284DFB
:101300006D7E0688B543264E757635462D7E068859
:10131000B543234E357635466D7E8678F607F60F53
:10132000964035431E4E757635462D7E86780227CB
:101330003E40760896403543194E357622E0184DEA
:10134000ED7E0688B543164EF5763546AD7E0688A9
:10135000B543134EB5768578ED07ED0F1646083E7A
:10136000B5400F4EF67E35430D4EF5768578022654
:1013700035406D081646083EB540094EB67E3543E9
:10138000074EB5760025009505E000BF6D462D7827
:101390006D1CEEB200966D462D78012DF5D9F8BD85
:1013A000206B0440C107C90F002905D00021394A2C
:1013B0001171002238490A7102210140002905D02B
:1013C0000021344A1172002233490A72042101407B
:1013D000002905D000212F4A117300222E490A73DB
:1013E00008210140002905D000212A4A1174002259
:1013F00029490A7410210140002905D00021254AFD
:101400001175002224490A7520210140002905D0C8
:101410000021204A117600221F490A76402101400E
:10142000002904D000221B494A711B494A718021BE
:101430000140002904D0002216494A7216494A7216
:10144000FF2101310140002904D0002211494A73D3
:1014500011494A73012149020140002904D00022A8
:101460000C494A740C494A7401218902014000293F
:1014700004D0002207494A7507494A750121C9026B
:101480000140002904D0002202494A7602494A76E6
:10149000704700000060004000610040C107C90FB4
:1014A000002905D001223C490A7100213B4A1171F3
:1014B00002210140002905D0012237490A7200218A
:1014C000364A117204210140002905D00122324917
:1014D0000A730021314A117308210140002905D007
:1014E00001222D490A7400212C4A11741021014057
:1014F000002905D0012228490A750021274A1175C3
:1015000020210140002905D0012223490A7600212B
:10151000224A117640210140002905D001221E49AE
:101520004A7100221D494A7180210140002905D0DD
:10153000012219494A72002218494A72FF210131D9
:101540000140002905D0012213494A7300221349A2
:101550004A73012149020140002905D001220E49A8
:101560004A7400220D494A74012189020140002970
:1015700005D0012208494A75002208494A7501210F
:10158000C9020140002905D0012203494A76002200
:1015900002494A7670470000006100400060004048
:1015A00010B50C480078002803D00B4A50689168A9
:1015B000884708484078002803D0084A5068916856
:1015C000884704488078002803D0054A506891680D
:1015D000884710BD006000402C030020AC040020B0
:1015E0002C06002010B508480079002803D0074ACF
:1015F00010695169884704484079002803D0044A9B
:1016000050689168884710BD006000402C0300209E
:10161000B804002010B50848007A002803D0074A13
:10162000D069116A88470448407A002803D0044AE8
:1016300050689168884710BD006000402C0300206E
:10164000C404002010B50848007B002803D0074AD6
:10165000906AD16A88470448407B002803D0044A36
:1016600050689168884710BD006000402C0300203E
:10167000D004002010B50848007C002803D0074A99
:10168000506B916B88470448407C002803D0044A83
:1016900050689168884710BD006000402C0300200E
:1016A000DC04002010B50848007D002803D0074A5C
:1016B000106C516C88470448407D002803D0044AD0
:1016C00050689168884710BD006000402C030020DE
:1016D000E804002010B50848007E002803D0074A1F
:1016E000D06C116D88470448407E002803D0044A1E
:1016F00050689168884710BD006000402C030020AE
:10170000F404002010B50848407F002803D0074AA1
:101710005068916888470448007F002803D0044A35
:10172000906DD16D884710BD00600040000500201D
:101730002C03002010B508484078002803D0074A41
:1017400050689168884704480078002803D0044A0C
:10175000506E916E884710BD206000400C0500203F
:101760002C03002010B509480079002803D0084A4E
:10177000106F516F88470548001D4078002803D03E
:10178000044A50689168884710BD000020600040FE
:101790002C0300201805002010B5034AD06F7832C2
:1017A0009168884710BD00002C03002010B5024A44
:1017B00050689168884710BDB003002010B50948F3
:1017C000007C002803D0084A506891688847054883
:1017D00010304078002803D0044A50689168884748
:1017E00010BD000020600040BC0300203C0500202C
:1017F00010B5024A50689168884710BDC8030020A0
:1018000010B5024A50689168884710BDD403002083
:1018100010B50948007F002803D0084A5068916835
:10182000884705481C304078002803D0044A506897
:101830009168884710BD000020600040E003002050
:101840006005002010B50C480078002803D00B4A32
:1018500050689168884708484078002803D0084AB3
:1018600050689168884704488078002803D0054A6A
:1018700050689168884710BD40600040EC0300202C
:101880006C050020EC06002010B50D4800790028FA
:1018900003D00C4A5068916888470948001D407879
:1018A000002803D0084A5068916888470448001D02
:1018B0008078002803D0054A50689168884710BD99
:1018C00040600040F803002078050020F806002062
:1018D00010B50D48007A002803D00C4A5068916872
:1018E0008847094808304078002803D0084A5068E3
:1018F00091688847044808308078002803D0054A5A
:1019000050689168884710BD406000400404002082
:10191000840500200407002010B50D48007B002836
:1019200003D00C4A50689168884709480C304078C9
:10193000002803D0084A50689168884704480C3052
:101940008078002803D0054A50689168884710BD08
:101950004060004010040020900500201007002087
:1019600010B50D48007C002803D00C4A50689168DF
:101970008847094810304078002803D0084A50684A
:1019800091688847044810308078002803D0054AC1
:1019900050689168884710BD406000401C040020DA
:1019A0009C0500201C07002010B5024A5068916871
:1019B000884710BD2804002010B50948007E002883
:1019C00003D0084A50689168884705481830407825
:1019D000002803D0044A50689168884710BD000071
:1019E0004060004034040020B405002010B50948D0
:1019F000007F002803D0084A50689168884705484E
:101A00001C304078002803D0044A50689168884709
:101A100010BD00004060004040040020C0050020D0
:101A200010B508480078002803D0074A506891682C
:101A3000884704484078002803D0044A50689168D9
:101A4000884710BD606000404C040020CC05002099
:101A500010B509480079002803D0084A50689168F9
:101A600088470548001D4078002803D0044A506884
:101A70009168884710BD0000606000405804002055
:101A8000D805002010B50948007A002803D0084A7C
:101A9000506891688847054808304078002803D08E
:101AA000044A50689168884710BD0000606000409B
:101AB00064040020E405002010B5024A50689168D3
:101AC000884710BD7004002010B5024A5068916824
:101AD000884710BD7C04002010B50948007D00280F
:101AE00003D0084A50689168884705481430407808
:101AF000002803D0044A50689168884710BD000050
:101B000060600040880400200806002010B50948E5
:101B1000007E002803D0084A50689168884705482D
:101B200018304078002803D0044A506891688847EC
:101B300010BD0000606000409404002014060020E6
:101B400010B50948007F002803D0084A5068916802
:101B5000884705481C304078002803D0044A506864
:101B60009168884710BD000060600040A00400201C
:101B70002006002010B5FE4800688079002806D0B5
:101B800001286ED002286DD003286CD104E2F848F9
:101B90000068407903000FF0B5F80A0614BC2BBCAE
:101BA00047BC67BC9BBC0BF0FFF80020F0490968FC
:101BB000C873EF4800684079401CED4909684871D6
:101BC000AEE0EC490969EA4A1268D27A885C0BF007
:101BD00063F9E74800684079401CE54909684871A5
:101BE000E34800684079401CE1490968487197E082
:101BF00001F014FF002810D10BF04EF9DC4800680A
:101C00004079401CDA4909684871D9480068407930
:101C1000401CD7490968487105E00BF0EFF8002037
:101C2000D349096848717BE001F0F8FE002811D122
:101C300001200BF031F9CE4800684079401CCC49B6
:101C400009684871CA4800684079401CC849096859
:101C5000487105E00BF0D2F80020C54909684871C9
:101C60005EE05FE0FEE0A3E101F0D8FE002828D1AD
:101C7000BF490968C97A24225143BF4A12688918AA
:101C8000BB4A1268D27B885C0BF006F9B848006842
:101C9000C07B401CB6490968C873B5480068C07B62
:101CA000242814D3B24800684079401CB049096820
:101CB0004871AF4800684079401CAD4909684871D7
:101CC00005E00BF09BF80020A9490968487127E05E
:101CD00001F0A4FE002815D1A5480068C07A401C78
:101CE000A3490968C872A2480068C07AA149097866
:101CF000884207DB00209E490968C87201209C4980
:101D0000096888710BF07AF80020994909684871D0
:101D100006E00BF073F8002095490968487100BF90
:101D200000BF4FE192480068407903000EF0EAFFDF
:101D3000080513912A91479170910BF035F8002016
:101D40008B490968C8738A4800684079401C8849F3
:101D50000968487184E087490969854A1268D27A1E
:101D6000885C0BF099F8824800684079401C8049F3
:101D7000096848717E4800684079401C7C490968C0
:101D800048716DE001F04AFE002811D126200BF0C9
:101D900083F8774800684079401C754909684871A4
:101DA000734800684079401C71490968487105E032
:101DB0000BF024F800206E490968487150E001F0EA
:101DC0002DFE00281DD101200BF066F86848006840
:101DD000C07B401C66490968C87365480068C07BC1
:101DE000242814D3624800684079401C604909687F
:101DF00048715F4800684079401C5D490968487136
:101E000005E00AF0FBFF002059490968487127E006
:101E100001F004FE002815D155480068C07A401C26
:101E200053490968C87252480068C07A5149097814
:101E3000884207DB00204E490968C87202204C49DD
:101E4000096888710AF0DAFF002049490968487179
:101E500006E00AF0D3FF002045490968487100BF39
:101E600000BFAFE042480068407903000EF04AFF2F
:101E70000805138B2A8B478B638B0AF095FF002094
:101E80003B490968C8733A4800684079401C3849A2
:101E9000096848717EE037490969354A1268D27A83
:101EA000885C0AF0F9FF324800684079401C3049EC
:101EB000096848712E4800684079401C2C4909681F
:101EC000487167E001F0AAFD002811D125200AF031
:101ED000E3FF274800684079401C2549096848719C
:101EE000234800684079401C21490968487105E091
:101EF0000AF084FF00201E49096848714AE001F099
:101F00008DFD002810D10AF0C7FF194800684079FC
:101F1000401C174909684871154800684079401C01
:101F200013490968487105E00AF068FF002010496C
:101F3000096848712EE001F071FD002815D10C48A8
:101F40000068C07A401C0A490968C87208480068DD
:101F5000C07A08490978884207DB002004490968EB
:101F6000C87203200249096888710AF047FF05E03A
:101F700004080020602B00200008002000201249E7
:101F80000968487106E00AF039FF00200E49096827
:101F9000487100BF00BF15E000200B490968887137
:101FA000094909684871062007490968C87009E0AD
:101FB0000AF024FF002004490968487102490968B1
:101FC000887100BF00BF10BD0408002010B56A482A
:101FD0000068407903000EF095FE090610C627C67A
:101FE00044C6608EC6000AF0DFFE63480068407990
:101FF000401C614909684871BCE0604909695E4A52
:102000001268D27A885C0AF047FF5B480068407922
:10201000401C594909684871574800684079401C7C
:10202000554909684871A5E001F0F8FC002811D174
:102030004F200AF031FF504800684079401C4E495B
:10204000096848714C4800684079401C4A49096851
:10205000487105E00AF0D2FE00204749096848713E
:1020600088E001F0DBFC002810D10AF015FF42489F
:1020700000684079401C4049096848713E48006842
:102080004079401C3C490968487105E00AF0B6FEF9
:1020900000203949096848716CE001F0BFFC002854
:1020A00022D135480068C07A401C33490968C8729B
:1020B00031480068C07A3149097888420FDB002036
:1020C0002D490968C8722C4800684079401C2A498B
:1020D00009684871002028490968486208E0002022
:1020E00025490968487103E00020234909684871BF
:1020F0000AF084FE3EE020480068407C002816D0AC
:102100001E48C068002803D01C48C16819208847B1
:102110000020194909684862174909684871164939
:1021200009688871052014490968C8701AE01248C6
:102130000068406A282807D20F480068406A401C9F
:102140000D49096848620DE000200B4909684862A2
:1021500009490968487108490968887105200649D4
:102160000968C87006E00AF049FE002002490968C3
:10217000487100BF00BF10BD04080020602B002084
:1021800010B50024F7480068807A01287ED1F54810
:102190000068C07900287AD0F24800688079002869
:1021A00004D0012874D0022873D191E1ED48006871
:1021B000007B24286ED2EB480068C07901287AD1D0
:1021C000002475E0E7480068C07A24214843E649C6
:1021D00009684018E3490968097B415CE1480068E7
:1021E000C07A24225043E14A12688018DD4A1268FE
:1021F000127B805C814229D0DA480068C07A2421B1
:102200004843DA4909684018D6490968097B415CA6
:10221000D4480068C07A24225043D34A12688018F8
:10222000D04A1268127B8154CE480068407B242833
:1022300005D3CC480068007BCA4909684873C9487F
:102240000068007BC7490968887308E0C5480068D2
:10225000407B242803D20120C24909688871C14803
:102260000068007B401CBF4909680873BD480068CE
:10227000007B242808D3BB480068407B242803D275
:102280000120B84909688871B64805E0D3E1CDE17D
:1022900069E0BAE138E00EE00068007B242804D24F
:1022A000B04800688079012800D103E0601CC4B206
:1022B000242C87D356E0002413E0AA480068C07A93
:1022C00024214843A94909684018015DA5480068D0
:1022D000C07A24225043A44A126880180155601C19
:1022E000C4B2242CE9D300209E49096848732320F6
:1022F0009C490968887301209A49096888712420DB
:102300009849096808732DE0002096490968087308
:1023100094480068C07A401C92490968C872914884
:102320000068C07A92490978884217DB8D480068B6
:10233000007C012804D102208A490968887106E0DE
:10234000002088490968887186490968C871002099
:1023500084490968C8728349096808740020814962
:102360000968487161E17F480068407903000EF018
:10237000C9FC080513A62AA651A68EA601207949F4
:10238000096808740AF010FD764800684079401C1E
:1023900074490968487199E075490969714A126878
:1023A000D27A885C0AF078FD6E4800684079401C5B
:1023B0006C49096848716B4800684079401C69495C
:1023C0000968487182E001F029FB00281BD16549AA
:1023D0000968497B491CC8B20AF05EFD6148006883
:1023E000407B60490968C8735E4800684079401CBA
:1023F0005C49096848715B4800684079401C59494C
:102400000968487105E00AF0F9FC0020554909689F
:1024100048715BE001F002FB00282BD151490968AB
:10242000C97A24225143504A126889184D4A1268C9
:10243000D27B885C0AF030FD4A480068C07B401CB3
:1024400048490968C87347480068C07B454909681E
:10245000897B88421ADD434800684079401C414925
:10246000096848713F4800684079401C3D49096847
:1024700048710BE00AF0C2FC3A480068407B3949D9
:102480000968C87300203749096848711EE001F0E7
:10249000C5FA00280CD133490968887124203149D4
:1024A0000968C8732F49096848732E4909688873F9
:1024B0000AF0A4FC00202B490968487106E00AF0E4
:1024C0009DFC002027490968487100BF00BFACE0AF
:1024D00024480068407903000EF014FC08050F8EB4
:1024E000268E4C8E688E0AF05FFC1E48006840798C
:1024F000401C1C490968487185E01D490969194A51
:102500001268D27A885C0AF0C7FC164800684079E5
:10251000401C144909684871124800684079401C01
:102520001049096848716EE001F078FA002811D16D
:1025300025200AF0B1FC0B4800684079401C09498D
:1025400009684871074800684079401C05490968D6
:10255000487105E00AF052FC002002490968487100
:1025600051E000000408002000080020FC070020C3
:10257000602B002001F052FA002810D10AF08CFCE8
:10258000644800684079401C6249096848716148A4
:1025900000684079401C5F490968487105E00AF00D
:1025A0002DFC00205B49096848712CE001F036FAE7
:1025B00000281AD157480068C07A401C554909685C
:1025C000C87254480068C07A5349097888420CDBC5
:1025D000002050490968C8724E49096888714D4900
:1025E000096848714B490968C8710AF007FC002066
:1025F00048490968487106E00AF000FC0020454996
:102600000968487100BF00BF0FE00AF0F7FB002027
:102610004049096848713F49096888713D4909681E
:1026200008733C490968C87200BF71E0002039494D
:10263000096888726CE037480068807A022867D1A0
:1026400034480068007A00285ED03248006840793B
:10265000002804D001280CD0032846D11BE00AF042
:10266000A3FB2C4800684079401C2A49096848713E
:1026700049E000200AF010FC264800684079401C20
:10268000244909684871234800684079401C214961
:102690000968487137E00AF051FB002812D11D4843
:1026A00000684078401C1B49096848701948006858
:1026B0004078032812D301F055FA00201549096823
:1026C00048700BE00020134909680872AA201149DC
:1026D0000968887000200F49096848700AF08EFB6D
:1026E00000200C49096848710DE00AF087FB0020C2
:1026F000084909684871074909684870AA200549CE
:102700000968887000BF03E00020024909688872E8
:1027100010BD000004080020602B0020F8B504461E
:102720000D4600260C2060431D49085C002801D09E
:102730000120F8BD0C2060431949401885600C2029
:10274000604340188068002801D10120F1E7012191
:102750000C206043124A115400222046E317DB0E7E
:102760001B185B115B01E31A9B000E4FDB19E71787
:10277000FF0E3F197F11DA550EF0F6FA00222046BF
:10278000E317DB0E1B185B115B01E31A9F00064B7E
:10279000FB18E717FF0E3F197F11DA553046C8E7DF
:1027A0002C030020006000400061004000BFFEE7F5
:1027B00010B51B480088401C19490880084600884D
:1027C000184988422BDD18480078002827D0084691
:1027D000134908801448007801280CD11348007868
:1027E000012808D1002012498870084602F042FFF3
:1027F00000200E4908700C48007802280CD10D48C2
:102800000078012808D1002009498870084602F0A4
:1028100031FF00200749087000200349087010BDEF
:1028200000010020DC05000004010020060100205A
:102830000901002007010020704700000020014925
:102840000880704700010020F0B505460E46174687
:1028500000243A463146284600F05EFE00BF42E0C2
:1028600000202101394A126850522101374A12686A
:102870008918488000212001344A1268801881801C
:102880002001324A12688018C18020012F4A126844
:102890008018017220012D4A1268801841722001AF
:1028A0002A4A1268801881722001284A126880180A
:1028B000C17200202101254A12688918087300217D
:1028C0002001224A126880184173002021011F4A0A
:1028D000126889188873002120011C4A1268801828
:1028E000C173601CC4B21A484078A042B8DC6420AE
:1028F0001849096808807D20C00016490968488089
:1029000015481449096888807D200001114909682B
:10291000C88010490968088110480E490968488133
:102920000F480C490968888140000A490968C88134
:102930003220084909680882FF20F53005490968F6
:102940004882044909688882F0BD0000C40700205D
:10295000B8070020C00700204C040000102700002A
:102960003075000038B5002404E0002013490855F4
:10297000601C84B2282CF8D3012168464170017094
:102980006A460F490D48FFF75FFF7D21C9003220DD
:1029900000F0B2F90B490C4800F0CCF9094864305A
:1029A00000F05EF90748C83000F06AF9074800F007
:1029B0007DF9074800F090F938BD00003C22002066
:1029C000141B020028230000B80B00005424000050
:1029D0001027000010B524480078002803D10120FA
:1029E000214908703EE020480078012810D11F4896
:1029F0000078012808D100201D498870084602F09F
:102A000039FE00201949087002201749087029E092
:102A100015480078022810D116480078012808D1FE
:102A2000002013498870084602F024FE0020114956
:102A3000087003200C49087014E00B480078032844
:102A400003D10520084908700CE0074800780528E4
:102A500003D005480078062804D1002002490870F8
:102A60000549087010BD0000040100200601002087
:102A7000090100200701002008010020F8B500240A
:102A8000002500263548007800281ED134480078FB
:102A9000002803D101203249087016E03048007840
:102AA000012803D102202E4908700EE02C4800783E
:102AB000022803D103202A49087006E0284800783C
:102AC000032802D1002026490870244800780128F4
:102AD0000ED101241725002622480123324629461B
:102AE0000090204601F038FF01201F49087034E0B3
:102AF0001A48007802280FD101243B2500261948E6
:102B0000401C0123324629460090204601F024FF54
:102B100001201649087020E01048007803280DD1E4
:102B2000FEF72CF9002803D101201149087102E0B9
:102B300000200F4908710EF0B7F80EE00748007842
:102B4000052803D106200549087006E003480078EF
:102B5000062802D1052001490870F8BD04010020B3
:102B600005010020090100200601002007010020C6
:102B70003022002010B5044623000EF0C3F809618E
:102B800006101C1D1E1F5F606400FAF725F82F4910
:102B9000884201D3FFF772FFFFF750FE54E0FAF7C7
:102BA0001BF82A49884203D3FFF714FF0BF034FEC9
:102BB000FFF744FE48E047E046E045E0FAF70CF84E
:102BC0002249884237D301F073FE21480078032858
:102BD00014D120480078002810D1FEF7DBF8002837
:102BE00006D101201C4988718879FBF77DF805E042
:102BF0000020194988718879FBF776F81448007825
:102C0000012805D113480078002801D1FAF76EF9A0
:102C100010480078052803D10120104908700AE007
:102C20000C480078062803D102200C49087002E005
:102C300000200A490870FFF701FE05E004E003E008
:102C4000FFF7B6FD00E000BF00BF10BDD60B0000CF
:102C5000050100200401002030220020080100208E
:102C600001460020054A126852898A4201DC01208F
:102C700002E0024A1268118170470000C00700207C
:102C800001460020084A126812898A4201DB0120AD
:102C900009E0054A126892898A4201DC012002E0BB
:102CA000014A126851817047C00700200146002088
:102CB000084A126852898A4201DB012009E0054A6C
:102CC0001268D2898A4201DC012002E0014A1268BE
:102CD00091817047C007002001460020054A126814
:102CE00092898A4201DB012002E0024A1268D18106
:102CF00070470000C0070020024600200C4B1B68F4
:102D00001B8A934201DD012010E08A4201DB012091
:102D10000CE0074B1B689B888B4201DC012005E01F
:102D2000034B1B681A80024B1B68598070470000D8
:102D3000C0070020024600200C4B1B681B8A9342F0
:102D400001DD012010E08A4201DB01200CE0074B8D
:102D50001B685B88934201DB012005E0034B1B6885
:102D60009A80024B1B68D98070470000C007002082
:102D700070B5044600250C206043FE4909684018E0
:102D80004068002807D00C216143FA4A126889186C
:102D90004868804705460C206043F6490968085C8E
:102DA000002873D10C206043F249096840188068FC
:102DB000002874D02001F04909684018C07A022820
:102DC0000AD1032D08D10C206043EA4A126880180A
:102DD00081680120884762E02001E74909684018BE
:102DE000C07A02280AD1042D08D10C206043E14AA0
:102DF0001268801881680220884750E02001DE496F
:102E000009684018C07A02280AD1052D08D10C2083
:102E10006043D84A126880188168032088473EE0E2
:102E20002001D54909684018C07A02280AD1062D28
:102E300008D10C206043CF4A1268801881680420B2
:102E400088472CE02001CC4909684018C07A022844
:102E50000AD1072D08D10C206043C64A1268801899
:102E60008168052088471AE02001C3490968401895
:102E7000C07A02280BD1082D09D10C206043BD4A2D
:102E80001268801881680620884708E00DE00C2051
:102E90006043B84A12688018816800208847200182
:102EA000B54909684018C5720CE30C206043B1496C
:102EB0000968085C012873D10C206043AD4909689A
:102EC00040188068002874D02001AB490968401878
:102ED000C07A03280AD1022D08D10C206043A54AEC
:102EE0001268801881680120884762E02001A249A9
:102EF00009684018C07A04280AD1022D08D10C2094
:102F000060439C4A1268801881680220884750E01C
:102F10002001994909684018C07A05280AD1022D74
:102F200008D10C206043934A1268801881680320FE
:102F300088473EE02001904909684018C07A062879
:102F40000AD1022D08D10C2060438A4A12688018E9
:102F50008168042088472CE02001874909684018CF
:102F6000C07A07280AD1022D08D10C206043814A7B
:102F7000126880188168052088471AE020017E4980
:102F800009684018C07A08280BD1022D09D10C20FD
:102F90006043784A1268801881680620884708E0F4
:102FA0000DE00C206043734A12688018816800208D
:102FB00088472001704909684018C57282E20C20D8
:102FC00060436C490968085C0228F7D1002D7DD167
:102FD000200169490968085A68490968098A8842CC
:102FE00075DA200164490968085A0A3081B2200163
:102FF000614A1268115220015F490968085A5F4905
:103000000968098A884231DB20015B490968401858
:1030100040885A4909680988884227DB20015649B7
:1030200009684018408855490968498888421DDC6C
:1030300000202101504A12688918488020014E4919
:1030400009684018807A0028B8D10C2060434949AB
:103050000968401880680028B0D00C206043454AB9
:10306000126880188168012088472BE220014249BC
:103070000968085A41490968098A88429EDB20018B
:103080003D490968401840883C4909688988884258
:1030900094DB20013849096840184088374909689D
:1030A000C98888428ADC00202101334A12688918C5
:1030B00048802001304909684018807A0028D4D11E
:1030C0000C2060432B490968401801E063E00BE0E5
:1030D00080680028C9D00C206043264A12688018F6
:1030E000816802208847EDE100202101224A126810
:1030F000891848802101204A12688918C872002165
:1031000020011D4A12688018C18020011A4A1268E5
:10311000801841722001184A12688018817218487C
:1031200001782001144A12688018017200202101E0
:10313000114A12688918888021010F4A126889187B
:10314000087321010C4A12688918487321010A4A40
:1031500012688918887300212001074A12688018B4
:10316000C1730C2060430349096840188068002837
:10317000B9D007E0BC070020C4070020C00700202A
:10318000B80700200C206043CF4A1268801881687D
:103190000020884796E1012DA5D12001CB4909687F
:1031A0004018C07AA84225D000212001C74A1268E1
:1031B0008018418000202101C44A12688918C88003
:1031C0002001C24909684018C572C1480078210130
:1031D000BE4A12688918487200202101BB4A126851
:1031E00089188880BA4801782001B84A1268801886
:1031F000017267E12001B54909684018007AB449B5
:103200000978884220D0B24800782101AF4A12687C
:10321000891808722001AD4909684018407AAC4904
:103220000978884209D02001A84909684018808897
:103230002101A64A12688918C88000212001A34AEA
:1032400012688018818012E02001A04909684018A6
:103250008088A04988420AD220019C490968401808
:1032600080880A302101994A1268891888802001D3
:103270009649096840184088964988420AD2200138
:1032800092490968401840880A3021018F4A126823
:103290008918488020018D4909684018407A8C4976
:1032A0000978884205D001202101884A12688918CE
:1032B0008872200185490968401840888649096854
:1032C0000988884204DB00212001804A12681152DB
:1032D00020017E4909684018807A00287ED10C20A0
:1032E00060437949096840188068002877D0200138
:1032F00076490968401840887749096809898842F1
:1033000014DB2001714909684018007B00280DD1A9
:103310000C2060436C4A126880188168032088473B
:1033200001202101694A1268891808732001674940
:10333000096840184088684909684989884214DB4F
:103340002001624909684018407B00280DD10C20FB
:1033500060435D4A12688018816804208847012014
:1033600021015A4A1268891848732001574909688F
:1033700040184088584909688989884214DB20012F
:10338000524909684018807B00280DD10C20604309
:103390004D4A126880188168052088470120210164
:1033A0004A4A1268891888732001484909684018F8
:1033B000408849490968C989884210DB200143498E
:1033C00009684018C07B00287CD10C2060433E4A2D
:1033D0001268801881680620884701E007E03BE01A
:1033E00001202101394A12688918C8736AE0200156
:1033F000364909684018407A01282ED134480078AF
:1034000002282AD12001314909684018C088324970
:103410000968498A884255DB20012C49096840180F
:1034200080882D490968898A88424BDB0C206043DB
:103430002549096840188068002843D00C20604363
:10344000214A1268801881680720884700202101DE
:103450001E4A12688918487234E020011B49096825
:103460004018407A02282DD119480078012829D126
:103470002001164909684018C08817490968898AD7
:1034800088421FDB200111490968401880881249D1
:103490000968498A884215DB0C2060430A4909689B
:1034A0004018806800280DD00C206043064A12683E
:1034B000801881680820884700202101034A12688B
:1034C0008918487270BD0000BC070020C4070020A6
:1034D000B8070020F0FF0000C007002010B500244E
:1034E00000BF04E02046FFF743FC601CC4B2024862
:1034F0004078A042F6DC10BDB807002010B50024CB
:10350000044802F0E9FA002800D000E00124204637
:1035100010BD00000304000010B5074B14781C70A8
:1035200054785C70054B1960054B186003461833DE
:10353000044C236010BD0000B8070020BC07002029
:10354000C0070020C407002010B50446012C09D193
:10355000FF220C21002000F0F9F80121022005F0E3
:1035600023F808E000220C21104600F0EFF80021BB
:10357000022005F019F810BD10B5002404210848F8
:10358000F7F7E6FD552801D1012407E0042001F0FA
:1035900077F8002801D0002400E00124204610BD67
:1035A0008408002010B50446012C09D1FF221C21FB
:1035B000002000F0CBF80121062004F0F5FF08E020
:1035C00000221C21104600F0C1F80021062004F062
:1035D000EBFF10BD10B50024062001F051F80028C3
:1035E00001D0012400E00024204610BD10B504469F
:1035F000012C09D1FF221721002000F0A7F801219A
:10360000042004F0D1FF08E000221721104600F04A
:103610009DF80021042004F0C7FF10BD00200449DC
:10362000097A002901D0012000E000207047000045
:10363000280A002010B50446022C1CD100220D21BE
:10364000104600F083F8FDF773FC002809D0FF2234
:103650000B21002000F07AF801210D2004F0A4FFD6
:1036600058E000220B21104600F070F800210D20D8
:1036700004F09AFF4EE0032C1CD100220B211046CF
:1036800000F064F8FDF754FC002809D0FF220D215A
:10369000002000F05BF801210D2004F085FF39E0E7
:1036A00000220D21104600F051F800210D2004F0F9
:1036B0007BFF2FE0042C0ED1FF220D21002000F013
:1036C00045F800220B21104600F040F801210D20A2
:1036D00004F06AFF1EE0012C0ED100220D211046DD
:1036E00000F034F8FF220B21002000F02FF8012118
:1036F0000D2004F059FF0DE000220D21104600F0CE
:1037000025F800220B21104600F020F800210D20A2
:1037100004F04AFF10BD000010B500240A480078EC
:10372000012801D101240CE0FCF7BCFD012801D1E6
:10373000032406E0FCF7B6FD022801D1022400E0D4
:103740000424204610BD00001101002010B5064BD6
:103750001B78834207DD242905D224234343034CED
:1037600024681B195A5410BD602B0020FC07002050
:1037700010B574480068407903000DF0C3FA0B07D8
:1037800011D325D35A6D77D38DA8D30009F00CFB44
:103790006C4800684079401C6A4909684871CFE06C
:1037A00069494969087809F077FB664800684079FB
:1037B000401C644909684871624800684079401CAF
:1037C000604909684871BBE000F028F9002811D170
:1037D0007F2009F061FB5B4800684079401C594933
:1037E00009684871574800684079401C5549096884
:1037F00048711DE0534800684078401C51490968F1
:10380000487050480068407803280BD300204D4989
:1038100009684870AA204B49096888700320494903
:103820000968C87009F0EAFA002046490968487139
:1038300086E000F0F3F8002807D14248006840799C
:10384000401C40490968487103E000203D4909686F
:10385000487109F0D3FA73E009F0A6FA3948006814
:103860004079401C37490968487169E0364949691F
:103870000978491CC8B209F00FFB3248006840794A
:10388000401C3049096848712E4800684079401C46
:103890002C490968487153E000F0C0F800280FD1A6
:1038A00009F054FA274909688870012009F0C8FA1C
:1038B000244800684079401C22490968487105E0A5
:1038C00009F09CFA00201F490968487138E01D483A
:1038D0000068807818280CD102201A4909680870FD
:1038E0000020184909684870042016490968C87002
:1038F00011E0144800684078401C1249096848707B
:10390000104800684078032805D300F02BF9002008
:103910000C490968487009F071FA002009490968E2
:1039200048710DE009F06AFA0020064909684871FB
:10393000044909684870AA2002490968887000BFD4
:1039400000BF10BD04080020602B002010B53148D6
:1039500000684079002804D001280CD0032848D101
:103960001DE009F021FA2B4800684079401C2949E4
:10397000096848714BE028490969087809F08CFA10
:10398000244800684079401C224909684871214850
:1039900000684079401C1F490968487137E000F011
:1039A0003DF800280CD101201A4909680870002050
:1039B000184909684870042016490968C87011E060
:1039C000144800684078401C124909684870114842
:1039D00000684078032805D300F0C4F800200D49A2
:1039E0000968487009F00AFA00200A490968487114
:1039F0000DE009F003FA00200649096848710549FD
:103A000009684870AA2003490968887000BF00BF90
:103A100010BD000004080020602B002010B509F044
:103A20008DF904461F4800680078002838D01D48EA
:103A30000068C078042833D3002C09D1002119482C
:103A40000068C07A8200174800681430815027E06F
:103A500014480068C07A8100124800681430405849
:103A60001149884211D20F480068C07A81000D4880
:103A7000006814304058401C0A490968C97A8A0015
:103A800008490968143188500AE000F06BF80021F9
:103A900004480068C07A82000248006814308150EF
:103AA000204610BD04080020B80B000000B587B008
:103AB0000120694608710A4802900A4803900A48A2
:103AC00004900A4805900A48069070210948F4F7C6
:103AD000EDFB01A9074800F00FF807B000BD00009A
:103AE0001D3E0100B95C0100850E0200811B020031
:103AF000801B0200A4220020F8B506460F460024D1
:103B000000253946304600F0EFF900BF14E00025EB
:103B10000EE00021242060430B4A126880184155B2
:103B200024206043094A126880184155681CC5B2B8
:103B3000242DEED3601CC4B205480078A042E6DC18
:103B400000F010F8F8BD0000FC070020000800207D
:103B5000602B0020012002490968087170470000AD
:103B60000408002010B500F073F90020034909682B
:103B7000087002490968C87010BD000004080020E0
:103B800007480068C078062808D105480068C07951
:103B9000002803D1012002490968C871704700005C
:103BA0000408002010B555480068C07803000DF0E7
:103BB000A9F808671D1A1714110E056650484068C9
:103BC000002803D04E4841680020884793E000F069
:103BD000E5F890E000F0C6F88DE000F0D1F88AE05A
:103BE000FFF7B4FE87E0FFF7C3FD84E04448406878
:103BF000002803D042484168012088473F480068B8
:103C0000407C00281AD03E48C068002803D03C48B9
:103C1000C168C82088470020384909684862374889
:103C200000680078002804D0042034490968C8706E
:103C300024E0022031490968C8701FE02F4800685D
:103C4000406A401C2D49096848622C480068406A57
:103C50007D21C900884211D30020284909684862A3
:103C6000264800680078002804D004202349096809
:103C7000C87003E0022021490968C8703BE000BF1A
:103C80001F484068002803D01D484168002088472D
:103C90001A480068407C002813D01948C0680028E2
:103CA00003D01748C168C820884700201349096815
:103CB000486212480068C078401C10490968C87002
:103CC00018E00E480068406A401C0C4909684862C8
:103CD0000A480068406A7D21C90088420AD3002052
:103CE00006490968486205480068C078401C0349D5
:103CF0000968C87000BF00BF10BD000004080020A4
:103D0000602B002010B515480068C078072824D023
:103D1000012012490968487408E0114880680028A9
:103D200002D00F4988688047FFF73CFF0B480068C6
:103D3000C0780628F1D109480068007A0028ECD143
:103D400006480068C0790028E7D104480068807AF6
:103D50000028E2D101490968487410BD0408002018
:103D6000602B002010B5054800680078012802D1BA
:103D7000FDF700FF01E0F5F771FC10BD040800201D
:103D800010B5054800680078012802D1FEF71EF939
:103D900001E0F6F741F810BD0408002010B51D48F9
:103DA0000068807A002829D11A480068007A002823
:103DB00003D0022017490968887216480068C07944
:103DC000002803D00120134909688872114800684F
:103DD0000079012812D100200E49096808710D49A7
:103DE0000968887207200B490968C8700A4840684A
:103DF000002803D00848416800208847054800682B
:103E00000078012802D1FEF7BBF901E0F6F7DEF8F1
:103E100010BD000004080020602B002010B50446EF
:103E20002146084801F074FE07480078002805D1B3
:103E3000002C03D032210548FCF770FD02480470C5
:103E400010BD0000010300001201002050C300005B
:103E50000020244909684870AA202249096888700E
:103E600000202049096848621E49096808711D49F7
:103E7000096848711B49096888711A490968C8713D
:103E8000184909680872174909688872154909684C
:103E9000C8721449096808732420124909684873D4
:103EA0001049096888730F490968C87300200D49D3
:103EB000096808740B49096848740A4909688874D4
:103EC00008490968C874074909684861002105481C
:103ED0000068816103480068C161024800680162AE
:103EE000704700000408002010B50A780D4B1860D8
:103EF000034628330C4C23602423534304462834C0
:103F00001B190A4C23600A4C4B6863608B68A360E2
:103F1000CB68E3604B6963610B6923610B782370A5
:103F200010BD000004080020FC070020000800204D
:103F3000602B002007480068C078062808D1054893
:103F40000068007A002803D101200249096808723C
:103F5000704700000408002010B50446012C09D168
:103F6000FF2220210020FFF7F1FB0121084604F089
:103F70001BFB08E0002220211046FFF7E7FB002191
:103F8000012004F011FB10BD10B50024032000F047
:103F900077FB002801D0012400E00024204610BD5A
:103FA00010B50446032C0ED1FF2215210020FFF787
:103FB000CDFB002214211046FFF7C8FB01210E2083
:103FC00004F0F2FA39E0022C1CD1FCF7B1FF002812
:103FD00009D0FF2214210020FFF7B8FB01210E2099
:103FE00004F0E2FA08E0002214211046FFF7AEFBCD
:103FF00000210E2004F0D8FA002215211046FFF708
:10400000A5FB1AE0012C0ED1FF2214210020FFF79E
:104010009DFB01210E2004F0C7FA00221521104655
:10402000FFF794FB09E0002215211046FFF78EFBF5
:10403000002214211046FFF789FB10BD10B50024A3
:10404000F8F7CAFD094988420DD3FCF7CBFF0028D9
:1040500007D1FCF771FE012801DD032404E00224EE
:1040600002E0022400E00124204610BDD60B00002F
:1040700010B50446012C09D1FF221D210020FFF7B5
:1040800065FB0121002004F08FFA08E000221D21C9
:104090001046FFF75BFB0021084604F085FA10BDCF
:1040A00010B50024022000F0EBFA002801D0012412
:1040B00000E00024204610BD10B50446012C09D1B3
:1040C000FF221E210020FFF741FB0121092004F0FF
:1040D0006BFA08E000221E211046FFF737FB002193
:1040E000092004F061FA10BD70B5002400250026F7
:1040F000FCF7DAFC0546FCF7E3FC0646022108481B
:10410000F7F726F8552800D108E0012E01D1002448
:1041100004E0012D01D1012400E00024204670BDFF
:104120008408002010B50446012C09D1FF221F216C
:104130000020FFF70BFB0121082004F035FA08E00E
:1041400000221F211046FFF701FB0021082004F088
:104150002BFA10BD70B500240025FCF72FFD054695
:1041600003211A48F6F7F4FF552806D10120184913
:10417000088000201749088023E01648008801289D
:1041800011D114490880FCF733FC762803DA0120AA
:104190000F49088015E0FCF72BFC782811DB002084
:1041A0000B4908800DE001200A490880FCF720FC3B
:1041B000762803DA01200649088002E0002004493D
:1041C000088003480488204670BD00008408002051
:1041D000300100203201002010B50446012C09D125
:1041E000FF2221210020FFF7B1FA0121072004F06E
:1041F000DBF908E0002221211046FFF7A7FA002191
:10420000072004F0D1F910BD10B50024FCF7DAFF47
:10421000012801D1012400E00024204610BD10B582
:104220000446012C09D1FF2216210020FFF78EFA47
:104230000121032004F0B8F908E0002216211046FD
:10424000FFF784FA0021032004F0AEF910BD10B589
:104250000024052000F014FA002801D0012400E019
:104260000024204610BD10B50446012C09D1FF22C0
:1042700019210020FFF76AFA0121052004F094F9C2
:104280003CE0022C17D1FCF753FE002809D0FF2296
:1042900019210020FFF75AFA0121052004F084F9C2
:1042A0002CE0002219211046FFF750FA00210520CA
:1042B00004F07AF922E0032C17D1FCF73FFE002826
:1042C00009D0FF2219210020FFF740FA0121052023
:1042D00004F06AF912E0002219211046FFF736FABD
:1042E0000021052004F060F908E0002219211046A1
:1042F000FFF72CFA0021052004F056F910BD00004C
:1043000010B50024FCF746FD012839D104214048AE
:10431000F6F71EFF552803D101203E49087032E010
:10432000FCF7DAFB01280BD0FCF7D6FB022807D0FC
:10433000FCF7D2FB032803D0FCF7CEFB052803D102
:104340000120344908701EE0FCF7C6FB042803D1A5
:1043500002203049087016E0FCF7BEFB062803D1A6
:1043600003202C4908700EE0FCF7B6FB002803D0B0
:10437000FCF7B2FB072806D100202649087002E0AE
:1043800000202449087024480078022813D12348CB
:104390000078002807D1FCF7CBFD002803D01D488A
:1043A00000781D490870FCF7C3FD1C490870FCF734
:1043B000BFFD044616E018480078032812D11748BC
:1043C0000078002807D1FCF7B9FD002803D0114878
:1043D000007811490870FCF7B1FD10490870FCF72E
:1043E000ADFD04460C48007802280ED00A4800783B
:1043F00003280AD007480078074908700846007863
:10440000002801D0012400E00024204610BD000057
:1044100084080020340100203501002036010020EE
:1044200010B50446012C0ED1FF221B210020FFF7FE
:104430008DF900221A211046FFF788F901210A2080
:1044400004F0B2F81EE0022C0ED1FF221A21002047
:10445000FFF77CF900221B211046FFF777F90121B5
:104460000A2004F0A1F80DE000221A211046FFF7FF
:104470006DF900221B211046FFF768F900210A2080
:1044800004F092F810BD000010B500241048007828
:10449000012801D1012418E0FCF756FD022803D0C1
:1044A000FCF75AFE02280FD1FCF71EFE012809D1A5
:1044B000FCF750FD012803D0FCF754FE012801D180
:1044C000012402E0022400E00224204610BD000086
:1044D0001101002010B5F8F791FB0446204610BDED
:1044E00010B540210448F3F7E1FE044B08220449CB
:1044F000014800F013F910BD64220020D5440100EA
:10450000201B020070B506465C488068002804D075
:104510005A4988688047054600E000250024A6E047
:10452000564841680C20604308184088A84207D0CC
:10453000524841680C2060430818408802287DD109
:104540004E4841680C2060430818806800280CD051
:104550004A494A680C216143511888688047474995
:104560000968E2008918487009E0444841680C2055
:104570006043095C41480068E200801841703F4890
:104580000068E100401840783C490968E200895C15
:1045900088420FD039480068E10040184178374818
:1045A0000068E2008154002034490968E20089185B
:1045B00048605AE031480068E100401841782F48CF
:1045C00042680C2060431018407881421FD12B486C
:1045D0000068E10040184168284842680C206043A8
:1045E0001018808881420BD824480068E1004018E8
:1045F0004068801921490968E2008918486034E060
:1046000001201E490968E200891848802DE01B48F6
:104610000068E10040184168184842680C20604377
:104620001018C08881420DD814480068E100401875
:104630004068811911480068E20000E009E0801834
:10464000416012E000200D490968E20089184880A5
:104650000BE0002009490968E20089184880002120
:1046600006480068E20080184160601C84B203487C
:104670008089A04200DD53E770BD0000182B0020A8
:104680000146064A92898A4205DD044A1268CB0037
:10469000D218508800E0002070470000182B00203E
:1046A000002000BF14E00D494A680C214143511815
:1046B000498801290AD10021084A1268C300D2188A
:1046C0005180064A1268C300D2185160411C88B25A
:1046D000024989898142E6DC70470000182B0020DE
:1046E000002000BF13E00C494A680C2141435118D7
:1046F0004988002909D1084A1268C300D21851809C
:10470000054A1268C300D2185160411C88B20249A0
:1047100089898142E7DC7047182B0020F0B50446F8
:104720000020164DAB6069602C60AA8100BF1FE0BD
:10473000124D6E680C254543755D104E3668C700F6
:10474000F61975700D4D6E680C254543755D0B4E61
:104750003668C700F5550025084E3668C700F619BB
:104760007580064E3668C700F6197560451CA8B2FC
:10477000024DAD898542DBDCF0BD0000182B002026
:104780000146002901D102207047002008714871BC
:1047900000BFF9E710B503460C46002B01D0002CF2
:1047A00001D1002010BD184600F034F8002800D1D7
:1047B000F8E72088FF21F53188420ADB00202080BD
:1047C000187A401CC0B218725979884201DB1879F6
:1047D0001872197A890018684058E3E710B5034643
:1047E0000C46002B01D1022010BD184600F012F833
:1047F000002800D1F8E7197907E08A001868805886
:10480000A04201D10120EFE7491C58798842F4DC2D
:104810000020E9E70146002900D1704748790A796C
:10482000801AC0B2F9E70346002B01D0002901D15C
:1048300002207047012A01DA0120FAE71960DA71D3
:104840000020187198715871187200BFF1E730B5E7
:1048500004460D46002C01D1032030BD002D01D1AE
:104860000420FAE76079401CE179884201DB0120ED
:10487000F3E729462046FFF7B1FF002801D00220C8
:10488000EBE761798900206845506079401C6071D0
:104890000020E2E770B505460E46002E05D03146F1
:1048A0002846F3F753FC044600E02C46204670BD32
:1048B00010B5FCF787FC012817D10C4800780128B7
:1048C00013D00A48007803280FD009480078002840
:1048D0000BD1FCF78DFB0749884202D108F03FF964
:1048E00003E07D20000108F041F910BD0501002022
:1048F000040100208813000008B500200090012268
:104900006946FF202130F4F7D5F96846007805495B
:10491000887100200449087004490870044908702F
:1049200008BD000030220020040100200601002004
:104930000701002008B50020009001226946FF20F1
:104940002130F4F7B7F90020024908716846007871
:10495000887108BD3022002070B5049C25789142F2
:1049600016DD01280AD18D4206DAFF26F61AAE427C
:104970000ED3EE18F5B20BE0154609E0022807D178
:10498000954204DD9D4203DBEE1AF5B200E00D46D0
:10499000257070BD00BF00BF00BF00BF00BF00BFDB
:1049A00000BF00BF00BF00BF00BF00BF00BF00BF0F
:1049B00000BF00BF00BF00BF00BF00BF00BF00BFFF
:1049C00000BF00BF00BF00BF00BF00BF00BF00BFEF
:1049D00000BF00BF00BF00BF00BF00BF00BF00BFDF
:1049E00000BF00BF00BF00BF00BF00BF00BF7047D7
:1049F0000D4A4168516081699161C168D160416A25
:104A00005162016A116201681160416951618168F6
:104A10009160C169D16101691161816A916200216E
:104A2000024A117070470000342B0020F807002064
:104A300010B5FFF735FEF7F723FFF8F7E5F810BDDF
:104A400010B5F6F7CFFCF7F71BFFFFF749FE0AF0AA
:104A500039F90AF0D5F9FBF7C7FAFAF7FFF8FFF7CB
:104A60004BFFF8F74DFCF6F789FAF9F749F95521AC
:104A70000448F6F7F1FCF8F779F9F9F7BBF8FBF71A
:104A800057F810BD900800201CB5F6F7BBFC0020BD
:104A900033490870FCF7DCFB08F036F90CF0C0FA7B
:104AA000F7F76EF8F9F764F9F6F7B2FCF8F75EF984
:104AB000F9F7A0F8F5F7DCFDF6F7C8F8E1204002B9
:104AC0000CF08AF800F0E6FAF6F758FA08F01CFB4A
:104AD000F7F7D6FEF9F708FFF8F7A2FCF8F71CFC89
:104AE000FFF7FEFCFDF73EFFFEF7E0FFFFF70AF9D8
:104AF000F9F70AFEFBF7A4FAFAF7B0F8194A1A49CF
:104B000001200AF043FA0022114601200AF082F93E
:104B100008F066F80AF0BCF80AF072F9FFF70AFF2D
:104B2000002012498871487108710120887048700E
:104B30001420087007226846F3F79FFB019900983C
:104B400001F036F80221012000F00EFFFAF7F0FF25
:104B5000F8F712F8012006490870064908701CBDD4
:104B6000110100200090D003EC040000240100207B
:104B700082000020830000207047000010B504462A
:104B8000552C03D105494869804702E0034908686C
:104B9000804700200249087010BD0000342B00201F
:104BA000F807002010B54648007803000CF0AAF87A
:104BB0000A06111B26303B4650517381414840681C
:104BC000002802D03F494868804701203C490870CE
:104BD00000BF3C488068002804D03A498868804774
:104BE0003749087069E03748C068002802D0354965
:104BF000C868804703203249087000BF3148006907
:104C0000002804D02F49086980472D49087054E0D6
:104C10002C484069002802D02A4948698047002072
:104C20002749087049E027488069002802D02549B3
:104C30008869804706202249087000BF2148C06962
:104C4000002804D01F49C86980471D49087034E016
:104C500000BF1B48007807280AD11A48006A0028BC
:104C600002D01849086A804709201549087011E0E8
:104C70001348007808280AD11248406A002802D058
:104C80001049486A804709200D49087002E0002059
:104C90000B49087000BF0A480078002808D009486E
:104CA000806A002804D00749886A80470449087050
:104CB00003E000200249087000BF00BF10BD0000E3
:104CC000F8070020342B00207047000010B50020AA
:104CD0000CF050FA09F0F2F809F046F909F05CF925
:104CE00000F036FDF6F752F80220FCF7B1FA00208A
:104CF00006490870FFF706F8FEF72CFFFEF752FF93
:104D0000F5F722FE10200AF057FD10BDC801002063
:104D100010B50124F7F772FF012801D1052407E03F
:104D2000F7F754FF0349884201D2012400E002242E
:104D3000204610BD8813000010B5062408F08CFC36
:104D4000002800D1002408F08DFC012803D008F0D1
:104D500089FC072800D90924204610BD10B5002081
:104D6000544908700AE00022524801781046FEF7C4
:104D7000EDFC50480078401C4E4908704D480078C2
:104D80002428F0DB00204C49087009E000214A4843
:104D9000007809F085FD48480078401C46490870B5
:104DA000454800780D28F1DBFEF7EAFEFEF7AAFF82
:104DB000F5F7ECFF0022114601200AF05DF9002111
:104DC0003E48F6F749FB00203D490880002400BF1B
:104DD00000F072FF32217D200001FBF79FFD0020D3
:104DE000344908700AE00022324801781046FEF784
:104DF000ADFC30480078401C2E4908702D480078E2
:104E00002428F0DB00202C49087009E000212A4802
:104E1000007809F045FD28480078401C26490870B4
:104E2000254800780D28F1DBFEF7BCFEF5F762FCA3
:104E300008F064FB23480078401C224908700846AB
:104E40000078052812D300200870FEF799FE1E484E
:104E500000780A2805D300201B490870FFF76AF87C
:104E600004E019480078401C1749087008F0FAFB64
:104E70000128ADD908F0F6FB0728A9D200200E4979
:104E8000087008E00C48007809F024FD0A48007812
:104E9000401C09490870084800780D28F2DBF5F736
:104EA000D5FE55210548F6F7D7FAF7F765FE2046F7
:104EB00010BD00002D0100202B01002090080020D3
:104EC000800000202C0100202E01002010B50324BA
:104ED0000BE000F0F1FE012000F0FEFD002802D101
:104EE00000F036FD01E0042400E0F2E700BF2046B8
:104EF00010BD000010B500202D4908702D49086034
:104F00000120FCF7A5F907F0FFFEF6F739FEF7F7E9
:104F10002DFFF8F76FFE0CF083F8F5F7A9FBF9F712
:104F2000ABFCF5F793FE08F0F9FAF8F7E9FEF6F7AF
:104F300059FAF6F76DFAF9F7D7FCF9F773FEF8F7B7
:104F40006FFAFFF7CDFAFDF70DFDFFF7C9FBFFF78D
:104F5000D3FCFEF7ABFDFEF7D5FE00F09BF8E12099
:104F600040020BF039FEF6F709F8FBF769F8F9F79C
:104F700075FE114A114901200AF008F80022114675
:104F8000012009F047FF09F083FE09F039FF0221F3
:104F9000012000F0E9FCFAF7CBFD07F043FEF7F73C
:104FA000EBFD0120064908700649087010BD00009D
:104FB0007C0000204C0000200090D003EC04000096
:104FC000820000208300002010B50720400200F07E
:104FD00083FD012812D114480068C82808D3002096
:104FE0001249086000210720400200F091FD19E0FD
:104FF0000D480068401C0C49086013E00B4800682D
:10500000022805D809480068401C0849086009E0E2
:105010000020064908600449086001210720400279
:1050200000F076FD10BD0000C8000020CC0000207C
:1050300070B506460D4614460E4806600E480560DB
:105040000E49206808600E49606808600D49A06834
:1050500008600D49206908600C49E06808600C4947
:105060006069086005480068002802D003480068AD
:10507000804770BDBC000020C4000020A4000020B8
:10508000A8000020AC000020B0000020B4000020E8
:10509000B800002000B587B00C4801900C48029081
:1050A0000C4803900020049005900B4806900020C7
:1050B0000A49086048600A490860486001AA01215D
:1050C000C9020848FFF7B4FF07B000BDE95001006E
:1050D000955401001D540100415301003C12002071
:1050E000340A00204417002001207047F3B5C3B0F4
:1050F0000446449E0020009057E002E0641C761EA7
:1051000000BF022E05D32078EB28F7D160789028D5
:10511000F4D1072E00D24AE0A778FD1CB54200D991
:1051200045E0A81E205C0002691E615C08434290B5
:10513000042D38D9291FA01C0BF09EFF42998842EC
:1051400026D11D480068002804D0B91EE01C1A4A68
:105150001268904719480068002824D0E178684612
:105160000171207981116846417120798106890E8B
:1051700068468171381FC1B26846C171C279611D2C
:1051800002A8F3F77AF801A80C49096888470AE0F1
:105190000020009002E00098401C00900098A84277
:1051A000F9D3002000906419761B072EA5D200BF0A
:1051B0004498801B45B0F0BDB0000020B80000202E
:1051C000F7B5C0B0154600260027E81DFF210131C4
:1051D000884202DD002043B0F0BDEB21684601703B
:1051E00090214170281DC1B2684681700021C170B4
:1051F0004098C1B2684601710524002605E0419837
:10520000805D69460855641C761CAE42F7DBA11E22
:1052100000A802300BF030FF0746381269460855E7
:10522000641C0F55641C06480068002805D0214600
:105230006846034A12689047CDE70020CBE700009C
:10524000A800002070B50024002500261B484068F7
:105250001A490968884200D170BD1848406817494A
:105260000968884205D91548406814490968451AF3
:1052700007E01248006811494968401A0121890273
:105280000D1AFF2D01D9FF2600E02E4600240DE067
:105290000A4801680830405C0949085507480088F9
:1052A000401C8005800D05490860641CB442EFD3A2
:1052B000314603480BF0ECFC00BFCDE73C12002068
:1052C0004416002070B500251A480068002830D028
:1052D000194A1288FF230133991A184A1268164B8B
:1052E0001B88D018134A126890470546002D20D01D
:1052F00011480088401910490880084601880F4865
:105300000068FFF7F3FE0446002C0DDD0A48008814
:10531000844209DA08480088021B0848006801191D
:1053200006480068F2F7A9FF03480088001B0249FD
:10533000088070BDAC000020C0000020BC00002030
:1053400038B504460020009030490860A078102845
:105350000CD120792E49087008460078012853D1D5
:10536000002211462020FFF72BFF4DE0A0781228E5
:1053700003D120792649087246E0A078052803D198
:105380002079234988723FE0A07802281DD1207936
:105390001F4948720846407A012806D10090012230
:1053A00069460420FFF70CFF2EE01948407A0228D6
:1053B0002AD100BFBFF34F8F16481749C860BFF30B
:1053C0004F8F00BF00BF00BFFDE7A07801281BD1B1
:1053D0002079332803D101200D49487005E0207958
:1053E000352802D100200A49487060790849887040
:1053F000607A0006217A09040843E179090208432A
:10540000A17908430249486038BD0000C800002067
:10541000280A00200400FA0500ED00E070B50346FC
:105420000022002400251A484068194E3668B04210
:1054300001D1002070BD16484068154E3668B04254
:1054400005D913484068124E3668841B07E010489F
:1054500000680F4E7668801B0126F602341AA142BE
:1054600001D9254600E00D4600220CE008480668F8
:105470000830805D985406480088401C4005400D67
:10548000034E3060521CAA42F0D32846D2E70000F7
:10549000340A002070B503460022002415484068F5
:1054A000144D2D68A84208D312484068114D2D684C
:1054B000401B0125AD022C1A04E00E4800680D4D7A
:1054C0006D68441BA14201D9012070BD00220CE08F
:1054D0009D5C084846680830855508388088401C1F
:1054E0008005800D034D6860521C8A42F0D3002075
:1054F000EBE700003C12002010B50248FFF778FAF5
:1055000010BD0000081C02000021014A11757047FF
:1055100040600040014600BFF020084000110A230F
:10552000584302460807000F8018C0B27047014672
:10553000002204E0501CC2B208460A38C1B20A294F
:10554000F8DA1007000E08437047000010B5044653
:1055500001218020F6F714F8607A012805D142482D
:10556000C078102108434049C870607AA22805D14C
:105570003E48007F802108433C490877607A3B49D8
:10558000087700203A4948770846407F2178084349
:1055900037494877E07B002805D00846407F202126
:1055A0000843334948773248407FC008C000A17A99
:1055B00008432F4948770846807FF72108402C4947
:1055C0008877E078FFF7B3FF29498874A078FFF760
:1055D000AEFF2749C8746078FFF7A9FF2449087512
:1055E0002078002805D10846007D2179084320490C
:1055F0000875E079FFF79BFF1D4988756079FFF713
:1056000096FF1B494875A079FFF791FF1849C875A7
:10561000207AFFF78CFF164908760846807F4006FF
:10562000400E8877E07A002806D00846807F402127
:1056300008430F49887703E00D48807F0C4988773D
:10564000A07BFFF774FF0A498876607BFFF76FFF46
:105650000749C876207B08770846807F1021884359
:105660000349887710BD0000200402406004044014
:10567000404F044010B504461B48807F0121084379
:10568000194988772078FFF752FF17490875607825
:10569000FFF74DFF1449C874A078FFF748FF12497F
:1056A000887420780C2806DD0846407F08210843CE
:1056B0000D49487709E00C48407F0B494877084678
:1056C000007DE1780843084908750748807F400855
:1056D00040000549887700BF0348807F02210840C9
:1056E0000028F9D110BD0000404F044010B5002043
:1056F0001449087616200BF02BFB00211248017686
:105700001248407F80210843104948770846807F2F
:10571000012108430D49887700BF0C48807F022192
:1057200008400028F9D00948807F40084000074918
:10573000887700BF0548807F022108400028F9D102
:1057400010BD00004060004040610040404F0440F8
:1057500010B500200749087000212020F5F710FF40
:1057600001210548017500200449087515200BF03A
:10577000D7FA10BD00500440406100404060004036
:1057800070B504460D46002C14D0002D12D0042D07
:1057900010D800F013F800280CD1002608E00649C4
:1057A000885D22460121F3F793FDA41C701CC6B24C
:1057B000AE42F4DB70BD0000841B020000200549EE
:1057C000897DC907C90F002901D0012000E0002010
:1057D000704700000050044030B585B005460C46C7
:1057E000002003900490009001900290072C0BDCA5
:1057F0000120A04081B2684681810121C17303A9C3
:105800000220FAF765FD3EE0082C01D0092C0BD1EF
:105810000120A04081B2684681810121C17303A9A2
:105820000120FAF755FD2EE00A2C03D00B2C01D0F5
:105830000D2C0BD10120A04081B26846818101214D
:10584000C17303A90020FAF743FD1CE00C2C01D022
:105850000F2C0BD10120A04081B26846818101212B
:10586000C17303A90E20FAF733FD0CE00E2C0AD108
:105870000120A04081B2684681810121C17303A942
:105880000C20FAF725FD002168460170C1704170B7
:105890000121817000210171C1720D218172FF21EE
:1058A000017200214172F3F777FD03491520FCF7DF
:1058B00035FF05B030BD00000955010010B50020CE
:1058C0001049087515200BF02BFA00210E480175C0
:1058D0001520002809DB00BF00BFC206D20E01213F
:1058E00091400A4A116000BF00BF00BF084880799C
:1058F0008011032805D00648007880210843044918
:10590000087010BD406000404061004000E100E0D0
:105910000050044010B5F3F739FE10BD10B5012357
:105920001A4600211846F5F7DFFD01221146104600
:10593000F5F746FEF2F7C6FB03480BF063FB02489F
:105940000249086010BD00000090D0037C070020D1
:1059500000BF04480069042108430249086130BFC0
:1059600000BF704700ED00E0F3B585B005460024A8
:1059700000270026002003900490EEB22804070EB2
:105980000F2F54DA082E52DA002009E00C2141438F
:10599000284A515AA94201D1044603E0411CC8B229
:1059A0001728F3D300BF0120B04086B20C2060431B
:1059B00020494018C3780C20604340188278F8B220
:1059C00031460190FAF728FD6846868101218173EE
:1059D0000021C17302214174F8B203A9FAF778FCDF
:1059E0000C216143134A8918C888FBF757FD0C2026
:1059F000604310494018C18868460181694606988D
:105A0000887202A8FBF764FC0C226243094BD2188F
:105A100091680C226243D21804201056FCF77EFED7
:105A20000C216143034A8918C888FBF7BBFC07B007
:105A3000F0BD0000A01D0200FEB505460C4600208A
:105A4000C0430290EFB22804060E0F2E42DA082F50
:105A500040DA0120B84069460880802020400028B4
:105A600016D101208870A007800F022801D148714B
:105A700009E0A007800F012802D16946487102E0C1
:105A8000002069464871F0B26946FAF721FC1FE030
:105A90000020694688700E202040002800D000BFFA
:105AA00010202040002802D16946087102E0012040
:105AB00069460871E007C00F002802D16946887165
:105AC00002E0012069468871F0B26946FAF700FCED
:105AD000002002900298FEBD30B50146CAB20C0407
:105AE000230E00200F2B0FDA082A0DDA0124944030
:105AF000A2B2064C03252D026419E45C1440002C6C
:105B000001D0012000E0002030BD00000000044072
:105B1000F8B504460F460020C0430090E6B22004CA
:105B2000050E0F2D11DA082E0FDA0120B04086B2D3
:105B3000002F04D1E8B23146FAF7C6FC03E0E8B220
:105B40003146FAF7D1FC002000900098F8BD000023
:105B50001649897F01221143144A917700BF1349E6
:105B6000897F022211400029F9D01049897C817077
:105B70000E49C97C41700D49097D01700B498A7D30
:105B80008271497D01710949CA7D42710A7EC271E3
:105B9000897F49084900054A917700BF0349897FF9
:105BA000022211400029F9D170470000404F044003
:105BB00003B585B00020019002900390049000216D
:105BC00068464173817E01A8C1706846417E01A884
:105BD00081706846017E4171002101A80171082190
:105BE00068460171817D01A8C1716846C17D41721D
:105BF000417D01A881716846017D01A801720021E3
:105C000068468173C17301A881730C2141734121DE
:105C1000684601740021C17401A8FFF797FC1820A1
:105C20000249888200F004F807B000BD204F04400C
:105C300010B5FFF75BFD10BD70B504460D46601E44
:105C40000D49884200D90124002C00D101244020B4
:105C50000A490870084600786043094948610321F1
:105C6000081F0BF08DF800200549886107200861A6
:105C70000448056070BD0000FFFFFF00A401002084
:105C800000E000E0A00100200020C043002809DB64
:105C9000C206D20E01219140054A1160BFF34F8F19
:105CA000BFF36F8F00BF0020024908618861704711
:105CB00080E100E000E000E010B50BF007F810BD57
:105CC0001A20084908722B2048723C2088724D2007
:105CD000C8727F20044909680860AC2003494870F5
:105CE0007047000000040240A8010020001002409C
:105CF00010B504460F488088002800D110BD0D481B
:105D00000088182250430B4A083281181822204676
:105D1000F2F7B3FA07490988481C1721F2F72CFA61
:105D200088B20449088008468088401E8880012087
:105D3000E4E700006C24002010B51C48007801281E
:105D400012D11B480078642809DB022019494871E8
:105D500008710020164908701449087004E01448BE
:105D60000078401C124908701348007801281CD1A3
:105D700012480078012804D1002010490870104909
:105D800008700F48007832280ADBF7F737F800214F
:105D90000C48F5F7A7FA55210B48F5F75DFB04E031
:105DA00007480078401C0649087010BD45070020D0
:105DB00044070020340700203E0700204007002051
:105DC0003F0700208408002090080020F8B5044612
:105DD0000D46002700200090032000032040001300
:105DE0000090102C04D0122C02D01148844217D1FC
:105DF00022202840222806D127073F0F3946009845
:105E0000F4F722FC06461220284012280ED1200763
:105E1000000F471C39460098F4F716FC064605E0CB
:105E20002107090F0098F4F70FFC06463046F8BD2D
:105E300010100000F8B504460D460026002701208A
:105E4000000320400713102C04D0122C02D00F485E
:105E5000844215D122202840222805D12607360F5A
:105E600031463846F9F724FF1220284012280CD179
:105E70002007000F461C31463846F9F719FF04E0A9
:105E80002107090F3846F9F713FFF8BD101000007D
:105E9000FFB587B01C460020059043480390029050
:105EA000424801900998002802D101980BB0F0BD3A
:105EB000102107980840002801D0022707E0402160
:105EC00007980840002801D0012700E00027002C97
:105ED00001D0FF2C02D11020069003E0109804702E
:105EE00001200690002551E0002C01D0FF2C07D1A5
:105EF00068002F4A115A0898F2F728F9059007E030
:105F0000254660002A4A115A0898F2F71FF90590B1
:105F1000059949086422514308460999F2F716F990
:105F200006B23846642148433230B0422CDA214868
:105F3000864229DA30463230F2F71EF9C1B20491B6
:105F4000642204995143891B0091002901DB0099C7
:105F500001E000994942184A084650433146F2F799
:105F60000BF980B2029003990298884208DA1098DF
:105F700005700498401EC1B21098417002980390B9
:105F80000398002800D191E7681CC5B206988542A5
:105F9000AADB0398F2F7F3F904490090F2F7B1F99C
:105FA0000190019882E70000FFFF00000000C84256
:105FB000B41E0200CE310000102700000246412A24
:105FC0002ED010DC212A2AD006DC102A45D0122A35
:105FD0004BD0202A59D11CE0222A26D0232A2AD0AD
:105FE000402A52D116E081235B01D01A9A4228D070
:105FF00008DC422A1AD0432A1ED02548101800284F
:1060000043D13AE0012822D020281BD021283CD1BE
:106010001EE000BF1F4803890B43038136E000BF29
:106020001C4843890B43438130E000BF19488389F2
:106030000B4383812AE000BF1648C3890B43C38109
:1060400024E000BF144883880B4383801EE000BF18
:106050001148C3880B43C38018E00E4843890B43A3
:10606000438103890B43038110E00A48C3890B4332
:10607000C38183890B43838108E00748C3880B43AE
:10608000C38083880B43838000E000BF00BF70475C
:10609000F0EFFFFF0011044000140440F0B5054686
:1060A0000E46412D30D010DC212D2CD006DC102DD9
:1060B00051D0122D56D0202D62D11CE0222D2AD095
:1060C000232D30D0402D5BD116E081214901681A83
:1060D0008D4230D008DC422D1ED0432D24D02A48DA
:1060E000281800284CD144E001282CD0202823D0A7
:1060F000212845D128E000BF244F3888314600F0E0
:1061000049F804463DE000BF204F7888314600F052
:1061100041F8044635E000BF1C4FB888314600F016
:1061200039F804462DE000BF184FF888314600F0DA
:1061300031F8044625E000BF154F3888314600F09D
:1061400029F804461DE000BF114F7888314600F061
:1061500021F8044615E00D4F7888314600F01AF812
:1061600004460EE0094FF888314600F013F8044663
:1061700007E0074F7888314600F00CF8044600E04D
:1061800000BF00BF2046F0BDF0EFFFFF001104404C
:10619000001404400246002013460B40002B01D09F
:1061A000012000E000207047FFB581B00E46174681
:1061B000012F07D1F748407D00090001C01DF549B6
:1061C000487505E0F348407D00090001F149487534
:1061D000049801287ED10A210198F1F7B7FF0546FE
:1061E000ED48445DE007C00F002807D0E948007C77
:1061F00000090001C01DE749087405E0E548007C7E
:1062000000090001E349087402202040002807D05B
:10621000E048C07BF02188437030DE49C87305E058
:10622000DC48C07BF0218843DA49C8730420204051
:10623000002807D0D748807C00090001C01DD5493F
:10624000887405E0D348807C00090001D149887436
:1062500008202040002807D0CE48407CF021884309
:106260007030CC49487405E0CA48407CF02188432E
:10627000C849487410202040002807D0C548407CF9
:1062800000090001C01DC349487405E0C148407CB5
:1062900000090001BF49487420202040002807D091
:1062A000BC48007CF02188437030BA49087405E08E
:1062B000B848007CF0218843B6490874402020404B
:1062C000002808D0B348807CF02188437030B14961
:1062D000887406E08BE0AF48807CF0218843AD49AC
:1062E00088740A210198F1F731FF0D46AA48445DF0
:1062F000E007C00F002807D0A648807BF021884324
:106300007030A449887305E0A248807BF02188435F
:10631000A049887302202040002807D09D48807B38
:1063200000090001C01D9B49887305E09948807BE6
:10633000000900019749887304202040002807D0F5
:106340009448007DF021884370309249087505E03B
:106350009048007DF02188438E4908750820204030
:10636000002807D08B48007D00090001C01D894925
:10637000087505E08748007D00090001854908751A
:1063800010202040002807D08248C07CF02188439C
:1063900070308049C87405E07E48C07CF021884395
:1063A0007C49C87420202040002807D07948C07B51
:1063B00000090001C01D7749C87305E07548C07B1E
:1063C000000900017349C87340202040002807D00D
:1063D0007048C07C00090001C01D6E49C87454E0BB
:1063E0006C48C07C000900016A49C8744DE06948E6
:1063F000007C00090001674908740846C07BF02151
:1064000088436449C8730846807C00090001887489
:106410000846407CF02188435E4948740846407C29
:106420000009000148740846007CF021884359495E
:1064300008740846807CF0218843564988740846D1
:10644000807BF0218843534988730846807B00098C
:10645000000188730846007DF02188434D49087586
:106460000846007D0009000108750846C07CF0213F
:1064700088434849C8740846C07B00090001C873B6
:106480000846C07C00090001C8740A9801287DD123
:106490000A213046F1F75AFE05463F48445DE007C1
:1064A000C00F002807D03B48407B00090001C01DF9
:1064B0003849487305E03748407B000900013549F9
:1064C000487302202040002807D03248007BF0218A
:1064D000884370302F49087305E02E48007BF02177
:1064E00088432C49087304202040002807D02948FD
:1064F000807DF021884370302649887505E0254865
:10650000807DF02188432349887508202040002899
:1065100007D02048807D00090001C01D1D498875F5
:1065200005E01C48807D000900011A49887510208B
:106530002040002807D01748407DF0218843703064
:106540001449487505E01348407DF02188431149FE
:10655000487520202040002807D00E48407BF021BD
:10656000884370300B49487305E00A48407BF021AE
:106570008843084948734020204000280ED0054831
:10658000C07D00090001C01D024900E092E0C8750D
:106590000AE000007C200020D81802006D48C07D71
:1065A000000900016B49C8750A213046F1F7CEFD9C
:1065B0000D466948445DE007C00F002807D06548D4
:1065C000C07AF021884370306249C87205E06148A2
:1065D000C07AF02188435F49C87202202040002819
:1065E00007D05C48C07A00090001C01D5949C87233
:1065F00005E05848C07A000900015649C8720420D5
:106600002040002807D05348407E00090001C01DEB
:106610005049487605E04F48407E000900014D4949
:10662000487608202040002807D04A48007EF02104
:10663000884370304749087605E04648007EF021DF
:1066400088434449087610202040002807D041485C
:10665000007E00090001C01D3E49087605E03D4866
:10666000007E000900013B490876202020400028D8
:1066700007D03848007B00090001C01D3549087368
:1066800005E03448007B00090001324908734020CE
:106690002040002807D02F48C07DF021884370306B
:1066A0002C49C87554E02B48C07DF0218843294906
:1066B000C8754DE02748407B000900012549487313
:1066C0000846007BF0218843224908730846807DF4
:1066D000F02188431F4988750846807D0009000124
:1066E00088750846407DF02188431A494875084658
:1066F000407BF0218843174948730846C07D000954
:106700000001C8750846C07AF02188431149C87253
:106710000846C07A00090001C8720846407E000998
:10672000000148760846007EF02188430949087632
:106730000846007E0009000108760846007B000933
:10674000000108730846C07DF02188430149C875DF
:1067500005B0F0BD7C200020D8180200FFB581B044
:106760000E461746019801287ED10498002826D1AC
:10677000FA480078012822D0F6F72EFAF849884224
:106780001DD3FAF7D5FB00280DD0F648807DF02107
:1067900088437030F34988750846C07C00090001C1
:1067A000C01DC87418E0EF48807DF0218843ED4992
:1067B00088750846C07C00090001C8740CE0E948EF
:1067C000807DF02188437030E64988750846C07C9A
:1067D00000090001C01DC874E248C07CF021884354
:1067E0007030E049C8740846007EF021884370305C
:1067F000DC4908760846807D00090001401C887548
:106800000846407DF02188431030D6494875084637
:10681000407D00090001401C48750846007DF021BC
:1068200088431030CF4908750846007D00090001F3
:10683000401C087533000AF065FA062E261E140C5B
:10684000042FC848007D00090001C01DC549087516
:1068500000BFC448007DF02188437030C1490875ED
:1068600000BFC048407D00E0ADE100090001C01D4F
:10687000BC49487500BFBB48407DF021884370305B
:10688000B849487500BFB748807D00090001C01DA8
:10689000B449887500BF00E000BF00BF049800281D
:1068A0005ED1AE48007801285AD0F6F795F9AC4988
:1068B000884255D3AB48C07FF0218843A949C877A7
:1068C0000846807F0009000188770846407FF02154
:1068D0008843A44948770846007FF0218843A149AE
:1068E00008770846C07DF02188439E49C875084650
:1068F000C07F00090001C8770846807FF0218843E7
:10690000984988770846407F00090001C01D4877F4
:106910000846807EF0218843924988760846807E2A
:106920000009000188760846407E0009000148768B
:106930000846007E0009000108760846007F00092D
:10694000000108770846C07EF02188438549C87653
:106950000846407EF0218843703082494876B8E18D
:1069600064213846F1F7F2FB0546012D07D17D4839
:10697000C07FF021884370307A49C87705E07948B4
:10698000C07FF02188437749C8770A213846F1F75C
:10699000DDFB0A210090F1F7D9FB0D46642F02D3ED
:1069A0007148445D01E07148445DE007C00F002874
:1069B00007D06C48807F00090001C01D69498877B5
:1069C00005E06848807F0009000166498877022059
:1069D0002040002807D06348407FF0218843703072
:1069E0006049487705E05F48407FF02188435D4972
:1069F000487704202040002807D05A48007FF02123
:106A0000884370305749087705E05648007FF021E9
:106A100088435449087708202040002807D051486F
:106A2000C07DF021884370304E49C87505E04D485F
:106A3000C07DF02188434B49C875102020400028B4
:106A400007D04848C07F00090001C01D4549C877EC
:106A500005E04448C07F000900014249C877202072
:106A60002040002807D03F48807FF02188437030C5
:106A70003C49887705E03B48807FF02188433949CD
:106A8000887740202040002807D03648407F000902
:106A90000001C01D3349487705E03248407F0009B6
:106AA0000001304948770A213846F1F74FFB0D467F
:106AB0002D48445DE007C00F002807D02948807E9C
:106AC000F021884370302749887605E02548807E8C
:106AD000F02188432349887602202040002807D0EF
:106AE0002048807E00090001C01D1E49887605E00F
:106AF0001C48807E000900011A4988760420204045
:106B0000002807D01748407E00090001C01D154924
:106B1000487605E01348407E000900011149487697
:106B200008202040002807D00E48007E0009000100
:106B3000C01D0C49087605E00A48007E00090001E6
:106B40000849087610202040002811D00548007F11
:106B500000090001C01D034908770FE01101002062
:106B6000D60B000050210020D8180200EB180200BC
:106B70005948007F0009000157490877202020402C
:106B8000002807D05448C07EF02188437030524915
:106B9000C87605E05048C07EF02188434E49C8764B
:106BA00040202040002807D04B48407EF0218843F9
:106BB0007030494948768CE04748407EF021884350
:106BC0004549487685E04448807D000900014249F6
:106BD00088750846407DF02188433F49487508463E
:106BE000407D0009000148750846007DF02188437A
:106BF000394908750846007D0009000108750846F6
:106C0000C07C00090001C8740846807DF0218843DB
:106C1000314988750846C07CF02188432E49C874E4
:106C20000846007EF02188432B4908760846C07F3D
:106C3000F02188432849C8770846807F0009000171
:106C400088770846407FF0218843234948770846E3
:106C5000007FF0218843204908770846C07DF02155
:106C600088431D49C8750846C07F00090001C877E0
:106C70000846807FF0218843174988770846407F7F
:106C80000009000148770846807EF02188431249B8
:106C900088760846807E0009000188760846407E96
:106CA0000009000148760846007E000900010876C8
:106CB0000846007F0009000108770846C07EF021E1
:106CC00088430549C8760846407EF021884302493A
:106CD000487605B0F0BD00005021002010B50146F7
:106CE000002200200A0EFE4B985CC307DB0F002B2E
:106CF00007D0FC4BDB7FF024A3437033F94CE377E0
:106D000005E0F84BDB7FF024A343F64CE377022346
:106D10000340002B07D0F34BDB7F1B091B01DB1D5E
:106D2000F04CE37705E0EF4BDB7F1B091B01ED4CDB
:106D3000E37704230340002B07D0EA4B9B7F1B091A
:106D40001B01DB1DE74CA37705E0E64B9B7F1B098E
:106D50001B01E44CA37708230340002B09D0E14B2F
:106D600020335B781B091B01DB1DDE4C2034637074
:106D700007E0DC4B20335B781B091B01D94C203426
:106D8000637010230340002B09D0D64B20331B78AF
:106D9000F024A3437033D34C2034237007E0D14B4D
:106DA00020331B78F024A343CE4C203423702023BF
:106DB0000340002B09D0CB4B20331B781B091B0150
:106DC000DB1DC84C2034237007E0C64B20331B78F2
:106DD0001B091B01C34C2034237040230340002BAC
:106DE00007D0C04B9B7FF024A3437033BD4CA377E7
:106DF00005E0BC4B9B7FF024A343BA4CA377FF2351
:106E00001B040B401A0CB64B985CC307DB0F002B1E
:106E100007D0B44B1B7F1B091B01DB1DB14C237733
:106E200005E0B04B1B7F1B091B01AE4C23770223EF
:106E30000340002B07D0AB4BDB7EF024A343703321
:106E4000A84CE37605E0A74BDB7EF024A343A54CDA
:106E5000E37604230340002B07D0A24B9B7EF02453
:106E6000A34370339F4CA37605E09E4B9B7EF0249A
:106E7000A3439C4CA37608230340002B07D0994BD7
:106E80005B7FF024A3437033964C637705E0954B0A
:106E90005B7FF024A343934C637710230340002BC4
:106EA00007D0904B5B7F1B091B01DB1D8D4C63776B
:106EB00005E08C4B5B7F1B091B018A4C6377202309
:106EC0000340002B07D0874B1B7FF024A343703374
:106ED000844C237705E0834B1B7FF024A343814C34
:106EE000237740230340002B07D07E4BDB7E1B091A
:106EF0001B01DB1D7B4CE37605E07A4BDB7E1B0937
:106F00001B01784CE376FF231B020B401A0A744BDB
:106F1000985CC307DB0F002B07D0724B1B7EF0245D
:106F2000A34370336F4C237605E06E4B1B7EF02439
:106F3000A3436C4C237602230340002B07D0694BFC
:106F40001B7E1B091B01DB1D664C237605E0654B90
:106F50001B7E1B091B01634C237604230340002B7B
:106F600007D0604BDB7D1B091B01DB1D5D4CE3750E
:106F700005E05C4BDB7D1B091B015A4CE3750823C4
:106F80000340002B07D0574B9B7E1B091B01DB1DC9
:106F9000544CA37605E0534B9B7E1B091B01514CBF
:106FA000A37610230340002B07D04E4B5B7EF024CA
:106FB000A34370334B4C637605E04A4B5B7EF02471
:106FC000A343484C637620230340002B07D0454B56
:106FD0005B7E1B091B01DB1D424C637605E0414BC8
:106FE0005B7E1B091B013F4C637640230340002B53
:106FF00007D03C4BDB7DF024A3437033394CE37561
:1070000005E0384BDB7DF024A343364CE375CAB270
:10701000334B985CC307DB0F002B07D0314B1B7D34
:10702000F024A34370332F4C237505E02D4B1B7DBB
:10703000F024A3432B4C237502230340002B07D0DD
:10704000284B1B7D1B091B01DB1D264C237505E00E
:10705000244B1B7D1B091B01224C23750423034079
:10706000002B07D01F4BDB7C1B091B01DB1D1D4CBC
:10707000E37405E01B4BDB7C1B091B01194CE3741B
:1070800008230340002B07D0164B9B7CF024A3431E
:107090007033144CA37405E0124B9B7CF024A34383
:1070A000104CA37410230340002B07D00D4B5B7DC5
:1070B000F024A34370330B4C637505E0094B5B7DF3
:1070C000F024A343074C637520230340002B0BD00F
:1070D000044B5B7D1B091B01DB1D024C637509E042
:1070E000D8180200302100200C4B5B7D1B091B01CE
:1070F0000A4C637540230340002B07D0074BDB7C11
:10710000F024A3437033054CE37405E0034BDB7CB0
:10711000F024A343014CE37410BD00003021002093
:1071200000B501287ED1FE4AD278F0239A4370320E
:10713000FB4BDA701A46127912091201D21D1A712C
:107140001A461279F0239A437032F54B1A711A4697
:10715000527912091201D21D5A711A465279F0233E
:107160009A437032EE4B5A711A46D27912091201C3
:10717000D21DDA711A46D279F0239A437032E84B65
:10718000DA711A46527A12091201D21D5A721A463F
:10719000527AF0239A437032E14B5A721A46927A2D
:1071A000F0239A437032DE4B9A721A469278F0239B
:1071B0009A437032DA4B9A701A46D27A1209120147
:1071C000D21DDA721A46527812091201D21D5A7073
:1071D0001A46D27AF0239A437032D14BDA721A46A9
:1071E000203AD27FF0239A437032CD4B203BDA779E
:1071F000CB4A127B12091201D21D20331A731A4690
:10720000203A927F12091201D21D203B9A77C44A7C
:10721000127BF0239A437032C14B1A731A46203AFC
:10722000127F00E0F2E1F0239A437032BC4B203B26
:107230001A77BB4A527B12091201D21D20335A73AE
:107240001A46203AD27E12091201D21D203BDA766C
:10725000B44AD278F0239A437032B24BDA701A46AD
:10726000127B12091201D21D1A731A4612791209E1
:107270001201D21D1A711A46927AF0239A43703283
:10728000A84B9A721A461279F0239A437032A54B92
:107290001A711A46527912091201D21D5A711A46F0
:1072A000927912091201D21D9A711A46127A1209A4
:1072B0001201D21D1A721A46127AF0239A437032C2
:1072C000984B1A721A46527A12091201D21D5A723A
:1072D000934A927912091201521C914B9A711A46E3
:1072E0009279F0239A4310328D4B9A711A46127A92
:1072F00012091201521C1A721A46127AF0239A438A
:107300001032874B1A721A46927A12091201521CD5
:107310009A721A46D27812091201521CDA701A4671
:10732000927812091201521C9A701A465278F02370
:107330009A4310327A4B5A701A461278F0239A43C5
:107340001032774B1A701A46127812091201521C29
:107350001A701A46203AD27F12091201521C203BA1
:10736000DA771A46927FF0239A4310326C4B203B17
:107370009A771A46527FF0239A431032684B203B8B
:107380005A771A46527F12091201521C5A771A462E
:10739000127F12091201521C1A771A46D27EF0236C
:1073A0009A4310325E4B203BDA761A46927EF023E7
:1073B0009A4310325A4B203B9A765A4A127BF0235A
:1073C0009A431032574B1A731A46D27AF0239A43D3
:1073D0001032544BDA721A46D27A12091201521C38
:1073E000DA721A46927A12091201521C9A721A46DD
:1073F000527AF0239A4310324A4B5A721A46527903
:10740000F0239A431032474B5A711A46D279F0232F
:107410009A431032434BDA710B0009F073FC19F3F5
:10742000E9DFD5CBC1B7ADA3998F87786E645A5089
:10743000463E362E261E160EF5003A4AD279F02325
:107440009A437032374BDA7100BF364A5279F023D3
:107450009A437032334B5A7100BF324A527AF0234A
:107460009A4370322F4B5A7200BF2E4A927A1209F9
:107470001201D21D2B4B9A7200BF2A4AD27A1209EE
:107480001201D21D274BDA7200BF264AD27AF023AE
:107490009A437032234BDA7200BF224A127BF023E8
:1074A0009A4370321F4B1A7300BF1D4A203A927ED6
:1074B000F0239A4370321A4B203B9A7600BF184A49
:1074C000203AD27EF0239A437032154B203BDA7675
:1074D00000BF134A203A127F12091201D21D104B2D
:1074E000203B1A7700BF0E4A203A527F1209120140
:1074F000D21D0B4B203B5A7700BF094A203A527FDE
:10750000F0239A437032064B203B5A7700BF044A5F
:10751000203A927FF0239A437032014B203B03E0E4
:107520009C200020702100209A7700BFDC4AD27F87
:1075300012091201D21DDA4BDA7700BFD84A203285
:10754000127812091201D21DD54B20331A7000BFD8
:10755000D34A20321278F0239A437032D04B203332
:107560001A7000BFCE4A20325278F0239A4370320C
:10757000CB4B20335A7000BFC94A2032927812098F
:107580001201D21DC64B20339A7000BFC44A20326C
:10759000D27812091201D21DC14B2033DA7000BF1C
:1075A000BF4A2032927A12091201D21DBC4B2033FD
:1075B0009A7200BFBA4A2032127AF0239A4370328C
:1075C000B74B20331A7200BFB54A2032127A120923
:1075D0001201D21DB24B20331A7200BFB04A2032C2
:1075E0009279F0239A437032AD4B20339A7100BFE9
:1075F000AB4A2032927912091201D21DA84B2033D6
:107600009A7100BF01E0FFE700BF47E1A44A2032C2
:10761000D278F0239A43A24B2033DA701A461279BB
:10762000120912011A711A461279F0239A439C4BDF
:1076300020331A711A465279120912015A711A46E8
:107640005279F0239A43964B20335A711A46D279D5
:1076500012091201DA711A46D279F0239A43904B3B
:107660002033DA711A46527A120912015A721A46F6
:10767000527AF0239A438A4B20335A721A46927AEE
:10768000F0239A43864B20339A721A469278F0235D
:107690009A43834B20339A701A46D27A1209120108
:1076A000DA721A465278120912015A701A46D27AC0
:1076B000F0239A437A4B2033DA72794AD27FF0234F
:1076C0009A43774BDA771A462032127B120912015D
:1076D00020331A73724A927F12091201203B9A7763
:1076E0001A462032127BF0239A436D4B20331A73D3
:1076F0006B4A127FF0239A43694B1A771A4620325D
:10770000527B1209120120335A73654AD27E120944
:107710001201203BDA76634AD278F0239A43614B18
:10772000DA701A46127B120912011A731A4612797C
:10773000120912011A711A46927AF0239A43594B90
:107740009A721A461279F0239A43564B1A711A46C6
:107750005279120912015A711A46927912091201CC
:107760009A711A46127A120912011A721A46127A7C
:10777000F0239A434B4B1A721A46527A120912019D
:107780005A72474A2032927912091201444B20332F
:107790009A711A469279F0239A43414B20339A7199
:1077A0001A46127A120912011A721A46127AF02334
:1077B0009A433B4B20331A721A46927A12091201ED
:1077C0009A721A46D27812091201DA701A46927821
:1077D000120912019A701A465278F0239A43304BDC
:1077E00020335A701A461278F0239A432C4B2033D8
:1077F0001A701A461278120912011A70284AD27F9A
:1078000012091201203BDA771A46927FF0239A433D
:10781000234B9A771A46527FF0239A43204B5A778C
:107820001A46527F120912015A771A46127F12091C
:1078300012011A771A46D27EF0239A43184BDA7651
:107840001A46927EF0239A43154B9A76154A127B7C
:10785000F0239A43134B1A731A46D27AF0239A43B1
:10786000104BDA721A46D27A12091201DA721A46EB
:10787000927A120912019A721A46527AF0239A43A6
:10788000084B5A721A465279F0239A43054B5A71A3
:107890001A46D279F0239A43024BDA7100BD0000F8
:1078A0007C20002070210020F7B582B006461746E4
:1078B000002500200190002E7ED1F9F753FA05280B
:1078C0005FD1F9F735FB00280DD0FA484079F02157
:1078D00088437030F74948710846807800090001F4
:1078E000C01D88700AE0F3484079F0218843F149CF
:1078F000487108468078000900018870ED48C07919
:1079000000090001EB49C8710846807900090001AF
:107910008871084640790009000148710846007ADC
:10792000F0218843E34908720846007A0009000103
:1079300008720846C079F0218843DE49C8710846BC
:10794000C07800090001C87008468078F02188439B
:10795000D849887008464078F0218843D549487056
:10796000084640780009000148700846007900097F
:10797000000108710846C078F0218843CD49C870DD
:1079800029E2CC484079F02188437030C9494871D8
:107990000846807800090001C01D88700846C0793B
:1079A00000090001C871084680790009000188714A
:1079B00008464079000900E034E0000148710846BB
:1079C000007AF0218843BB4908720846007A000912
:1079D000000108720846C079F0218843B549C87192
:1079E0000846C07800090001C87008468078F02178
:1079F0008843B049887008464078F0218843AD49F3
:107A0000487008464078000900014870084600792F
:107A10000009000108710846C078F0218843A54993
:107A2000C870ADE7012E5FD1F9F782FA00280DD0BA
:107A3000A0484079F021884370309E49487108463B
:107A4000807800090001C01D88700AE099484079DB
:107A5000F021884397494871084680780009000161
:107A600088709448C079000900019249C87108469D
:107A700080790009000188710846407900090001F9
:107A800048710846007AF02188438A4908720846FE
:107A9000007A0009000108720846C079F021884385
:107AA0008449C8710846C07800090001C8700846BA
:107AB0008078F02188437F49887008464078F0211B
:107AC00088437C49487008464078000900014870A6
:107AD000084600790009000108710846C078F021C5
:107AE00088437449C870EAE3022E7DD1F9F73AF968
:107AF00005287AD1F9F71CFA002877D0012F76D122
:107B00000A210398F0F722FB0546F9F749F9002806
:107B100002D16948445D01E06848445DE007C00F58
:107B2000002807D06348C07900090001C01D6149E1
:107B3000C87105E05F48C079000900015D49C8715E
:107B400002202040002807D05A488079000900010F
:107B5000C01D5849887105E0564880790009000128
:107B60005449887104202040002807D051484079AA
:107B700000090001C01D4F49487105E04D4840799A
:107B8000000900014B49487108202040002807D017
:107B90004848007AF021884370304649087205E071
:107BA0004448007AF021884342490872102020405E
:107BB000002807D03F48007A00090001C01D3D4958
:107BC000087205E03B48007A000900013949087253
:107BD0002020204000280BD03648C079F02188436F
:107BE00070303449C87109E0AEE242E1F4E0A4E04B
:107BF0003048C079F02188432E49C8714020204088
:107C0000002807D02B484079F0218843703029495B
:107C1000487105E027484079F0218843254948719B
:107C20000A210398F0F792FA0D462348445DE007D5
:107C3000C00F002807D01F48C07800090001C01DF0
:107C40001C49C87005E01B48C078000900011949AB
:107C5000C87002202040002807D016488078F02104
:107C6000884370301349887005E012488078F0210D
:107C700088431049887004202040002807D00D4810
:107C80004078F021884370300A49487005E009487F
:107C90004078F02188430749487008202040002898
:107CA0000ED00448407800090001C01D0149487009
:107CB0000CE00000BC200020D8180200EB180200E5
:107CC000FE48407800090001FC494870102020401F
:107CD000002807D0F948007900090001C01DF749C4
:107CE000087105E0F548007900090001F3490871C1
:107CF00020202040002807D0F048C078F021884399
:107D00007030EE49C87005E0EC48C078F021884337
:107D1000EA49C87040202040002807D0E748807812
:107D200000090001C01DE5498870C8E2E348807879
:107D300000090001E1498870C1E2E0484079F02182
:107D400088437030DD494871084680780009000199
:107D5000C01D88700846C07900090001C871084636
:107D60008079000900018871084640790009000106
:107D700048710846007AF0218843D04908720846C5
:107D8000007A0009000108720846C079F021884392
:107D9000CA49C8710846C07800090001C870084681
:107DA0008078F0218843C549887008464078F021E2
:107DB0008843C2494870084640780009000148706D
:107DC000084600790009000108710846C078F021D2
:107DD0008843BA49C87072E2B8484079F0218843B4
:107DE000B649487108468078000900018870084645
:107DF000C07900090001C8710846807900090001B6
:107E00008871084640790009000148710846007AE7
:107E1000F0218843A94908720846007A0009000148
:107E200008720846C079F0218843A449C871084601
:107E3000C07800090001C87008468078F0218843A6
:107E40009E49887008464078F02188439B494870D5
:107E5000084640780009000148700846007900098A
:107E6000000108710846C078F02188439349C87022
:107E700025E2012F73D10A210398F0F767F905462F
:107E8000F8F78EFF002802D18D48445D01E08D484F
:107E9000445DE007C00F002807D08848C07900097A
:107EA0000001C01D8549C87105E08448C0790009FA
:107EB00000018249C87102202040002807D07F4875
:107EC000807900090001C01D7C49887105E07B486C
:107ED0008079000900017949887104202040002838
:107EE00007D07648407900090001C01D73494871E8
:107EF00005E0724840790009000170494871082086
:107F00002040002807D06D48007AF0218843703067
:107F10006A49087205E06948007AF0218843674998
:107F2000087210202040002807D06448007A000919
:107F30000001C01D6149087205E06048007A00092F
:107F400000015E49087220202040002808D05B48CC
:107F5000C079F021884370305849C87106E09DE02F
:107F60005648C079F02188435449C87140202040C8
:107F7000002807D051484079F021884370304F499C
:107F8000487105E04D484079F02188434B494871DC
:107F90000A210398F0F7DAF80D464948445DE007F6
:107FA000C00F002807D04548C07800090001C01D57
:107FB0004249C87005E04148C078000900013F49C6
:107FC000C87002202040002807D03C488078F0216B
:107FD000884370303949887005E038488078F0214E
:107FE00088433649887004202040002807D0334851
:107FF0004078F021884370303049487005E02F48C0
:108000004078F02188432D494870082020400028FE
:1080100007D02A48407800090001C01D2749487050
:1080200005E02648407800090001244948701020E6
:108030002040002807D02148007900090001C01D18
:108040001E49087105E01D480079000900011B491F
:10805000087120202040002807D01848C078F0215F
:10806000884370301549C87005E01448C078F02185
:1080700088431249C87040202040002807D00F488C
:10808000807800090001C01D0C49887017E10B4879
:108090008078000900010949887010E1074840799B
:1080A000F0218843703005494871084680780009FE
:1080B0000001C01D88700846C07905E0BC20002082
:1080C000D8180200EB18020000090001C871084628
:1080D0008079000900018871084640790009000193
:1080E00048710846007AF0218843764908720846AC
:1080F000007A0009000108720846C079F02188431F
:108100007049C8710846C07800090001C870084667
:108110008078F02188436B49887008464078F021C8
:108120008843684948700846407800090001487053
:10813000084600790009000108710846C078F0215E
:1081400088436049C870BAE0032E9FD1F8F70AFE51
:1081500005285FD1F8F7ECFE00280DD0594840798A
:10816000F0218843703057494871084680780009EB
:108170000001C01D88700AE052484079F021884310
:1081800050494871084680780009000188704D48C0
:10819000C079000900014B49C8710846807900097F
:1081A00000018871084640790009000148710846BD
:1081B000007AF0218843434908720846007A000992
:1081C000000108720846C079F02188433D49C87112
:1081D0000846C07800090001C87008468078F02180
:1081E00088433849887008464078F02188433549EB
:1081F0004870084640780009000148700846007938
:108200000009000108710846C078F02188432D4913
:10821000C87054E02B480079F02188437030294918
:10822000087108464079F02188437030254948712B
:108230000846807800090001C01D88700846C07992
:1082400000090001C87108468079000900018871A1
:10825000084640790009000148710846007AF0217B
:108260008843184908720846007A0009000108721C
:108270000846C079F02188431249C8710846C07881
:1082800000090001C87008468078F02188430D4934
:10829000887008464078F02188430A4948700846AB
:1082A0004078000900014870084600790009000183
:1082B00008710846C078F02188430249C87005B0AB
:1082C000F0BD0000BC20002070B505460C46012D15
:1082D0007ED1B248407D00090001C01DAF494875FC
:1082E0000846007DF02188431030AC4908750846E7
:1082F000007D00090001401C08750846C07CF02183
:1083000088431030A549C8740846807CF021884312
:108310001030A24988740846807C00090001401C86
:108320008874F8F75FFE022803D0F8F75BFE012897
:108330006CD19B480078012868D0F4F74DFC99492E
:10834000884263D3F8F7F4FD00282FD09348007DCE
:10835000F02188437030914908750846007D000976
:108360000001C01D08750846C07CF02188437030AC
:108370008A49C8740846807CF02188437030874958
:1083800088740846807C00090001C01D8874084676
:10839000407DF02188437030804948750846407C14
:1083A000F021884370307D494874F6E07B48007DB9
:1083B000F02188431030794908750846007D00098E
:1083C0000001401C08750846C07CF021884300E08D
:1083D000B6E010307149C8740846807CF0218843AB
:1083E00010306E4988740846807C00090001401CEA
:1083F00088740846407DF0218843684948750846DE
:10840000407CF021884365494874C6E0F8F794FC45
:10841000002825D1F4F7E0FB62491E3188421FD3C2
:10842000F8F786FD00280ED05C48407DF021884397
:1084300070305A4948750846407CF02188437030B6
:10844000564948741AE05548407DF0218843534905
:1084500048750846407CF0218843504948740DE037
:108460004E48407DF021884370304C49487508469D
:10847000407CF0218843703048494874F8F75CFC30
:1084800001282BD146480078012827D0F4F7A4FB17
:1084900044491E31884221D34048407DF021884321
:1084A00070303E4948750846407CF0218843703062
:1084B0003A494874F8F73CFD002807D03748007D5A
:1084C000F021884370303549087566E03348007DF7
:1084D000F02188431030314908755EE0230008F030
:1084E00011FC062C241C140C042D2C48807C000943
:1084F0000001C01D2949887400BF2848807CF021F4
:10850000884370302549887400BF2448C07CF0211E
:10851000884370302149C87400BF2048007D00099D
:108520000001C01D1D49087500BF1C48007DF021D9
:10853000884370301949087500BF00E000BF2CE087
:108540001648407DF0218843144948750846007D4F
:10855000F0218843114908750846007D0009000193
:1085600008750846C07CF02188430C49C874084649
:10857000807CF0218843094988740846807C000982
:10858000000188740846407D0009000148750846CE
:10859000407CF02188430149487470BD9C20002034
:1085A00011010020B80B000030B50246002901D1AE
:1085B000002000E00720130008F0A4FB0F09141F9F
:1085C0002B3743505D67727C88929FA9B500574B4B
:1085D0005B7EF024A3430401F0252C402343534C3D
:1085E0006376A1E0524B9B79F024A3430401F0256C
:1085F0002C4023434E4CA37196E04D4B2033DB7946
:108600001B091B010407240F2343494C2034E37149
:108610008AE0464B2033DB7C1B091B010407240F37
:108620002343424C2034E3747EE0404B40331B78BC
:108630001B091B010407240F23433C4C40342370C7
:1086400072E03A4B2033DB7FF024A3430401F02592
:108650002C402343354C2034E37765E0334B203303
:108660005B7BF024A3430401F0252C4023432F4CD3
:108670002034637358E02E4B9B791B091B010407C0
:10868000240F23432A4CA3714EE0294B9B7CF024FA
:10869000A3430401F0252C402343254CA37443E05D
:1086A000234BDB7E1B091B010407240F2343204CB3
:1086B000E37639E01D4B2033DB7F1B091B010407E8
:1086C000240F2343194C2034E3772DE0174B9B7E76
:1086D0001B091B010407240F2343144CA37623E03A
:1086E000134B20339B79F024A3430401F0252C4045
:1086F00023430F4C2034A37116E00D4BDB7D1B0987
:108700001B010407240F2343094CE3750CE0074BBE
:1087100020335B7C1B091B010407240F2343034CFC
:108720002034637400E000BF00BF30BD7C20002017
:1087300050210020F7B582B00746154600260024D8
:10874000FE480078012804D0F4F746FAFC49884234
:1087500079D2FC48407CF02188437030F949487454
:108760000846807C00090001C01D88740846007D11
:1087700000090001C01D08750846007DF0218843EE
:108780007030F04908750846807CF02188437030CD
:10879000EC4988740846C07C00090001C01DC874FB
:1087A0000846C07CF02188437030E649C87408460A
:1087B000407C00090001C01D48740846407D000946
:1087C0000001C01D48750846407DF0218843703087
:1087D000DC4948750846007CF02188437030D9494F
:1087E00008740846007C00090001C01D0874084692
:1087F000C07BF02188437030D249C873FF220A2120
:108800000020FAF7A3FFFF2213210020FAF79EFFB2
:10881000FF2211210020FAF799FFFF2212210020E8
:10882000FAF794FFFF220E210020FAF78FFFFF22B4
:108830000F210020FAF78AFFFF2210210020FAF70B
:1088400085FFF4E3FFE7039836283DD019DC0828BC
:108850007ED007DC801E030008F054FA0635A8FC21
:10886000FBFAF97E102874D006DC092872D00D2896
:1088700071D00E2870D1FDE333286ED03428F9D1A1
:1088800070E13F286AD00FDC3738082864D24300F3
:108890007B449B885B009F448A009702FF025F0035
:1088A0005F006503CB0318004E287BD006DC402810
:1088B00079D0412878D04D28DCD1BBE14F2874D045
:1088C0005028D7D14FE100BF00BF9E48407CF02127
:1088D00088439C4948740846807C000900018874DC
:1088E0000846007D00090001C01D08750846007D8E
:1088F000F02188437030934908750846807CF02148
:108900008843904988740846C07C00090001C01D56
:10891000C8740846C07CF02188438A49C874084658
:10892000407C0009000148740846407D00090001B0
:1089300048750846407DF0218843824948750846BD
:10894000007CF02188437F4908740846007C06E0DB
:10895000A1E2FDE337E2D2E3FBE394E028E0000983
:10896000000108740846C07BF02188437549C8732C
:10897000FF220A210020FAF7E9FEFF22132100203E
:10898000FAF7E4FE00220E211046FAF7DFFE00227D
:108990000F211046FAF7DAFE002210211046FAF7EE
:1089A000D5FE77E2ABE110E2DDE26DE000BF00BF93
:1089B0006448407CF0218843624948740846807CC2
:1089C0000009000188740846007D00090001C01DEF
:1089D00008750846007DF0218843703059490875B4
:1089E0000846807CF0218843564988740846C07C3C
:1089F00000090001C8740846C07CF0218843514931
:108A0000C8740846407C0009000148740846407D4F
:108A100000090001C01D48750846407DF0218843CB
:108A2000484948750846007CF02188434549087448
:108A30000846007C0009000108740846C07BF0214C
:108A400088434049C873FF220A21002003E055E112
:108A5000EFE086E016E0FAF779FEFF22132100200E
:108A6000FAF774FE00220E211046FAF76FFE00227C
:108A70000F211046FAF76AFE002210211046FAF77D
:108A800065FE8EE700BF00BF2E48407CF021884382
:108A90002C4948740846807C00090001C01D887478
:108AA0000846007D00090001C01D08750846007DCC
:108AB000F02188437030234908750846807CF021F6
:108AC000884370301F4988740846C07C0009000143
:108AD000C8740846C07CF02188431A49C874084607
:108AE000407C0009000148740846407D00090001EF
:108AF00048750846407DF02188431249487508466C
:108B0000007CF02188430F4908740846007C000966
:108B1000000108740846C07BF02188430949C873E6
:108B2000FF220A210020FAF711FEFF221321002064
:108B3000FAF70CFE00220E21104605E0110100207C
:108B4000D60B0000BC200020FAF700FE00220F2107
:108B50001046FAF7FBFD002210211046FAF7F6FD49
:108B60001FE700BF00BFFE48407CF0218843FC495E
:108B700048740846807C00090001C01D88740846BE
:108B8000007D00090001C01D08750846007DF02128
:108B900088437030F24908750846807CF02188438C
:108BA000EF4988740846C07C00090001C874084673
:108BB000C07CF0218843EA49C8740846407C00091B
:108BC0000001C01D48740846407D00090001487539
:108BD0000846407DF0218843E14948750846007CFD
:108BE000F0218843DE4908740846007C0009000132
:108BF00008740846C07BF0218843D949C873FF2216
:108C00000A210020FAF7A2FDFF2213210020FAF723
:108C10009DFD00220E211046FAF798FD00220F213B
:108C20001046FAF793FD002210211046FAF78EFD48
:108C3000F6E300BFCA48407CF0218843C849487425
:108C40000846807C0009000188740846007D000900
:108C5000000108750846007DF02188437030C04946
:108C600008750846807CF0218843BD498874084611
:108C7000C07C00090001C8740846C07CF02188430C
:108C80007030B749C8740846407C00090001487438
:108C90000846407D0009000148750846407DF021E6
:108CA0008843AF4948750846007CF0218843AC49A9
:108CB00008740846007C0009000108740846C07B5F
:108CC000F0218843A649C873FF220A210020FAF741
:108CD0003DFDFF2213210020FAF738FD00220E216E
:108CE0001046FAF733FD00220F211046FAF72EFD49
:108CF000002210211046FAF729FD91E300BF9848A1
:108D0000407CF0218843964948740846807C0009DD
:108D1000000188740846007D0009000108750846B6
:108D2000007DF021884370308D4908750846807CAD
:108D3000F02188438A4988740846C07C00090001F4
:108D4000C8740846C07CF02188438549C874084629
:108D5000407C0009000148740846407D000900017C
:108D600048750846407DF021884370307C4948753D
:108D70000846007CF0218843794908740846007C45
:108D80000009000108740846C07BF021884374493B
:108D9000C873FF220A210020FAF7D8FCFF22132112
:108DA0000020FAF7D3FC00220E211046FAF7CEFC81
:108DB00000220F211046FAF7C9FC002210211046AC
:108DC000FAF7C4FC2CE300BF00BF6548407CF021EB
:108DD00088437030624948740846807C000900016D
:108DE000C01D88740846007D00090001C01D08757B
:108DF0000846007DF02188437030594908750846BF
:108E0000807CF0218843564988740846C07C00095C
:108E10000001C8740846C07CF02188435049C874DA
:108E20000846407C0009000148740846407D00095E
:108E3000000148750846407DF0218843484948753F
:108E40000846007CF0218843454908740846007CA8
:108E50000009000108740846C07BF021884340499E
:108E6000C873FF220A210020FAF770FCFF221321A9
:108E70000020FAF76BFC00220E211046FAF766FC80
:108E800000220F211046FAF761FC00221021104643
:108E9000FAF75CFCC4E200BF3148407CF021884313
:108EA0002F4948740846807C0009000188740846F0
:108EB000007D0009000108750846007DF021884307
:108EC0007030274908750846807CF0218843244982
:108ED00088740846C07C00090001C8740846C07C3C
:108EE000F021884370301E49C8740846407C000950
:108EF000000148740846407D000900014875084695
:108F0000407DF0218843164948750846007CF021D1
:108F10008843134908740846007C0009000108745E
:108F20000846C07BF02188430D49C873FF220A21FF
:108F30000020FAF70BFCFF2213210020FAF706FCB1
:108F400000220E211046FAF701FC00220F211046E4
:108F5000FAF7FCFB002210211046FAF7F7FB5FE25C
:108F6000BC20002000BFFC48407CF0218843FA4927
:108F700048740846807C0009000188740846007D1A
:108F80000009000108750846007DF0218843703013
:108F9000F14908750846807CF0218843EE498874C1
:108FA0000846C07C00090001C8740846C07CF02156
:108FB0008843E949C8740846407C000900014874A8
:108FC0000846407D0009000148750846407DF021B3
:108FD00088437030E04948750846007CF02188439A
:108FE000DD4908740846007C000900010874084641
:108FF000C07BF0218843D849C873FF220A21002092
:10900000FAF7A4FBFF2213210020FAF79FFB0022AE
:109010000E211046FAF79AFB00220F211046FAF7AC
:1090200095FB002210211046FAF790FBF8E1F8E1D9
:10903000C948407CF02188437030C74948740846CD
:10904000807C00090001C01D88740846007D00096D
:109050000001C01D08750846007DF0218843BE4907
:1090600008750846807CF0218843BB49887408460F
:10907000C07C00E0A9E000090001C8740846C07C7B
:10908000F0218843B449C8740846407C00090001B7
:1090900048740846407D0009000148750846407D37
:1090A000F0218843AC4948750846007CF02188438C
:1090B000A94908740846007C0009000108740846A4
:1090C000C07BF0218843A449C873FF220A210020F5
:1090D000FAF73CFBFF2213210020FAF737FB0022AE
:1090E0000E211046FAF732FB00220F211046FAF744
:1090F0002DFB002210211046FAF728FB90E196483C
:10910000407CF0218843944948740846807C0009DB
:10911000000188740846007D0009000108750846B2
:10912000007DF02188438C4908750846807CF02139
:109130008843894988740846C07C00090001C874C6
:109140000846C07CF02188438349C874084601E082
:109150009EE003E1407C0009000148740846407D20
:109160000009000148750846407DF02188437A498E
:1091700048750846007CF021884377490874084602
:10918000007C0009000108740846C07BF021884378
:1091900070307149C87300220A211046FAF7D6FAD6
:1091A000002213211046FAF7D1FAFF220E210020E7
:1091B000FAF7CCFA00220F211046FAF7C7FA00227C
:1091C00010211046FAF7C2FA2AE16348407CF021E8
:1091D0008843614948740846807C0009000188740E
:1091E0000846007D0009000108750846007DF02151
:1091F0008843594908750846807CF02188435649C0
:1092000088740846C07C00090001C8740846C07C08
:10921000F02188435049C8740846407C0009000189
:1092200048740846407D0009000148750846407DA5
:10923000F0218843484948750846007CF02188435E
:10924000454908740846007C00090001C01D0874E7
:109250000846C07BF02188433F49C87300220A2199
:109260001046FAF773FA002213211046FAF76EFA45
:1092700000220E211046FAF769FAFF220F21002082
:10928000FAF764FA002210211046FAF75FFAC7E0F5
:109290003148407CF02188432F4948740846807C3F
:1092A0000009000188740846007D00090001087566
:1092B0000846007DF0218843274908750846807CD0
:1092C000F0218843244988740846C07C00090001C5
:1092D000C8740846C07CF02188431F49C8740846FA
:1092E000407C0009000148740846407D00090001E7
:1092F00048750846407DF02188431749487508465F
:10930000007CF02188437030134908740846007CC3
:109310000009000108740846C07BF02188430E490B
:10932000C87300220A211046FAF710FA002213210E
:109330001046FAF70BFA00220E211046FAF706FA49
:1093400000220F211046FAF701FAFF221021002017
:10935000FAF7FCF964E00000BC200020FD48407CE6
:10936000F0218843FB4948740846807C00090001CD
:1093700088740846007D0009000108750846007DD4
:10938000F0218843F34908750846807CF021884322
:10939000F04988740846C07C00090001C87408467A
:1093A000C07CF0218843EB49C8740846407C000922
:1093B000000148740846407D0009000148750846D0
:1093C000407DF0218843E34948750846007CF02140
:1093D0008843E04908740846007C000900010874CD
:1093E0000846C07BF0218843DA49C87300220A216D
:1093F0001046FAF7ABF9002213211046FAF7A6F946
:1094000000220E211046FAF7A1F900220F21104682
:10941000FAF79CF9002210211046FAF797F900BFDD
:1094200000BF002F03D0CC48007A002808D1F3F702
:10943000D3FBCA49884203D3C9480078012872D1B6
:10944000FF2211210020FAF781F9FF2212210020CA
:10945000FAF77CF9C2480078012804D0F3F7BCFB86
:10946000BE49884216D2BF48807BF02188437030C5
:10947000BC498873084640300078F021884370303A
:10948000B849403108700846007800090001C01D45
:1094900008702DE07D20C000854214D2B148807B49
:1094A000F0218843AF498873084640300078F021A6
:1094B00088437030AB494031087008460078000995
:1094C0000001087014E0A748807BF02188437030C9
:1094D000A4498873084640300078F0218843A149A8
:1094E000403108700846007800090001C01D08706E
:1094F0007D20C000854205D201462846EEF726FEB3
:10950000064604E098492846EEF720FE06469448B1
:109510000078012804D0F3F75FFB9049884203D21A
:109520009248845D02E0A0E29148845DE007C00FAC
:10953000002809D08B484030C07800090001C01DC8
:1095400088494031C87007E086484030C07800093B
:10955000000184494031C87002202040002807D013
:109560008048C07900090001C01D7E49C87105E02E
:109570007C48C079000900017A49C8710420204064
:10958000002807D07748807900090001C01D75497F
:10959000887105E07348807900090001714988717C
:1095A00008202040002807D06E484079F0218843E9
:1095B00070306C49487105E06A484079F021884371
:1095C0006849487110202040002807D0654840793C
:1095D00000090001C01D6349487105E061484079F8
:1095E000000900015F49487120202040002807D071
:1095F0005C480079F021884370305A49087105E0D1
:1096000058480079F021884356490871402020408D
:10961000002807D053488079F021884370305149A1
:10962000887105E04F488079F02188434D49887161
:109630007D20C000854213D264212846EEF786FDC6
:10964000064647480078012804D0F3F7C5FA434995
:10965000884202D24548845D23E04548845D20E08D
:10966000642128463230EEF771FD7D21C90000905B
:10967000EEF76CFD019164210198EEF767FD064657
:109680003C48854208D236480078012804D0F3F7D8
:10969000A3FA3249884202D23448845D01E034485A
:1096A000845DE007C00F002809D02E484030807844
:1096B000F021884370302B494031887007E02948F9
:1096C00040308078F021884326494031887002205C
:1096D0002040002807D02348807A00090001C01DDF
:1096E0002049887205E01F48807A000900011D4961
:1096F000887204202040002807D01A48407A0009C8
:109700000001C01D1749487205E01648407A00095B
:1097100000011449487208202040002807D0114851
:10972000007AF021884370300E49087205E00D4838
:10973000007AF02188430B4908721020204000284D
:109740001AD00848007A00090001C01D05490872B6
:1097500018E00000BC200020280A0020D60B0000E2
:109760001101002030210020A0860100D81802003D
:10977000EB18020010270000FE48007A00090001E3
:10978000FC49087220202040002807D0F948C07901
:10979000F02188437030F749C87105E0F548C07979
:1097A000F0218843F349C87140202040002807D0A9
:1097B000F048407AF02188437030EE49487205E065
:1097C000EC48407AF0218843EA4948727D20C00085
:1097D000854219D20A212846EEF7B8FC0A210190E9
:1097E000EEF7B4FC0E460A2D08D2E34800780128B3
:1097F00004D0F3F7F1F9E149884202D2E048845DF0
:1098000012E0E048845D0FE0642128463230EEF734
:109810009DFC0A210090EEF799FC0A210190EEF7D9
:1098200095FC0E46D6498C5DE007C00F002809D094
:10983000D0484030807800090001C01DCD4940313A
:10984000887007E0CB484030807800090001C949A2
:109850004031887002202040002807D0C548807B16
:1098600000090001C01DC349887305E0C148807B21
:1098700000090001BF49887304202040002807D058
:10988000BC48407B00090001C01DBA49487305E08F
:10989000B848407B00090001B649487308202040C1
:1098A000002807D0B348007BF02188437030B149CD
:1098B000087305E0AF48007BF0218843AD49087389
:1098C00010202040002807D0AA48C07A00090001D3
:1098D000C01DA849C87205E0A648C07A0009000169
:1098E000A449C87220202040002807D0A148807ACF
:1098F000F021884370309F49887205E09D48807A46
:10990000F02188439B49887240202040002807D0DE
:109910009848407BF021884370309649487305E0B1
:109920009448407BF0218843924948737D20C000D1
:10993000854207D20A212846EEF708FC0E469048D9
:10994000845D0BE0642128463230EEF7FFFB0A21EC
:109950000190EEF7FBFB0E4689498C5DE007C00FD6
:10996000002809D0834840304078F0218843703087
:1099700080494031487007E07E4840304078F0210F
:1099800088437C494031487002202040002809D09B
:1099900078484030407800090001C01D75494031C9
:1099A000487007E073484030407800090001714971
:1099B0004031487004202040002807D06D48007CCA
:1099C000F021884370306B49087405E06948007CD9
:1099D000F02188436749087408202040002807D0F8
:1099E0006448007C00090001C01D6249087405E05C
:1099F0006048007C000900015E4908741020204086
:109A0000002807D05B48C07BF0218843703059495B
:109A1000C87305E05748C07BF02188435549C87397
:109A200020202040002807D05248C07B00090001B8
:109A3000C01D5049C87305E04E48C07B00090001B5
:109A40004C49C87340202040002807D04948407C3A
:109A500000090001C01D47494874ECE04548407CBE
:109A60000009000143494874E5E000220A2110463C
:109A7000F9F76CFE002213211046F9F767FE002269
:109A800011211046F9F762FE002212211046F9F763
:109A90005DFE00220E211046F9F758FE00220F212C
:109AA0001046F9F753FE002210211046F9F74EFE3A
:109AB00030484030C078000900012E494031C8705C
:109AC0002C48C079000900014039C87108468079E6
:109AD00000090001887108464079F0218843254932
:109AE000487108464079000900014871084600792C
:109AF000F02188431F49087108468079F021884386
:109B00001C498871084640308078F0218843194903
:109B1000403188701748807A000900014039887206
:109B20000846407A0009000148720846007AF02190
:109B30008843104908720846007A0009000108723B
:109B40000846C079F02188430A49C8710846407A1E
:109B5000F021884307494872084640308078000960
:109B60000001403188700348807B000900014039C2
:109B7000887309E03021002011010020D60B00007D
:109B8000D8180200EB1802000846407B00090001CB
